:020000040000FA
:100000000002040000000000C0A10000C0A1000028
:10001000C0A10000C0A10000C0A10000C0A100005C
:10002000C0A10000C0A10000C0A10000C0A100004C
:10003000C0A10000C0A10000C0A10000C0A100003C
:10004000C0A10000C0A10000C0A10000C0A100002C
:10005000C0A100008C700000B2700000C0A10000C0
:10006000C0A10000C0A10000C0A10000C0A100000C
:10007000C0A10000C0A10000C0A10000C0A10000FC
:10008000C0A10000C0A10000C0A10000C0A10000EC
:10009000C0A10000C0A10000C0A10000C0A10000DC
:1000A000C0A10000C0A10000C0A10000C0A10000CC
:1000B000C0A10000C0A10000C0A10000C0A10000BC
:1000C000C0A10000C0A10000C0A10000C0A10000AC
:1000D000C0A10000C0A10000C0A10000C0A100009C
:1000E000C0A10000C0A10000C0A10000C0A100008C
:1000F000C0A10000C0A10000C0A10000C0A100007C
:10010000C0A10000C0A10000C0A10000C0A100006B
:10011000C0A10000C0A10000C0A10000C0A100005B
:10012000C0A10000C0A10000C0A10000C0A100004B
:10013000C0A10000C0A10000C0A10000C0A100003B
:10014000C0A10000C0A10000C0A10000C0A100002B
:10015000C0A10000C0A10000C0A10000C0A100001B
:10016000C0A10000C0A10000C0A10000C0A100000B
:10017000C0A10000C0A10000C0A10000C0A10000FB
:10018000C0A10000C0A10000C0A10000C0A10000EB
:10019000C0A10000C0A10000C0A10000C0A10000DB
:1001A000C0A10000C0A10000C0A10000C0A10000CB
:1001B000C0A10000C0A10000C0A10000C0A10000BB
:1001C000C0A10000C0A10000C0A10000C0A10000AB
:1001D000C0A10000C0A10000C0A10000C0A100009B
:1001E000C0A10000C0A10000C0A10000C0A100008B
:1001F000C0A10000C0A10000C0A10000C0A100007B
:10020000FFFFFF00FFFFFF00C0A10000C0A1000032
:10021000C0A10000C0A10000C0A10000C0A100005A
:10022000C0A10000C0A10000C0A10000C0A100004A
:10023000C0A10000C0A10000C0A10000C0A100003A
:10024000C0A10000C0A10000C0A10000C0A100002A
:10025000C0A100008C700000B2700000C0A10000BE
:10026000C0A10000C0A10000C0A10000C0A100000A
:10027000C0A10000C0A10000C0A10000C0A10000FA
:10028000C0A10000C0A10000C0A10000C0A10000EA
:10029000C0A10000C0A10000C0A10000C0A10000DA
:1002A000C0A10000C0A10000C0A10000C0A10000CA
:1002B000C0A10000C0A10000C0A10000C0A10000BA
:1002C000C0A10000C0A10000C0A10000C0A10000AA
:1002D000C0A10000C0A10000C0A10000C0A100009A
:1002E000C0A10000C0A10000C0A10000C0A100008A
:1002F000C0A10000C0A10000C0A10000C0A100007A
:10030000C0A10000C0A10000C0A10000C0A1000069
:10031000C0A10000C0A10000C0A10000C0A1000059
:10032000C0A10000C0A10000C0A10000C0A1000049
:10033000C0A10000C0A10000C0A10000C0A1000039
:10034000C0A10000C0A10000C0A10000C0A1000029
:10035000C0A10000C0A10000C0A10000C0A1000019
:10036000C0A10000C0A10000C0A10000C0A1000009
:10037000C0A10000C0A10000C0A10000C0A10000F9
:10038000C0A10000C0A10000C0A10000C0A10000E9
:10039000C0A10000C0A10000C0A10000C0A10000D9
:1003A000C0A10000C0A10000C0A10000C0A10000C9
:1003B000C0A10000C0A10000C0A10000C0A10000B9
:1003C000C0A10000C0A10000C0A10000C0A10000A9
:1003D000C0A10000C0A10000C0A10000C0A1000099
:1003E000C0A10000C0A10000C0A10000C0A1000089
:1003F000C0A10000C0A10000C0A10000C0A1000079
:10040000EF272200007F220000018800000000008A
:100410000C000700A0DE28000100200011000700EA
:10042000000020000000E000020032000000020096
:100430000000000046A10200000000000040DA00B9
:100440000000FE004440A900403120000000E00010
:100450000300320000002000A00188004440A800F2
:100460000000060091018800800078000000EB0089
:1004700015003700E280400032A0B4009101BA00BC
:10048000E280400032A0B4009102BA00E280400055
:1004900032A0B4000002EB00472BDE00F507B200EB
:1004A000602CE10004003A000059EB008301E900F0
:1004B000FDFF3E00040037006128E100010032002A
:1004C0000082EB00040007001101BA000200E00006
:1004D000E8FF3A00000006003159BA008301E90044
:1004E0000C0032002159BA008301E90008003200F3
:1004F0000400E00003003A00E280400032A0B400B3
:10050000F5FF370011D9BA008301E900FAFF3A007C
:100510008100E800E180400032A0B4000000060045
:1005200000000000000000000000000000000000CB
:1005300000000000000000000000000000000000BB
:1005400000000000000000000000000000000000AB
:10055000000000000000000000000000000000009B
:1007F000889FBE008A9FBE00010578000100E000CE
:100800000400350008003C000000E0002000320039
:100810000500370060001000E080180002003B0077
:1008200001F02C001A0037000004BE006011B8006F
:100830006B0920000982CF00020039000882CF0036
:100840000441B000694252000E00320008003B0033
:1008500082817100610164008904D1000884D300A1
:100860008B05E8000442E800F9FF3A000500370074
:100870000804440089844C008B05E9000442E90027
:10088000FBFF3A002C0107000AF0A70001F0A000CE
:100890004F05BE004F04BE0000000600F4FF2F000D
:1008A0004B0137001400200049013700889FBE002B
:1008B0008A9FBE008C1F780060010700670133002B
:1008C00003866C006450E1002E0032006420E100D9
:1008D000330032006150E1002F0032006120E1005E
:1008E0003100320085855500EB07B000090020007B
:1008F00008042000050037000804440089844C00E7
:100900000A0031000603430087834B0000015300B7
:1009100081815B00F8FF33000203BE000800A000E5
:100920000804440089844C00F6FF3900C639DD0014
:100930008301730001003200130020008904D100FC
:100940000884D3000998A300050032000800A7001E
:100950000300A0008904D1000884D3008B05E800BF
:100960008904D1000884D3000001EB000281D20089
:10097000F100070001F0A1000CF0A70001F0A000B9
:100980003F0137006420E100410132000801BE0050
:100990000200BE00F7FF37006120E1003C01320099
:1009A0006000B800F3FF37000000200001F82700C6
:1009B000F0FF370003F0A200889FBE008A9FBE00B0
:1009C0008C1F78001D010700240133006450E100F2
:1009D0004F0032006420E1005200320003826C00BC
:1009E00007003B000905D0000306D000820F540029
:1009F0000C065D0002003900020032008901780017
:100A0000030678008582550004003D000003FD00C8
:100A10008103FD008502EA008B854200840F72008D
:100A200002003B0060001000E08018006011B80078
:100A30000005EB007A28E1000A0039000600780082
:100A4000C75DDD00F707B200878075002D00370015
:100A5000828171000A017800610560008180D10007
:100A60000080D3008502E900F9FF3B000604400046
:100A70008784480002003B0060041400E0841C00EE
:100A80000988A300070032008A8171008281710009
:100A9000610164008904D1000884D3008B05E8005B
:100AA000170037000978A30013003A000B00E0009C
:100AB000130034008B05E9000804440089844C00CD
:100AC0000A4474000978A3000D003A000B00E0000E
:100AD000070034008B05E9000804440089844C00B9
:100AE00001003A000B0020000978A300F7FF320054
:100AF0000001EB0002003700828171000A017800DA
:100B00008D0007000CF0A70001F0A000DC0037000A
:100B10006420E10002003A00838F6C00DC003300A7
:100B20000801BE000200BE00D5003700889FBE004D
:100B30008A9FBE008C1F7800C0000700C7003300EA
:100B400003866C006450E100240032006420E10060
:100B5000270032006150E100220032006120E100F4
:100B6000210032008B854200EB07B1000134B80050
:100B7000003AB8000804420089844A00013AB800EB
:100B80000030B8008880400009014A0004003300AA
:100B90000000400081804800020149008B05E90007
:100BA000C909DD008301700001003200130020003C
:100BB000C814DE004814DD004709DE001200B20050
:100BC000C808DE00088470005B00070001F0A10087
:100BD0000CF0A70001F0A000A90037006120E1009F
:100BE000AB0032000801BE000200BE00F7FF370074
:100BF0006150E100FCFF3A00A50037000001BE0093
:100C0000A60007000470A70003F0A10003F8A300EA
:100C100013003A006509B1001000320009003500E8
:100C20006928E100020035000100280000000500ED
:100C300000004000818048008502E900FCFF3A0086
:100C400000000600F88F4200050035008100D10049
:100C50000080D3008502E800FCFF3A000000060097
:100C60008000EB00000005006022B80006022000B2
:100C70000000D0008180D2000482D2008582D200A0
:100C80000000A0000202520083825A0003003100DB
:100C90000202420083824A000000A1000603E9002C
:100CA000F3FF3A0000000600EFFF07000400BE005B
:100CB000000006000001BE00780007000470A700D5
:100CC00003F0A1006509B100160032000D003500E7
:100CD0006828E10006003500F0FF2F00F1FF270033
:100CE0000300E00013003B000100280000000500A5
:100CF00000004000818048008502E900FCFF3A00C6
:100D000008003700F88F420002003C008000EB0032
:100D1000000005008100D1000080D3008502E800BA
:100D2000FCFF3A000300E00002003B0060001000FE
:100D3000E08018000000060081002000618055005E
:100D40000B003D000B00200061FE2F000100E100C0
:100D50001D00340082817100610164008904D100AA
:100D60000884D3000000E800FAFF3A007100200078
:100D7000610064000300700002006000090032009E
:100D800061044400E0844C000988A500050032009D
:100D90008B05E8006808E10002003A008904D100F0
:100DA0000884D300F20F20000258E10005003D0046
:100DB000C75DDD00F907B200898075000800780082
:100DC000000006000BF827008B00780000000500EB
:100DD000889FBE008A9FBE00841F7800170007000E
:100DE0004F00780011003300F0FF2F00838F6C005C
:100DF00006003B00040565000A00A7000800370054
:100E000009F0A6001000200008003700820F5400EF
:100E1000838F5C00030039001000200001003E00B9
:100E20000000200009F0A7000000EA004F05BE0006
:100E30004F04BE000000E000000006000004BE00F9
:100E4000160007000003BE000405BE000200BE003D
:100E500012000700844F7500000006000200BE006B
:100E60006450E100050036006420E1000200360015
:100E70000968A30001003A000800BE000160A0005C
:100E80004F0678004F05BE004F04BE00000006006C
:100E9000F0FF2F00F1FF2700F9FF3700C70ADE003F
:100EA000F107B200F50FB20008003200E1CF4200B6
:100EB000020032000170A00024000500810F7000C4
:100EC000010032000408050044000500810F700095
:100ED00002003A00140005008502E900000040000D
:100EE00081C04800FCFF3B000170A0002400050009
:100EF000005E0000BCE20000613F0000DD830000F6
:100F0000C29C00007E200000A3FD00001F410000E5
:100F10009DC30000217F0000FCA20000401E0000D5
:100F20005F010000E3BD00003E60000082DC0000C5
:100F3000237D00009FC10000421C0000FEA00000B5
:100F4000E1BF00005D03000080DE00003C620000A5
:100F5000BEE00000025C0000DF810000633D000095
:100F60007C220000C09E00001D430000A1FF000085
:100F700046180000FAA40000277900009BC5000075
:100F800084DA000038660000E5BB00005907000065
:100F9000DB85000067390000BAE400000658000055
:100FA00019470000A5FB000078260000C49A000045
:100FB000653B0000D9870000045A0000B8E6000035
:100FC000A7F900001B450000C69800007A24000025
:100FD000F8A60000441A000099C70000257B000015
:100FE0003A64000086D800005B050000E7B9000005
:100FF0008CD20000306E0000EDB30000510F0000F5
:101000004E100000F2AC00002F71000093CD0000E4
:10101000114F0000ADF30000702E0000CC920000D4
:10102000D38D00006F310000B2EC00000E500000C4
:10103000AFF10000134D0000CE900000722C0000B4
:101040006D330000D18F00000C520000B0EE0000A4
:10105000326C00008ED00000530D0000EFB1000094
:10106000F0AE00004C12000091CF00002D73000084
:10107000CA94000076280000ABF500001749000074
:1010800008560000B4EA000069370000D58B000064
:1010900057090000EBB50000366800008AD4000054
:1010A00095CB000029770000F4AA00004816000044
:1010B000E9B70000550B000088D60000346A000034
:1010C0002B75000097C900004A140000F6A8000024
:1010D000742A0000C8960000154B0000A9F7000014
:1010E000B6E800000A540000D78900006B35000004
:1010F0004C45000054000000494600000054000028
:10110000484500004E000000454C000053450000DB
:10111000004700004F5400004F000000474F000000
:101120005355000042000000524500005455000095
:10113000524E000000520000454D000000500000DB
:10114000524900004E540000004900004E5000007B
:1011500055540000004600004F52000000540000AB
:101160004F0000004E45000058540000005200009F
:10117000454100004400000044410000544100008B
:10118000005300005441000052540000005300007E
:10119000544100005254000052000000535400001B
:1011A0004F50000000530000544F00005052000008
:1011B00000530000454E000044000000524500006E
:1011C000434500004956000045000000434C000024
:1011D0004B00000044410000540000004249000060
:1011E000545200004541000044000000414400000A
:1011F000430000004155000058000000505300001B
:1012000055000000505500004C4C000055500000A7
:101210000041000055580000504900004E000000F9
:1012200046520000455100000044000055540000A3
:1012300059000000444500004C41000059000000E6
:101240004D410000435200004F000000454E000099
:101250004400000000520000554E0000004C000009
:101260004953000054000000455800004954000054
:10127000004400004542000055470000004E0000B9
:1012800045570000000000003E200000000800005C
:101290002008000000000000203D000020000000A9
:1012A0005652000045470000207400006F6F000098
:1012B000206C00006F7700002C2000006973000094
:1012C0002074000068650000726500002061000065
:1012D00020730000686F0000727400003F0000007F
:1012E0002E2000003C0000003E0000002E200000E8
:1012F000000D00000A280000002900003E20000028
:101300000042000075730000205000006972000068
:10131000617400006520000076310000610000006B
:1013200046690000726D0000776100007265000080
:1013300020760000352E00003420000028720000C6
:10134000343500003429000000200000280000008F
:10135000413300000042000034000000423500002C
:101360000042000038000000554E00004B00000015
:101370002900000049090000004F0000090000009A
:1013800048090000004C000009000000456E000004
:101390007465000072200000726100007720000078
:1013A000766100006C75000065200000666F00002B
:1013B00072200000425200004700000001000000BF
:1013C0000000000003020000000000000000000018
:1013D00001000000060000000401000000030000FE
:1013E00000000000000000000600000008050000EA
:1013F00007030000000600000000000000000000DD
:10140000000000000000000030620000003000001A
:10141000303000002C0000003030000000300000B0
:101420003132000033340000353600003738000018
:1014300039410000424300004445000046300000AE
:1014400078000000436F0000756C0000646E0000BF
:1014500027740000206B000065650000702000000C
:10146000757000000000000053500000493100007A
:1014700000000000002900000020000057000000CC
:1014800020520000004900003243000031000000FB
:101490003A200000000000002E000000315700003C
:1014A00030310000000000000808000008080000BB
:1014B0000800000000000000204800007A00000042
:1014C0000000000000410000525400003100000004
:1014D00042420000494F000031000000524100002C
:1014E0005731000000000000314100004C53000063
:1014F000000000004F4300004431000000000000E5
:1015000000000000000000002900000000000000B2
:1015100000000000000000001A00FA000000EB00CC
:10152000100F98000000EB00606988000000EB00DD
:10153000506988000000EB00A04088000000EB002C
:10154000706988000000EB00100798000000EB00B5
:1015500040079800140037000000EB0020079800B7
:101560000B0037004E009000AE0090004500DD00FB
:101570008100400000D32000808040000040EB004C
:10158000804878002E0090000000E80020079800B6
:101590002E009000FF0F5000F2FF34004E0090002C
:1015A0000000E800400798004E009000E40F500053
:1015B000E9FF34000000EB00806E8800A14080004D
:1015C000E00220000088B900610220008080400015
:1015D000E093200000804000D86B02000000000073
:1015E000D140800000202000008060000000E0006A
:1015F0000400320071002000C0592000569D0200F6
:101600000000000040942800D86B02000000000099
:10161000ED003700806E80000000E00063003200C3
:10162000806E80000000E900806E88000000EB0002
:10163000200798001E00370052698000806E8000ED
:10164000AE0090004500DD008100400000D3200086
:101650000080400090407800A0C2200000004100BF
:1016600001487800806E8000AE0090004500DD00EB
:101670008100400000D3200000804000104078002E
:101680003470020000000000506980000000E80093
:10169000506988002E0090000000E80020079800A4
:1016A00051698000F00F20000080600050698800C0
:1016B000806E8000AE0090004500DD00810040009B
:1016C00000D3200000804000104078000004E000BB
:1016D000D9FF3A000000EB00806E8800330037002D
:1016E00090B7200010407800624060000004E000E5
:1016F0002E003200A1408000E00220000088B900E6
:10170000FA004000E09320000080400010007800C4
:10171000000001000000E00024003200A140800031
:10172000E00220000088B9006102200080804000B3
:10173000E093200000804000D86B02000000000011
:1017400040942800D86B020000000000616980000E
:1017500050698000808F5000140032006069800062
:10176000200798000D003700AE009000A0C22000B6
:10177000008040001040780034700200000000003B
:10178000AE009000F00F200000806000200798005D
:101790002E0090000000E80020079800AE009000A6
:1017A00050698000808F5000EFFF3A0016700200F1
:1017B000000000000004E000C9FF320022700200B7
:1017C00000000000604798006E4090000080FB0021
:1017D000200F98002E089000E80F500011003200F2
:1017E000AE089000E88F500007003C002E099000E2
:1017F0000200E0003C003200AE099000E28F510090
:10180000440032004B0037002E089000EA0F5000D1
:1018100013003200AE089000ED8F5000100032002F
:10182000440037005169800060698000808F50005B
:1018300065003200506980000000E90050698800AE
:1018400051698000F00F200000806000506988001E
:1018500070942800D86B0200000000005A00370086
:1018600010002000100F9800506980008000E800F0
:10187000F00F20008080600060698000808F500041
:101880000D00320051698000A0C22000808040001D
:101890000040EB0080487800506980000000E800BC
:1018A0005069880051698000F00F200000806000BE
:1018B000506988000800370070C0B300347002001F
:1018C0000000000051698000A0C22000808040001C
:1018D0000040EB0080487800B0942800046C0200BF
:1018E00000000000380037001E0090000000E800F3
:1018F000100798001E009000F40F500032003A00CC
:1019000072710200000000000000EB001007980058
:101910002D0037001E009000E40F50002A00340014
:10192000CE870200000000000000EB0010079800C6
:1019300025003700506980008000E800F00F20008B
:101940008080600060698000808F50001600320047
:101950006E409000FF4F50001B0036006E4090001C
:101960000004E000180035006E4090003470020062
:1019700000000000516980006E419000A0C220006C
:101980000080400002487800506980000000E800B4
:101990005069880051698000F00F200000806000CD
:1019A000506988000800370070C0B300347002002E
:1019B0000000000051698000A0C22000808040002B
:1019C0000040EB00804878001E0890000000E00016
:1019D00010FF320050698000700798006069800035
:1019E000600798000000EB00100F98000000EB006B
:1019F000000F98000000EB0070698800D140800063
:101A000000202000008060000000E000BA043200E6
:101A10009A3002000000000051002000305A2000DF
:101A2000E09D02000000000010002000000F980060
:101A3000B104370061698000A0C22000008040002E
:101A400010407800604798006E4090000080FB00D6
:101A50006101B900320F9800430F9800D0072000B1
:101A6000010020003E099000CE099000800F510037
:101A7000818F590072043E003E089000CE0890000D
:101A800000600100700437006D0437006C043700FB
:101A90006B0437006A0437006904370068043700B4
:101AA00067043700660437006504370066043700B2
:101AB00063043700620437006304370060043700B2
:101AC0005F0437005E0437005D0437005C043700B4
:101AD0005B0437005A0437005904370058043700B4
:101AE00057043700560437005504370054043700B4
:101AF00053043700520437005104370050043700B4
:101B00004F043700500437002D043700A40237007B
:101B1000020137000F013700BE013700AC0137006A
:101B2000470437007B023700450437004404370080
:101B30004504370044043700D9033700F203370067
:101B4000BD0337001E0337001D0337001C03370099
:101B50001B0337001A033700190337001803370037
:101B60001703370016033700150337003404370016
:101B700033043700BC013700A900370030043700B8
:101B80004600370021013700130137002C043700CD
:101B90007F0037008B013700290437002804370005
:101BA00027043700260437002504370024043700B3
:101BB0002304370080003700210437002004370059
:101BC0001F0437001E0437001D0437001C043700B3
:101BD0001B0437001A0437001904370018043700B3
:101BE00020013700160437001504370014043700AD
:101BF000CF0237009D033700DF023700D1033700E3
:101C0000B40337000E043700E60037002E0037001B
:101C1000550037005D0137000904370030003700F8
:101C200032003700150037001F003700040437006A
:101C3000030437006D00370021003700000437002F
:101C400023003700FE033700FD0337003C03370055
:101C500081013700FA033700F90337001E0037000F
:101C600036013700F6033700F5033700F403370079
:101C7000B802370087003700C8023700AD060700FA
:101C80000000E000F0033A006069800060079800FF
:101C90005069800070079800EB033700F69D020042
:101CA00000000000E803370002080700A0408000A1
:101CB0000000E000E403320060080700E2033700A0
:101CC00014060700E003370086090700DE0337002B
:101CD0005E090700DC033700D2080700DA0337008B
:101CE000E27B020000000000D7033700606980003B
:101CF0008000E800F00F200080806000A0C220007B
:101D00000080400090407800F0C6B30080CF5000C3
:101D10000A003A00606980000080E800606988007D
:101D200061698000F00F2000008060006069880019
:101D30004C85020000000000C3033700A040800073
:101D40000000E00005003A00D1012000305D2000D5
:101D5000E09D020000000000BB033700467A02004D
:101D600000000000B803370090B720001040780052
:101D70000000A10091B72000804878006101200098
:101D8000805A2000E09D020000000000AE033700F2
:101D900090B72000104078000000A00091B720000C
:101DA0008048780051012000E05B2000E09D0200A7
:101DB00000000000A403370090B720001040780016
:101DC0000020A00091B7200080487800C1012000C9
:101DD000B07E2000569D020000000000B094280054
:101DE000046C0200000000009703370090B7200049
:101DF000104078000020A10091B7200080487800B2
:101E0000B1012000007D2000569D0200000000006E
:101E1000B0942800046C0200000000008A03370020
:101E2000606980000000E8006069880061698000E6
:101E3000F00F20000080600060698800A3050700A3
:101E4000B7030700200798002E009000D26E020012
:101E500000000000C0942800D86B020000000000C1
:101E60002E009000706E020000000000C094280058
:101E7000D86B0200000000002E009000386C0200B9
:101E800000000000B0942800046C02000000000074
:101E90006D033700606980000000E8006069880019
:101EA00061698000F00F2000008060006069880098
:101EB000860507009A030700200798002E0090006F
:101EC000C4980200000000000080FB00200798007A
:101ED0002E009000D26E020000000000C094280086
:101EE000D86B0200000000002E009000706E02000F
:101EF00000000000C0942800D86B02000000000021
:101F00002E009000386C020000000000B094280001
:101F1000046C0200000000004B033700869E0200A4
:101F2000000000000000E0004703320051002000E4
:101F300030632000E09D02000000000023C2BF00CB
:101F4000614060000004E000FCFF32000000FE0081
:101F50003D033700869E0200000000000000E00004
:101F600039033200A100200080632000E09D0200C0
:101F700000000000400620006298020000000000FF
:101F8000DE9602000000000023C2BF006140600036
:101F90000004E000FCFF320081BF2A000140010084
:101FA00029033700030507000000E80040079800F8
:101FB00002003700207D0200000000004E0090006B
:101FC0000000E900400798004E0090000000E0008B
:101FD000F8FF3A001C033700F60407000000E80091
:101FE0004007980002003700FE7C0200000000005D
:101FF0004E0090000000E900400798004E0090005D
:102000000000E000F8FF3A000F033700E904070082
:102010000000E800400798000B0037006101200035
:1020200020642000569D020000000000427D020056
:1020300000000000C26B020000000000B094280005
:10204000046C0200000000004E0090000000E90057
:10205000400798004E0090000000E000EFFF3A00BB
:10206000F9023700A04080000000E00005003A00BF
:10207000D1012000305D2000E09D02000000000042
:10208000F1023700C082A900C282A800C8A2A9003C
:10209000CAA2A80021E3A800200020006298020044
:1020A00000000000A0C0B300249702000000000060
:1020B00080007800001B2000808F50000F00360049
:1020C00090C0B30024970200000000008000780058
:1020D000702B2000808F5000080036001101200076
:1020E00080652000569D020000000000B09428008A
:1020F000046C0200000000000E003700C082A9003E
:10210000C282A900C8A2A900CAA2A90000952800FD
:10211000046C0200000000002101200090662000F5
:10212000569D020000000000B0942800046C0200DC
:102130000000000021E3A900C3023700A040800096
:102140000000E00005003A00D1012000305D2000D1
:10215000E09D020000000000BB023700C082A90021
:10216000C282A900C8A2A900CAA2A9002101200018
:1021700090662000569D020000000000B0942800E8
:10218000046C020000000000AF023700F1002000E4
:10219000A0392000569D0200000000003E9702007A
:1021A0000000000011002000903A2000569D02001F
:1021B00000000000B0942800046C02000000000041
:1021C000A102370050970200000000009E02370075
:1021D0007804070040079800610020007068200024
:1021E000569D0200000000004E009000126E02009A
:1021F0000000000021002000D0682000E09D0200C7
:10220000000000004E0090008E98020000000000C8
:102210008D02370067040700400798006100200026
:1022200070682000569D0200000000004E009000E3
:10223000126E0200000000002100200090EC20003F
:10224000E09D0200000000004E0090006298020035
:10225000000000007C023700D04080000090A00009
:10226000D040880078023700100020007069880094
:1022700010002000200798001000370061698000DE
:102280002E00900080804000F00F200080806000D1
:10229000A0C220000080400090407800E0C3B3005E
:1022A00080CF500002003A000000EB007069880007
:1022B0002E0090000000E80020079800616980006F
:1022C0002E00900080804000F00F20008080600091
:1022D000A0C2200000804000104078000004E00010
:1022E000E6FF3A00AE00900020022000808F5000F0
:1022F00002003400100020007069880070698000BE
:102300000000E00050023A00606980000000E80030
:102310006069880061698000F00F20000080600023
:10232000606988007E0207002007980061698000CC
:10233000F00F200080806000A0C2200000804000DC
:1023400090407800D0C3B30080CF500044003A00E2
:102350002E0090000000E0003E0034002E009000AF
:10236000E50F50003B003C00606980000000E80081
:102370006069880061698000F00F200000806000C3
:10238000606988002E0090000000E9002007980096
:102390000000EB00400798000B0037002E00900073
:1023A000CE0090004500DD008100400000D32000F9
:1023B000808040000040EB00804878004E00900094
:1023C0000000E800400798004E009000FF0F50000A
:1023D000F2FF34000000EB004007980015003700C2
:1023E000AE0190004E02900061698000A0C2200002
:1023F00000804000104178004518DD008400400056
:1024000000D3200000804000024878004E00900079
:102410000000E80040079800606980000000E800C4
:102420006069880061698000F00F20000080600012
:102430006069880061698000A0C2200000804000BF
:1024400090407800E0C3B30080CF5000E4FF3A0032
:10245000FD0137001000200070698800FA01370084
:102460002E0090000000E0001B003A000000EB008E
:1024700040079800140037004E0090000040E8002C
:10248000706E02000000000000972800D86B020068
:10249000000000004E0090004500DD008000780044
:1024A00000D3200000804000D86B02000000000034
:1024B00040972800046C0200000000004E009000CD
:1024C0000000E800400798004E009000E40F500024
:1024D000E9FF3400DC0137002E0090000000E0002E
:1024E000090034002E009000E50F500006003C006B
:1024F000B0942800046C020000000000AE009000C0
:10250000816E8800D00137001000200070698800BB
:10251000CD013700606980000000E8006069880034
:1025200061698000F00F2000008060006069880011
:10253000FB01070050079800E40307006169800071
:10254000F00F200080806000A0C2200000804000CA
:102550009040780090C2B30080CF50000D003A0048
:10256000A1408000E00220000088B900FC0040008B
:10257000E093200000804000900078005E00900012
:1025800001000100B0942800046C0200000000006B
:10259000AD0137001000200070698800AA013700E3
:1025A00010002000706988001000200020079800AB
:1025B00010003700616980002E009000808040008C
:1025C000F00F200080806000A0C22000008040004A
:1025D0009040780020C2B30080CF500002003A0043
:1025E0000000EB00706988002E0090000000E800F9
:1025F00020079800616980002E00900080804000D4
:10260000F00F200080806000A0C220000080400009
:10261000104078000004E000E6FF3A007069800096
:102620000000E00088013A0071002000F0682000FE
:10263000569D02000000000020C2B300347002006A
:10264000000000002300370061698000F00F2000C7
:10265000008060006069880061698000A0C220007D
:10266000008040001040780034700200000000003C
:1026700061698000A0C22000008040001040780006
:102680000000FB005007980090B720001040780031
:10269000644060000004E000050032005E0090002D
:1026A000C4980200000000000080FB005007980062
:1026B000A1408000E00220000088B900E80040004E
:1026C000E093200000804000900078005E009000C1
:1026D00001000100606980000000E8006069880076
:1026E00061698000F00F200080806000A0C220009F
:1026F000008040009040780020C2B30080CF50009E
:10270000D1FF3A0060698000F10F200001006000F5
:102710006069880020C2B30034700200000000002D
:10272000B0942800046C020000000000460137004D
:10273000A1408000E00220000088B90080007800FD
:10274000E0932000008040001000780000000100AD
:102750003D013700A1408000E00220000088B90060
:102760008080E800E09320000080400010007800A6
:102770000000010034013700A1408000E002200089
:102780000088B900E4004000E09320000080400091
:1027900010007800000001002B013700A1408000EC
:1027A000E00220000088B900E6004000E09320002D
:1027B0000080400010007800000001002201370076
:1027C00071002000F0682000569D0200000000000B
:1027D0005301070050079800606980000000E9007D
:1027E0006069880061698000F00F2000008060004F
:1027F00060698800EF0207000000E80040079800C9
:102800000F030700000F78001E00E00042003200B6
:102810001E00780080407800A0B7200001487800B2
:102820003D0037005E009000DC97020000000000D1
:10283000A0B7200010407800E84F50000700320099
:10284000B0C3B3003470020000000000A0B7200045
:1028500010407800706E02000000000090B7200069
:1028600010407800644060000004E0000500320081
:102870005E009000C4980200000000000080FB0091
:1028800050079800A1408000E00220000088B900B5
:10289000E8004000E09320000080400090007800B5
:1028A0005E009000010001002007980000C2B30004
:1028B0003470020000000000AE009000F00F200015
:1028C000808F500014003C006100200060692000EF
:1028D000569D02000000000090B7200010407800D4
:1028E000644060000004E000050032002E0090000B
:1028F000C4980200000000000080FB002007980040
:102900002E009000DC9702000000000000C2B3001F
:1029100034700200000000004E0090000000E9004A
:10292000400798004E0090000000E000BDFF3A0014
:10293000B0942800046C020000000000C2003700C0
:102940006100200060692000569D02000000000028
:10295000980207000000E80040079800B80207004E
:10296000000F78001E00E000290032001E007800F1
:1029700080407800A0B7200001487800240037008C
:10298000A1408000E00220000088B900EA00400079
:10299000E09320000080400010007800000001005B
:1029A0006047980090B720001040780064406000B5
:1029B0000004E000040032006E409000C498020061
:1029C00000000000604798006E4090000080FB000F
:1029D000DC97020000000000A0B720001040780043
:1029E000E84F500007003200B0C3B300347002005B
:1029F00000000000A0B7200010407800706E0200B8
:102A00000000000000C2B3003470020000000000AB
:102A10004E0090000000E900400798004E00900032
:102A20000000E000D6FF3A00B0942800046C0200D9
:102A3000000000008400370081002000C0692000F1
:102A4000E09D020000000000A1408000E0022000A4
:102A50000088B900EC004000E093200000804000B6
:102A6000100078000000010077003700810020008E
:102A7000406A2000E09D020000000000A1408000AC
:102A8000E00220000088B900EE004000E093200042
:102A90000080400010007800000001006A0037004C
:102AA000E1002000C06A2000E09D0200000000005C
:102AB000A1408000E00220000088B900F000400042
:102AC000E09320000080400010007800000001002A
:102AD0005D003700E1002000A06B2000E09D0200B7
:102AE00000000000A1408000E00220000088B90042
:102AF000F2004000E09320000080400010007800C9
:102B00000000010050003700C1002000B067200025
:102B1000569D020000000000A1408000E00220005D
:102B20000088B900F4004000E093200000804000DD
:102B30001000780000000100C26B020000000000DD
:102B4000410037001B02070040079800D100200019
:102B5000806D2000569D0200000000004E00900095
:102B6000DC970200000000004E0090000000E8002A
:102B70004007980008003700A1408000E0022000D4
:102B80000088B900F6004000E0932000008040007B
:102B900010007800000001004E0090000000E900E5
:102BA000400798004E0090000000E000F2FF3A005D
:102BB000B0942800046C02000000000022003700DE
:102BC000FC0107000000E80040079800A100200079
:102BD000506E2000569D0200000000000D003700DE
:102BE000A1408000E00220000088B900F800400009
:102BF000E0932000008040001000780000000100F9
:102C0000C26B02000000000000C2B300347002007A
:102C1000000000004E0090000000E900400798000E
:102C20004E0090000000E000EDFF3A00010120009E
:102C3000806C2000E09D02000000000002003700D0
:102C40001000200070698800606980000000E800C2
:102C50006069880061698000F00F200000806000DA
:102C600060698800706980000000E0001C0032008C
:102C700051012000F06E2000569D0200000000006F
:102C8000EE00900060698000808F500007003100E6
:102C900060698000804078006E00900000C05000A5
:102CA000706E0200000000000600370060698000BE
:102CB000804078006E00900000C05000706E0200EE
:102CC000000000000000EB00706988001000200088
:102CD000000F9800B0942800046C0200000000006F
:102CE0006169800050698000808F500002003A00C6
:102CF00010002000000F98000E0890000000E00077
:102D00004CFB32007E009000606988007E009000DD
:102D1000506988000000EB00100F980027FA370078
:102D20000600FA000000EB00100798000000EB001E
:102D3000000F7800616980001E00900080804000D4
:102D4000F00F200080806000A0C2200000804000C2
:102D50009040780000C3B30080CF5000430034009F
:102D6000616980001E00900080804000F00F20000C
:102D700080806000A0C22000008040009040780069
:102D800090C3B30080CF500038003C0061698000E0
:102D90001E00900080804000F00F200080806000C6
:102DA000A0C2200000804000104078008000FB009E
:102DB00000FD2F00008F40001E0090000000E80082
:102DC00010079800120037001E0078006A00B90052
:102DD000000F7800616980001E0090008080400034
:102DE000F00F200080806000A0C220000080400022
:102DF000104078000000FB009E00400000FD2F0006
:102E0000008F40001E0090000000E80010079800AE
:102E1000616980001E00900080804000F00F20005B
:102E200080806000A0C220000080400090407800B8
:102E3000F0C2B30080CF50005101340061698000BE
:102E40001E00900080804000F00F20008080600015
:102E5000A0C22000008040009040780090C3B300E2
:102E600080CF5000D8FF34004501370061698000F1
:102E70001E00900080804000F00F200080806000E5
:102E8000A0C22000008040009040780000C3B30042
:102E900080CF500035013A001E0090000000E8008D
:102EA00010079800616980001E009000808040003B
:102EB000F00F200080806000A0C220000080400051
:102EC0009040780020C6B30080CF50000B00320045
:102ED000616980001E00900080804000F00F20009B
:102EE00080806000A0C220000080400090407800F8
:102EF00020C4B30080CF50002D003A001E00900087
:102F00000000E80010079800120037001E0078004B
:102F100000004000000F7800616980001E009000F2
:102F200080804000F00F200080806000A0C2200060
:102F300000804000104078000000FB009E00400030
:102F400000FD2F00008F40001E0090000000E800F0
:102F500010079800616980001E009000808040008A
:102F6000F00F200080806000A0C2200000804000A0
:102F70009040780010C3B30080CF5000E3FF3200D0
:102F8000616980001E00900080804000F00F2000EA
:102F900080806000A0C22000008040009040780047
:102FA00000C3B30080CF5000D8FF3200F4003700D8
:102FB000616980001E00900080804000F00F2000BA
:102FC00080806000A0C22000008040009040780017
:102FD00080C7B30080CF50000B00320061698000D1
:102FE0001E00900080804000F00F20008080600074
:102FF000A0C22000008040009040780080C5B3004F
:1030000080CF50008E003A001E0090000000E800C3
:1030100010079800470037001E0078004400DD00CC
:10302000000F7800616980001E00900080804000E1
:10303000F00F200080806000A0C2200000804000CF
:1030400090407800F0C2B30080CF500018003400E8
:10305000616980001E00900080804000F00F200019
:1030600080806000A0C22000008040009040780076
:1030700090C3B30080CF50000D003C006169800018
:103080001E00900080804000F00F200080806000D3
:10309000A0C2200000804000104078000000FB002B
:1030A0009E00400000FD2F00008F40001E003700F2
:1030B000616980001E00900080804000F00F2000B9
:1030C00000816000616980001E00900080804000E7
:1030D000F00F200080806000A0C22000008040002F
:1030E0009040780000C2B30080C07000A0C22000F1
:1030F0000000410001487800616980001E009000D6
:1031000080804000F00F200080806000A0C220007E
:1031100000804000104078000000FB009E0040004E
:1031200090FA2F00008F40001E0090000000E80081
:1031300010079800616980001E00900080804000A8
:10314000F00F200080806000A0C2200000804000BE
:1031500090407800F0C2B30080CF50000B003400E4
:10316000616980001E00900080804000F00F200008
:1031700080806000A0C22000008040009040780065
:1031800090C3B30080CF5000A3FF3400616980007A
:103190001E00900080804000F00F200080806000C2
:1031A000A0C22000008040009040780000C4B3001E
:1031B00080CF50000B003400616980001E00900039
:1031C00080804000F00F200080806000A0C22000BE
:1031D000008040009040780060C4B30080CF500071
:1031E0008DFF3400616980001E00900080804000E7
:1031F000F00F200080806000A0C22000008040000E
:103200009040780000C6B30080CF50005C003400CE
:10321000616980001E00900080804000F00F200057
:1032200080806000A0C220000080400090407800B4
:1032300060C6B30080CF500077FF340050003700E5
:10324000616980001E00900080804000F00F200027
:1032500080806000A0C22000008040009040780084
:10326000F0C2B30080CF5000450034006169800097
:103270001E00900080804000F00F200080806000E1
:10328000A0C22000008040009040780090C3B300AE
:1032900080CF50003A003C00616980001E00900021
:1032A00080804000F00F200080806000A0C22000DD
:1032B00000804000104078008000FB0000FD2F00DF
:1032C000008F4000120037001E0078006A00B9002D
:1032D000000F7800616980001E009000808040002F
:1032E000F00F200080806000A0C22000008040001D
:1032F000104078000000FB009E00400000FD2F0001
:10330000008F40001E0090000000E80010079800A9
:10331000616980001E00900080804000F00F200056
:1033200080806000A0C220000080400090407800B3
:10333000F0C2B30080CF50001100340061698000FA
:103340001E00900080804000F00F20008080600010
:10335000A0C22000008040009040780090C3B300DD
:1033600080CF5000D8FF3400050037001000200047
:10337000706988000000EB00200798000A00370001
:10338000616980001E009000008040006069880034
:1033900061698000F00F2000008060006069880093
:1033A0001E007800200798002E0090000080FA0090
:1033B000000006000400FA00606980008000E80058
:1033C000F00F200080806000A0C22000008040003C
:1033D00090407800A0C3B30080CF500013003A00A3
:1033E000606980000080E800606988006169800091
:1033F000F00F2000008060006069880048FE070030
:10340000000F7800606980000000E90060698800B2
:1034100061698000F00F2000008060006069880012
:103420001E007800100798000200370010002000EE
:10343000100798001E0090000080FA0000000600AF
:103440000400FA00606980008000E800F00F2000AE
:1034500080806000A0C22000008040009040780082
:10346000B0C3B30080CF500013003A006069800001
:103470000080E8006069880061698000F00F20002A
:10348000008060006069880025FE0700000F78005A
:10349000606980000000E90060698800616980005F
:1034A000F00F200000806000606988001E00780036
:1034B00010079800020037000000EB00100798008A
:1034C0001E0090000080FA00000006000000FA00D4
:1034D00007003700606980000000E800606988002C
:1034E00061698000F00F2000008060006069880042
:1034F00061698000A0C220000080400090407800F8
:1035000000C2B30080CF5000F2FF32000080FA000A
:10351000000006000400FA000000EB00000F780035
:10352000606980000000E8006069880061698000CF
:10353000F00F20000080600060698800E3FF070052
:10354000F7FD0700000F78001E00E0004D003A0074
:103550000000EB0010079800130037001E009000D9
:103560000040E800706E0200000000006097280034
:10357000D86B0200000000009E009000E0022000D6
:103580000088B9006102200080804000E0932000A4
:1035900000804000046C0200000000001E0090004B
:1035A0000000E800100798001E009000E80F50008F
:1035B000EAFF34007101200040702000E09D02000D
:1035C000000000000000EB0070698800130020007C
:1035D000920020001100200010002000F6000700DB
:1035E000000FE900E0FF2F009E0F100003003200E3
:1035F0000080EB009E0F100005003A00E100200063
:10360000B0712000E09D0200000000004200370081
:10361000A1408000E00220000088B90001022000E3
:1036200080804000E093200000804000100078007F
:1036300000000100DE960200000000001E0078007D
:10364000A0408800A1408000E00220000088B9006E
:10365000FE004000E0932000008040001000780051
:10366000000001001E00E00001003200CA82A80034
:1036700051002000305A2000E09D020000000000B0
:10368000250037001E0FE900800020009E0F10006B
:103690001D003C00A1408000E00220000088B9002D
:1036A0000102200080804000E09320000080400064
:1036B0001000780000000100DE960200000000000B
:1036C0001E007800A0408800A1408000E002200099
:1036D0000088B900FE004000E09320000080400018
:1036E00010007800000001001E00E0000100320020
:1036F000CA82A80051002000305A2000E09D02003C
:1037000000000000040037005101200090722000EA
:10371000E09D020000000000506980008000E90088
:10372000F00F200000806000606988000080FA00CF
:10373000000006002600FA00100020002007980074
:10374000606980000000E900100798009E0090006A
:10375000F00F200000806000100798004300370041
:103760009E009000A0C22000008040001040780021
:103770000004E00036003A001E0090008000E800DF
:10378000F00F200080806000A0C220000080400078
:10379000104078000004E0002D0032002E00900060
:1037A000706E02000000000060972800D86B0200D5
:1037B0000000000010002000000F78000A00370011
:1037C0001E0090009E004000F00F200080806000EE
:1037D000A0C2200000804000104078003470020039
:1037E000000000001E0FE8001E0090009E00400038
:1037F000F00F200080806000A0C220000080400008
:10380000104078000004E000EDFF3A00AE019000A7
:103810001E0090008000E800F00F20000081600092
:10382000E60047000380410002B078002E009000BF
:103830000000E800200798002E009000EF0F5000D5
:103840000E003200B0942800046C0200000000005A
:103850001E0090000000E900100798009E009000F4
:10386000F00F200000806000100798009E0090007C
:1038700060698000808F5000B9FF3A00710020001D
:10388000E0732000E09D0200000000001300200013
:103890002E019000110020000000EB004600070000
:1038A000100798001E009000E10F400003003A004E
:1038B00010002000201798003C0037000000EB00AB
:1038C0002007980016003700516980002E009000F4
:1038D00080804000F00F2000008160001E009000FA
:1038E000E600470000004000E08078002E009000D5
:1038F00080804000F00F200080806000A0C2200087
:103900000080400090407800A0C2200000004100EC
:10391000014878002E0090000000E8002007980081
:103920001E009000E600470000004000E0807800A4
:103930002E00900080804000F00F2000808060000A
:10394000A0C2200000804000104078000004E00089
:10395000DDFF3A00506980008000E900F00F200090
:103960000080600060698800616980002E0090001E
:10397000008040008080E800F00F200000806000A0
:1039800050698800506980008000E900F00F200035
:1039900080806000A0C22000808040000040EB00DA
:1039A000804878000000EB00201798002E1090004F
:1039B0000080FA00000006001E00FA00100F9800B8
:1039C000210F9800320F9800430F98000000EB0081
:1039D000400798000000EB00200798000000EB0073
:1039E000100798000000EB00000F78009097280067
:1039F000D86B0200000000001E089000706E0200EC
:103A000000000000D0972800D86B020000000000E2
:103A1000670037002270020000000000204F98006D
:103A20002E4890000000FB00600F98006E08900088
:103A3000ED0F500029003200EE089000ED8F50008D
:103A400007003C006E099000E80F51000D003200A5
:103A50006E089000EA0F5000200032003500370059
:103A6000D0022000EE089000808F50001E0032002F
:103A7000800720006E099000800F5100270032005F
:103A80002C0037004E0090000000E00007003200DC
:103A90004E0090000000E900400798007094280054
:103AA000D86B020000000000410037001E00E0005B
:103AB000060032000000EB00000F78007094280030
:103AC000D86B0200000000003900370070C0B3005E
:103AD00034700200000000003500370010002000A4
:103AE00020079800320037004E0090000000E000F0
:103AF00006003A00D0C2B30034700200000000009B
:103B000010002000000F78002900370070C0B300BB
:103B10003470020000000000250037004E089000BD
:103B20000000E000030032000080EB00500F98001E
:103B30005D003700AE489000F0C2B30080CF500067
:103B400018003400AE48900090C3B30080CF5000FE
:103B500014003C004E009000E30F500006003400BB
:103B600070C0B3003470020000000000400020006C
:103B7000400798000E0037002E4890003470020075
:103B800000000000CE0090006B0047002E4990001E
:103B9000827078004E0090000000E8004007980016
:103BA0000300370070C0B300347002000000000052
:103BB0002E0090000000E00096FF3200B094280034
:103BC000046C0200000000004E0090000000E000C5
:103BD00003003A001E089000500F98003200370092
:103BE0000000EB00100798004E0090000000E90074
:103BF00040079800CE009000310798001100370070
:103C00001E0090006A00B90010079800BE009000E6
:103C10004E009000808050006B00470061407800AB
:103C20008000FB001E0090008080400000FD2F00FF
:103C300000804000100798004E0090000000E9004E
:103C4000400798004E0090000000E000ECFF3D00AF
:103C50009E0090002E089000808F50000D003500CF
:103C60009E0090003E089000808F500009003C00AC
:103C70001E00E000040032001E0090000000EA0078
:103C8000500F9800080037001E019000520F980056
:103C900005003700B1012000E0EA2000E09D0200AD
:103CA0000000000049FF37005E0890000080FA0025
:103CB000000006000400FA0010982800046C0200BE
:103CC0000000000000992800D86B020000000000EE
:103CD000D100200070802000569D020000000000EE
:103CE000A1BF2A000000EB004C71020000000000A0
:103CF000000F78001E0078004800DE00706E0200A1
:103D000000000000E0C2B3003470020000000000B8
:103D10001E007800706E020000000000B0942800C1
:103D2000046C02000000000061002000007620000A
:103D3000569D020000000000B04080002A6F020083
:103D4000000000007100200070EA2000569D020073
:103D500000000000C04080002A6F02000000000048
:103D6000509A2800D86B020000000000C04080007C
:103D700010079800200423009E009000808F5000C0
:103D800016003200200423009E009000808F500017
:103D900005003E00300023009E009000808F500000
:103DA0000A00320019003700300423009E00900002
:103DB000808F50000D003200600423009E009000B0
:103DC000808F50000D00320010003700809A2800CC
:103DD000D86B0200000000000F003700B09A2800E6
:103DE000D86B0200000000000B003700E09A2800AA
:103DF000D86B02000000000007003700109B28006D
:103E0000D86B02000000000003003700409B280030
:103E1000D86B020000000000809B2800046C0200A8
:103E200000000000E101200060762000E09D02001B
:103E3000000000000080FA00000006000000FA0008
:103E40005100200020922000569D0200000000003A
:103E5000C1BF2A000000EB004C710200000000000E
:103E60002A6F020000000000610020007092200014
:103E7000569D020000000000E1BF2A000000EB0098
:103E80004C710200000000002A6F020000000000D8
:103E9000B0942800046C020000000000C100200063
:103EA00040782000E09D0200000000005D00070057
:103EB000CAC2BF000042B2000004E00005003200A8
:103EC0001101200080652000569D020000000000C6
:103ED000040037002101200090662000569D02005A
:103EE00000000000C0C2B3003470020000000000F7
:103EF00000C2B300347002000000000090B7200040
:103F000010407800684060000004E00005003200C6
:103F10002102200000792000E09D02000000000046
:103F200004003700E1012000207B2000E09D02001A
:103F30000000000090B7200010407800644060004E
:103F40000004E00005003A00B1012000007D2000DF
:103F5000569D02000000000004003700C10120004F
:103F6000B07E2000569D020000000000C0C2B300D9
:103F7000347002000000000000C2B3003470020080
:103F800000000000B1012000C0202100569D020069
:103F900000000000A0B7200010407800706E020002
:103FA00000000000B0942800046C02000000000033
:103FB00090B7200010407800614060000004E000ED
:103FC0000500320051012000E05B2000E09D02006E
:103FD000000000000400370061012000805A20002A
:103FE000E09D020000000000A1408000E0022000EF
:103FF0000088B9004102200080804000E09320004A
:10400000008040001000780000000100C100200086
:1040100040782000E09D0200000000000080FA00CF
:10402000000006000000FA00A1002000A005210009
:10403000E09D02000000000061042000200B210030
:10404000E09D020000000000A101200040062100C8
:10405000569D020000000000A1408000E002200008
:104060000088B9002102200080804000E0932000F9
:10407000008040001000780000000100A100200036
:10408000E0072100569D02000000000000402000D3
:1040900050000700001020004E0007000020200004
:1040A0004C000700000420004A0007000008200020
:1040B00048000700B0942800046C020000000000D3
:1040C00041002000800F2100569D020000000000EA
:1040D00021E3A800A0C0B300249702000000000064
:1040E000746F02000000000011002000903A2000D0
:1040F000569D02000000000090C0B3003470020022
:104100000000000090C0B3002497020000000000EF
:10411000746F02000000000011002000903A20009F
:10412000569D02000000000090C0B30034700200F1
:1041300000000000C0C0B30024970200000000008F
:10414000746F02000000000011002000903A20006F
:10415000569D02000000000090C0B30034700200C1
:1041600000000000B0C0B30024970200000000006F
:10417000746F02000000000011002000903A20003F
:10418000569D02000000000090C0B3003470020091
:104190000000000021E3A900004020001C000700EF
:1041A000001020001A00070000202000180007005F
:1041B000000420001600070000082000140007007B
:1041C000B0942800046C0200000000000080FA0097
:1041D000000006000200FA00000F78004016800080
:1041E0001E0060000000E00004003200A09B2800D8
:1041F000D86B02000000000003003700D09B2800AD
:10420000D86B0200000000000080FA0000000600E9
:104210000200FA00000F7800501680001E006000B7
:104220000000E00004003200009C2800D86B02006F
:104230000000000003003700309C2800D86B02000B
:10424000000000000080FA00000006000200FA00F2
:10425000606980000000E800606988006169800092
:10426000F00F2000008060006069880097FC070064
:10427000ABFA0700000F78001E00E00006003400D3
:10428000400020009E0F100003003C001E00E900CB
:10429000904088000D0037000000EB007069880036
:1042A0002102200040812000E09D0200000000006B
:1042B0008001EB00420020001100200010002000CF
:1042C000BDFD07000000E9009040880021012000AA
:1042D00060832000E09D0200000000000080FA00E2
:1042E000000006000200FA00606980000000E8009B
:1042F0006069880061698000F00F20000080600024
:104300006069880071FC070085FA07001047980073
:104310001E4090000004E000090032001E409000A2
:10432000EA4F500006003E001E4090000040E900A9
:104330008040780000812000014878000F0037009D
:104340000000EB0070698800D10820003087200051
:10435000E09D0200000000008001EB00A2002000B0
:10436000110020009000200093FD07000040E900AC
:104370008040780000812000014878000081200002
:1043800010407800E94F500010003A004FFC070041
:1043900063FA0700004F78001E04E0000B003A00AB
:1043A0000000EB0070698800609C2800046C02002B
:1043B000000000008001EB00F2FF27008000EB000E
:1043C000200220007CFD0700004F78004101200002
:1043D00000902000E09D020000000000110120007C
:1043E000B01F2100E09D02000000000023C2BF00BA
:1043F000614060000004E000FCFF3200008120000A
:1044000010407800E94F500003003A001E40780049
:104410005270020000000000AE9702000000000091
:104420000000370016700200000000000004E000E9
:10443000FCFF320022700200000000008040780083
:1044400000C2B30080CF500001003200F5FF3700FA
:104450000080FA00000006000000FA00717380007E
:1044600060E72000008040009040780030C8B30032
:1044700080CF50000E003A00707380000000E8000A
:104480007073880003003700707380000000E8003C
:10449000707388007173800060E720000080400026
:1044A0009040780000CEB30080CF5000F6FF360079
:1044B0000080FA00000006000A00FA0030079800A9
:1044C0000000EB0020079800AE00900060E720009D
:1044D000008040009040780000CEB30080CF5000B4
:1044E00003003E000080EB004007980023003700E7
:1044F000AE00900060E7200000804000104078008F
:104500008080FB0000F22F00008040001007980020
:104510002E0090008000E80060E72000008040004E
:10452000104078000080FB004801DD002E00900064
:104530008080E80060E720000080400010407800A4
:104540000080FB00000F41009E0078003E009000BC
:10455000808F500003003A002E0090004007980022
:10456000060037009E0090002E0090000080400062
:104570006300400020079800D3FF37004E009000F2
:104580000080FA00000006000600FA00881F78008C
:104590000000EB00000F78007173800060E72000DE
:1045A000008040009040780080C2B30080CF50006F
:1045B00010003A00707380000000E80070738800FB
:1045C0001D010700000F78007173800060E7200074
:1045D000008040009040780090C2B30080CF50002F
:1045E000AA003A00707380000000E8007073880031
:1045F000A60037007173800060E720000080400053
:104600009040780000C4B30080CF50001600360000
:104610007173800060E720000080400090407800C7
:10462000A0C5B30080CF50000F003E007273800021
:1046300060E7200000004100104078008080FB000F
:10464000F0FB2F000080400080004000E0E02000F0
:104650000080400010007800200798000200E80069
:10466000707388008B0037007173800060E7200052
:10467000008040009040780000C8B30080CF500018
:10468000740036007173800060E7200000804000F5
:10469000104078000080FB00100798000100E8003F
:1046A00070738800700920009E009000808F500079
:1046B00041003200700920009E009000808F500061
:1046C0000D003C00400920009E009000808F5000AB
:1046D00016003200600920009E009000808F50007C
:1046E0002B003200300920009E009000808F500087
:1046F0001800320046003700900920009E0090000C
:10470000808F50001E003200900920009E00900013
:10471000808F500039003500A00920009E009000D5
:10472000808F50002E00320039003700A1408000F9
:10473000E00220000088B900EA004000E093200079
:10474000008040001000780000000100000F780099
:104750004E003700A1408000E00220000088B90030
:10476000E8004000E0932000008040001004780042
:104770008200070008000100000F780043003700A6
:10478000427D020000000000000F78003F0037006B
:10479000A1408000E00220000088B900F400400041
:1047A000E09320000080400010007800000001002D
:1047B000000F780035003700A1408000E0022000A3
:1047C0000088B900F8004000E0932000008040001D
:1047D0001000780000000100000F78002B00370067
:1047E000CAC2BF000080FB004500DE0061406000DF
:1047F0000080FB00000F780024003700C0C0B30029
:104800002497020000000000000F78001F0037000E
:104810000000EB00000F78001C0037001E0078003D
:104820006A00B900000F78007173800060E7200013
:1048300000804000104078000080FB009E00400097
:1048400000FD2F00008F4000707380000000E80022
:10485000707388007173800060E720000080400062
:1048600090407800F0C2B30080CF500007003600BF
:104870007173800060E72000008040009040780065
:1048800090C3B30080CF5000E4FF36001E007800D4
:10489000200798002E0090004F0478000080FA0056
:1048A000000006000600FA0037FF0700000F78003E
:1048B000000037007173800060E720000080400036
:1048C00090407800A0C2B30080CF50000A003200B0
:1048D0007173800060E72000008040009040780005
:1048E000F0C2B30080CF5000030032001E007800F9
:1048F000200798001E0037007173800060E72000D9
:1049000000804000104078000080FB0010079800F5
:104910000100E80070738800A00220009E00900053
:10492000808F500005003200F00220009E009000B1
:10493000808F500007003200DEFF370012FF0700B3
:10494000800078001E0078000180B900000F780018
:10495000D8FF37000CFF0700000178001E00780028
:10496000110009000200D800000F7800D1FF3700C5
:104970002E0090000080FA00000006000600FA00F9
:10498000C8FF0700000F7800000037007173800037
:1049900060E720000080400090407800D0C2B30063
:1049A00080CF50000A0032007173800060E7200061
:1049B0000080400090407800B0C2B30080CF50002B
:1049C000030032001E00780020079800170037000F
:1049D0007173800060E72000008040001040780084
:1049E0000080FB00100798000100E8007073880049
:1049F000B00220009E009000808F5000080032001E
:104A0000D00220009E009000808F500001003200F4
:104A1000DEFF3700A3FF07001E0F1000DBFF37008B
:104A2000A0FF07001E0F4000D8FF37002E009000A7
:104A30000080FA00000006000C00FA00727380008B
:104A400060E7200000004100104078008080FB00FB
:104A5000F0FB2F000080400080004000E0E02000DC
:104A60000080400090007800210798000200E800D4
:104A7000707388000000EB00000F78000B00370017
:104A80009E0178007273800060E720000000410002
:104A900010407800804078006600470081717800FF
:104AA0000200E800707388001E0FE8007173800038
:104AB00060E72000008040009040780000C4B30010
:104AC00080CF5000070036007173800060E720003F
:104AD0000080400090407800A0C5B30080CF500017
:104AE0000E0036007173800060E7200000804000F7
:104AF00090407800F0C2B30080CF5000E0FF360055
:104B00007173800060E720000080400090407800D2
:104B100090C3B30080CF5000D9FF3E0097FF07003D
:104B20001007980066004700104078000000FB0066
:104B300050079800C0032000DE009000808F5000D6
:104B400032003200C0032000DE009000808F500051
:104B500005003C0010022000DE009000808F500015
:104B6000410032004E003700D0032000DE009000EC
:104B7000808F500005003200E0032000DE0090002E
:104B8000808F50000A003200450037000000EB0023
:104B900040079800AE0090001E009000808F5000EB
:104BA00041003A0011002000410798003E00370004
:104BB0006600470090409000D0C3B30080CF500003
:104BC00009003A000000EB0040079800AE0090009A
:104BD0001E009000808F500033003500110020002F
:104BE00041079800300037000000EB0040079800B4
:104BF000AE0090001E009000808F50002A0034000C
:104C00001100200041079800270037006600470088
:104C100090409000D0C3B30080CF500009003A000C
:104C20000000EB0040079800AE0090001E009000CE
:104C3000808F50001C003C001100200041079800AC
:104C4000190037000000EB0040079800AE0090000C
:104C50001E009000808F500013003D0011002000C6
:104C60004107980010003700660047009040900010
:104C7000D0C3B30080CF500009003A000000EB0021
:104C800040079800AE0090001E009000808F5000FA
:104C90000500320011002000410798000200370093
:104CA0000000EB00400798004E0090000080FA00E2
:104CB000000006001C00FA00881F78000000EB00CE
:104CC000707388000000EB00300798000000EB00D4
:104CD000200798000000EB00100798000000EB0090
:104CE000807388000000EB00907388000000EB00E8
:104CF000A07388000000EB0050079800D0408000AF
:104D00000080A000D04088000000EB004007980021
:104D1000090037004E00900080004000E0E02000D5
:104D2000808040000000EB00800878004E0090007A
:104D30000000E800400798004E009000F90F500076
:104D4000F4FF3400330437001E0090000000E00040
:104D500021003A007173800060E72000008040006D
:104D600090407800F0CDB30080CF500003003E00AB
:104D7000200020003007980029043700717380005C
:104D800060E7200000804000104078008080FB0039
:104D900000F22F00008040006007980070738000D0
:104DA0008000E80060E720000080400010407800AC
:104DB0000080FB004801DD00707380008080E80007
:104DC00060E7200000804000104078000080FB0079
:104DD00000007100500798000000EB0010079800D9
:104DE00070738000E300400060E720000080400016
:104DF000104078000080FB006101B90000F82F002E
:104E0000F1FF2F000201400083814800420F98000B
:104E1000530F980010022000010020004E0990005E
:104E2000DE099000800F5100818F5900ED033E0094
:104E30004E089000DE08900000600100210037005D
:104E400035003700E7033700E6033700710037000D
:104E500081003700A3003700B7003700BE003700DD
:104E60003B01370088013700DE033700EE013700D1
:104E70003502370099023700A0023700AE02370032
:104E8000BC023700CA023700D8023700D50337000A
:104E90007A0337005E033700D2033700D1033700AF
:104EA000E2023700F0023700A1033700AC033700FD
:104EB000000337001403370034033700B40337000E
:104EC000C503370010002000200798007073800091
:104ED0006600400070738800707380008080E90075
:104EE00060E7200000804000104078008080FB00D8
:104EF000F0FB2F0000844000A0FE070000017800B6
:104F000088004400E0E020000080400002087800B3
:104F100051FD0700B503370010002000200798005E
:104F2000707380006400400070738800C2FE070048
:104F30000000E0001C00320071738000310F980007
:104F400060E720003E09900000004100904078009A
:104F50008041EB004357980020C8B30080CF500039
:104F600002003A0010C0B30040579800BE089000FD
:104F70000100E800707388004E5190000204E000C8
:104F80009A03320010002000100798007073800010
:104F900063005000707388009403370070738000C2
:104FA0000000E800707388007173800060E72000E3
:104FB000008040009040780030C8B30080CF50009F
:104FC000070032007173800060E72000008040001D
:104FD0009040780000CEB30080CF5000EFFF360045
:104FE0007173800060E720000080400090407800EE
:104FF00030C8B30080CF50007C033A00100020007E
:1050000010079800707380000080E90070738800BA
:10501000760337001000200020079800707380008E
:10502000640040007073880054FE070022FD0700F2
:10503000000F78008081EB009E8F1100030032008A
:105040001E0078007073880068033700600020003D
:1050500030079800650337001000200020079800F3
:10506000707380006400400070738800907380004B
:10507000E90F500018003C009273800071738000AB
:105080006E009000008040008001E9008200410035
:1050900020E4200000804000030878009073800026
:1050A0000000E8009073880034FE070002FD07004E
:1050B000000F78008080EB009E8F1000030032000C
:1050C0001E017800727388004803370060002000DA
:1050D0003007980045033700700020003007980023
:1050E0004203370040892800D86B0200000000000E
:1050F0001000200020079800907380000000E0005E
:105100000A003200907380000000E900907388006C
:10511000907380008000400020E420000080400068
:105120001000780070738800300337008000200082
:10513000300798002D03370010002000200798004A
:10514000717380006E00900000804000630040009A
:105150007073880025033700100020002007980096
:10516000707380006400400070738800570037003F
:105170007173800060E7200000804000904078005C
:1051800020C2B30080CF50001F003A00707380002F
:105190000000E8007073880010003700D0408000E5
:1051A0000080A100D04088007173800060E720007B
:1051B0000080400010407800004178000100E800C5
:1051C0007073880002407800347002000000000014
:1051D000D04080000080A000D04088007173800023
:1051E00060E72000008040009040780020C2B300BB
:1051F00080CF5000E9FF3A00707380000000E800A3
:1052000070738800310037007173800060E7200000
:10521000008040009040780000C4B30080CF500070
:10522000070036007173800060E7200000804000B6
:1052300090407800A0C5B30080CF50000D0036002C
:105240007173800060E7200000804000104078000B
:105250000004E00013003D007173800060E720004F
:105260000080400090407800F0CDB30080CF500027
:105270000C003E00C1FD0700000F7800D040800008
:105280000080A100D04088001E007800126E02004D
:1052900000000000D04080000080A000D0408800C6
:1052A0000A0037007173800060E720000080400032
:1052B00090407800B0C3B30080CF500003003A00A4
:1052C000707380000000E8007073880071738000C4
:1052D00060E720000080400090407800F0CDB300EF
:1052E00080CF500007003E007173800060E720000F
:1052F000008040009040780030C8B30080CF50005C
:105300009BFF3A00707380008000E90060E7200096
:105310000080400090407800B0C3B30080CF5000C0
:1053200009003200D04080000080A100D0408800F9
:10533000A0922800046C020000000000D040800011
:105340000080A000D040880043FC0700A70237007F
:105350001000200020079800D04080000080A100AD
:10536000D040880070738000640040007073880033
:105370007173800060E7200000804000904078005A
:1053800020C2B30080CF500018003A007073800034
:105390000000E800707388000A0037007173800015
:1053A00060E7200000804000104078000041780055
:1053B0000100E80070738800024078003470020039
:1053C000000000007173800060E720000080400052
:1053D0009040780020C2B30080CF5000EFFF3A0029
:1053E000707380000000E8007073880071738000A3
:1053F00060E720000080400090407800C0C2B30009
:1054000080CF500004003A00707380000000E80074
:1054100070738800020037003000200030079800C9
:105420007173800060E72000008040001040780029
:105430008080FB00F0FB2F00008440008001EB0027
:10544000F2FF27008000EB000000EB00DC1C0200F4
:10545000000000000001780088004400E0E0200027
:105460000080400002087800707380000000E800AF
:1054700070738800F8FB0700D04080000080A00017
:10548000D040880059023700100020002007980003
:105490007073800064004000707388008073800027
:1054A000E30F500004003C00807380000000E8001F
:1054B0008073880002003700400020003007980009
:1054C000827380007373800060E7200000804100D9
:1054D000104078008080FB0000FC2F00008240001C
:1054E0006610B9008080E80060E520000080400080
:1054F000040878000300E80070738800717380006E
:1055000060E720000080400090407800D0C3B300E6
:1055100080CF500011003A00707380000000E80056
:1055200070738800807380006600B9008080E80096
:1055300060E5200000804000100078000004E900D1
:105540000EFD07000001780088004400E0E0200024
:105550000080400002087800020037003000200080
:105560003007980073738000130F980060E72000E5
:105570009E08900000804000904078000041EB00C1
:1055800002579800B0C8B30080CF500002003A0024
:1055900013C0B300035798009E0890000100E80074
:1055A000707388000E5190000204E0000900320080
:1055B00088738000F1FC0700000178006640B900A4
:1055C000E400400060E52000008040000208780010
:1055D000020037003000200030079800717380000F
:1055E00060E720000080400090407800F0CDB300DC
:1055F00080CF5000080036008073800072738000F6
:105600006600B9008000780060E52000008040005E
:1056100002087800020037003000200030079800B0
:105620008DFB0700F10137001000200020079800D3
:105630007073800064004000707388007273800093
:1056400060E7200000004100104078008080FB00EF
:1056500000FC2F00008F40000200E80070738800FB
:1056600050002000300798000000EB004007980031
:105670002F0037004E0090006600B9008080E800DF
:1056800060E5200000804000100078009E0F500070
:1056900024003A001E00E90080004000E0E0200005
:1056A00000804000100178004E0090006600B900B4
:1056B000E400400060E52000008040001000780019
:1056C000800F510012003D009E00E9000181400062
:1056D000E0E0200000004100100078000001E80038
:1056E00081804000E0E02000008040000208780057
:1056F0004E0090006600B9008000780060E5200050
:1057000000804000100078007073880003003700AC
:10571000807380000000E900807388000000EB00C7
:10572000300798004E0090000000E8004007980005
:10573000817380004E009000810F5000CDFF340037
:1057400045FB0700A9013700100020002007980042
:10575000707380006400400070738800A073800044
:105760000000E00027003A000000EB00400798002E
:105770000A003700CE00900060E720000080400063
:10578000104078008080FB004E0090008080400038
:1057900030F22F0000804000400798004E0090003B
:1057A000E300400060E72000008040009040780067
:1057B000E0C8B30080CF500006003200CE00900059
:1057C00060E7200000804000104078000004E00006
:1057D000E8FF3A00CE00900060E720000080400023
:1057E000104078000004E000040032004E009000F9
:1057F00064004000A0738800020037009000200081
:105800003007980073738000030F7800A073800046
:10581000707388009E00780060E7200000804000E0
:10582000104078008080FB00F0FB2F0000844000D7
:1058300055FB07000001780088004400E0E02000EC
:10584000008040000208780070738000A073880018
:105850001E00E80070738800A173800060E72000DC
:105860000080400090407800C0C2B30080CF50005C
:1058700003003A00A07380000000E800A0738800D5
:10588000A173800060E72000008040009040780015
:1058900000CEB30080CF50000E003600A073800011
:1058A000E300400060E72000008040009040780066
:1058B000E0C8B30080CF5000030032000000EB00CE
:1058C000A073880003003700A073800064004000CC
:1058D000A0738800E0FA07004401370010002000A0
:1058E00020079800717380006E00900000804000D7
:1058F00063004000707388003C01370010002000F6
:105900002007980070738000640040007073880066
:10591000A1408000E00220000088B90080007800EB
:10592000E09320000080400010007800000001009B
:10593000C9FA07002D013700100020002007980049
:10594000707380006400400070738800A140800084
:10595000E00220000088B9008080E800E093200089
:10596000008040001000780000000100BAFA070033
:105970001E0137001000200020079800707380007F
:105980006400400070738800A1408000E0022000A5
:105990000088B900E4004000E0932000008040004F
:1059A0001000780000000100ABFA07000F0137007B
:1059B00010002000200798007073800064004000F1
:1059C00070738800A1408000E00220000088B900C8
:1059D000E6004000E09320000080400010007800C6
:1059E000000001009CFA07000001370010002000B1
:1059F0002007980070738000640040007073880076
:105A0000A1408000E00220000088B900E8004000CA
:105A1000E09320000080400010047800D7FB0700CE
:105A2000080001008CFA0700F00037001000200089
:105A30002007980070738000640040007073880035
:105A4000CEFB07000000E00003003200FE7C0200F5
:105A50000000000002003700207D0200000000006E
:105A60007DFA0700E10037001000200020079800B1
:105A7000707380006400400070738800BFFB0700F3
:105A80000000E00005003200C082A900C282A80028
:105A9000C8A2A900CAA2A80004003700C082A900B9
:105AA000C282A900C8A2A900CAA2A9006AFA070076
:105AB000CE0037001000200020079800707380008F
:105AC0006400400070738800ACFB07000000E00039
:105AD0000600320090B72000104078000000A000BF
:105AE00091B72000804878000500370090B720006B
:105AF000104078000000A00091B720008048780096
:105B000055FA0700B9003700100020002007980060
:105B100070738000640040007073880097FB07007A
:105B200030618800306180000000E00002003D002C
:105B30000000EB00306188003161800000FA200035
:105B4000808F50000200340000FA2000306188008D
:105B500040618000E10F500002003C002000200066
:105B6000406188004161800030062000808F500035
:105B7000020034003006200040618800A479020051
:105B80000000000034FA07009800370010002000E1
:105B900020079800707380006400400070738800D4
:105BA00076FB070040618800306180000000E00063
:105BB00002003D000000EB00306188003161800090
:105BC00000FA2000808F50000200340000FA20000C
:105BD0003061880040618000E10F500002003C000D
:105BE00020002000406188004161800030062000D4
:105BF000808F500002003400300620004061880091
:105C0000A47902000000000013FA070077003700B3
:105C1000100020002007980070738000640040008E
:105C20007073880055FB07000000E0000900320097
:105C3000A1408000E00220000088B900F000400090
:105C4000E093200000804000100078000000010078
:105C500008003700A1408000E00220000088B90061
:105C6000F2004000E0932000008040001000780027
:105C700000000100F8F907005C0037001000200068
:105C800020079800707380006400400070738800E3
:105C90003AFB0700700798007E009000E10F50006B
:105CA00010003200FE009000E28F5000160032001B
:105CB0007E0190000200E000010032001A0037006F
:105CC000A1408000E00220000088B900EE00400002
:105CD000E0932000008040001000780000000100E8
:105CE00011003700A1408000E00220000088B900C8
:105CF000EC004000E093200000804000100078009D
:105D00000000010008003700A1408000E0022000F0
:105D10000088B900F6004000E093200000804000B9
:105D20001000780000000100CBF907002F003700B9
:105D3000100020002007980070738000640040006D
:105D400070738800717380006E00900000804000C6
:105D50000000E90070738800BFF9070023003700D6
:105D6000100020002007980070738000640040003D
:105D70007073880001FB0700000F78001E00780098
:105D80006298020000000000B3F907001700370016
:105D9000100020002007980070738000640040000D
:105DA00070738800F5FA0700000F7800A1408000AA
:105DB000E00220000088B900FC004000E0932000D1
:105DC00000804000900078001E0078000100010073
:105DD000A1F90700050037001000200030079800E7
:105DE0000200370030002000300798002E0090009D
:105DF0000000E00005003A00717380006E00900022
:105E00000080400063004000707388000000EB00D9
:105E1000200798003E0090000000E000CAFB32001E
:105E2000D04080000080A100D04088003E0090005B
:105E3000E10F50001800320061002000A03A20005D
:105E4000569D0200000000003E009000126E02000D
:105E50000000000081002000003B2000569D020051
:105E6000000000005E009000126E020000000000C2
:105E7000B1002000803B2000569D02000000000081
:105E800070738000126E020000000000A0922800D3
:105E9000046C0200000000004F0478000080FA004B
:105EA000000006000200FA00000F780000C2B300F4
:105EB00034700200000000001E007800D86B020061
:105EC0000000000000C2B3003470020000000000B7
:105ED0000080FA00000006000400FA000000EB0059
:105EE000707388003F0037007173800060E7200006
:105EF0000080400090407800214798002E4090009C
:105F00000004E000040035002E40900034700200D0
:105F10000000000030003700AE40900000CEB3001B
:105F200080CF50001C003600A0922800046C0200B4
:105F300000000000707380008000E80060E720002F
:105F400000804000104078000080FB004801DD0028
:105F5000707380008080E80060E7200000804000CF
:105F6000104078000080FB0000004100000F780026
:105F7000707380000080E800707388001E00780055
:105F8000126E02000000000000C2B3003470020074
:105F9000000000001000370000C2B300347002009F
:105FA000000000002E4090008080FB0000F82F00D1
:105FB000008040008000400020B3200000804000AE
:105FC00010007800D86B02000000000000C2B3008F
:105FD0003470020000000000707380000000E800D0
:105FE000707388007173800060E7200000804000BB
:105FF000104078000004E000BBFF3A00A0922800A7
:10600000046C020000000000707380000000E900D2
:10601000126E02000000000071002000303C2000E1
:10602000E09D0200000000000080FA000000060071
:106030000600FA001007980060698000000F7800E1
:10604000170037001E009000104178006169800041
:10605000A0C220000080400010407800804F510016
:10606000050032001E007800606988000000EB0027
:106070002007980010003700606980000000E800E9
:106080006069880061698000F00F20000080600076
:10609000606988001E0090000000E800100798006A
:1060A0001E009000104078000004E000E5FF3A0078
:1060B00010002000200798002E0090000080FA00B9
:1060C000000006000400FA000000EB00000F78005A
:1060D000100037001E0078008000400020B3200030
:1060E0000080400010007800D1FF07000000E000B1
:1060F000070032001E0078008040780000C8B3001E
:1061000000C040000080FB00100798000600370028
:106110001E0FE800000220009E0F1000EDFF34006B
:106120000000EB00100798001E0090000080FA00AD
:10613000000006003200FA006069800060079800E5
:106140001F003700EE009000A0C220000080400039
:106150009040780000C6B30080CF5000110034009A
:10616000EE009000A0C22000008040009040780027
:10617000A0C7B30080CF50000A003C006E01900021
:10618000EE009000A0C22000008040009040780007
:10619000F0CDB30080C06000A0C22000000041002C
:1061A000014878006E0090000000E8006007980049
:1061B000EE009000F00F2000008060006007980063
:1061C000EE00900050698000808F5000DDFF3A00A3
:1061D0000000EB006007980061698000A0C2200009
:1061E0000080400090407800F0C2B30080CF5000A3
:1061F0001F01340061698000A0C2200000804000BF
:106200009040780090C3B30080CF500018013C004C
:106210000000EB0060079800070037006E01900057
:10622000EE0047000040EB0000F178006E009000A7
:106230000000E80060079800EE00900020022000B7
:10624000808F5000F5FF340090160200000000001F
:10625000400798004E0090004880DE0080407800A3
:106260006E004700114098004E009000804078007A
:1062700000C0EB0080C060006E0047002140980025
:106280004E0090008CF80700300798003E00900008
:10629000E10F40002B003200BE00900060E72000BC
:1062A00000804000104078008080FB0030F22F001A
:1062B00000804000100798003E00900060079800A2
:1062C0000D0037006E019000EE0090001E0090005F
:1062D0008080400060E7200000804000904078000F
:1062E00060E7200000004100014878006E00900047
:1062F0000000E80060079800014020001E009000A8
:10630000808050006E009000808F5000EDFF3C00B8
:1063100008003700EE00900060E720008080400019
:106320000040EB00804878006E0090000000E8001C
:1063300060079800EE009000F03F2000808F500032
:10634000F4FF340030002000600798000000EB00EC
:10635000000F7800661A0200000000003E003700BF
:106360001E00E00002003A00661A02000000000071
:106370001E00E00004003A0052FF07000080FB000E
:1063800040079800020037000000EB00400798002B
:106390004E0090000000E0000C0032006E01900002
:1063A0004E009000804078006E0047000171780038
:1063B000CE00900070082000808F50001A003A0034
:1063C00010002000000F780017003700616980007E
:1063D000A0C22000008040009040780020C2B3009E
:1063E00080CF500001003A001E00A2006E01900014
:1063F00061698000A0C22000008040001040780049
:10640000804078006E00470001717800606980006C
:106410000000E8006069880061698000F00F2000DA
:1064200000806000606988006E0090000000E80055
:1064300060079800EE00900030022000808F50002E
:106440000500340091002000A03C2000E09D0200E7
:1064500000000000E500370061698000506980009D
:10646000808F5000BEFF3A006E009000E30F500096
:10647000DE0032006E009000E40F5000DB003200BE
:106480006E00900080407800C0CDB30000C0400096
:10649000804078006E004700014878000000EB0063
:1064A000600798000000EB00200798000000EB0058
:1064B000300798003D003700EE00900060E72000B4
:1064C000008040009040780000CEB30080CF5000A4
:1064D00025003600EE00900060E7200000804000BC
:1064E000104078008080FB0000F22F000080400008
:1064F000100798006E0090008000E80060E7200020
:1065000000804000904078006E00470010409000EE
:1065100080CF50000E003E006E0090008080E800AA
:1065200060E7200000804000904078006E00470047
:106530002040900080CF500005003100EE00900018
:106540001E0090000080400063004000300798006B
:106550009E0090006E0090000080400063004000AC
:1065600060079800020037006E0090002007980036
:106570006E0090008000E80060E72000008040008E
:10658000104078000080FB004801DD006E009000A4
:106590008080E80060E72000008040001040780024
:1065A0000080FB0000004100400798002E00900092
:1065B0000000E000C0FF32006E004700104078008D
:1065C0008080FB0030F22F000080400040079800E0
:1065D0002E009000600798000D003700EE0090003C
:1065E0004E00900000814000EE00900060E7200027
:1065F000008040009040780060E7200000004100EB
:10660000014878006E0090000000E90060079800E3
:10661000EE0090003E009000808F5000EFFF3D00A4
:106620000000EB00600798000C003700BE009000EF
:106630006E00900000814000EE0090006E00470068
:10664000E140780060E72000000041000148780048
:106650006E0090000000E80060079800EE009000D7
:106660004E009000808F5000F0FF35005F00370033
:10667000B09228006EFE07000000E0000500320026
:106680008CF90700A0922800046C020000000000B2
:1066900056003700F092280065FE07000000E00079
:1066A000020032000CFE0700500037004093280023
:1066B0005FFE07000000E00004003200D0408000D0
:1066C0000090A100D0408800480037009093280037
:1066D00057FE07000000E000200032000000EB0041
:1066E00060079800180037000000EB005007980082
:1066F0000F003700EE0090005E00900080804000A8
:1067000060E7200000804000104078000080FB001F
:10671000D26E02000000000000C2B300347002001C
:10672000000000005E0090000000E80050079800A4
:106730005E009000EF0F5000EEFF34006E009000FE
:106740007000400060079800EE009000F03F2000CD
:10675000808F5000E4FF340024003700F0932800BD
:1067600033FE07000000E0001C0032000000EB00D8
:106770006007980008003700EE00900060E72000F6
:10678000808040000040EB00804878006E00900060
:106790000000E80060079800EE009000F03F200045
:1067A000808F5000F4FF340011CEB30060E720006A
:1067B0000148780080C0EB0070E7200001487800B5
:1067C00080C0EB0080E720000148780011CAB300C8
:1067D00090E720000148780004003700C100200045
:1067E000303D2000E09D0200000000000080FA0023
:1067F0000000060057524900544520004249540009
:106800003A2020002A6E650078742000636C6F00C7
:10681000636B2000285E2900207769006C6C2000E3
:1068200075736500207468006973200076616C00E0
:106830007565310057495200452072006F7574002C
:10684000696E650073202800432920003230300033
:1068500030204D006963680061656C002050650060
:1068600061726300652047004E55200047504C0080
:106870004E6F200064657600696365002C2074000B
:106880007279200028414C0041524D0029205300CC
:1068900045415200434820006D616300726F200043
:1068A00066697200737441004444520045535300BA
:1068B000204D410043524F00202030002E4D6100FA
:1068C00063726F00206D65006E754D00616372002C
:1068D0006F20200020202000315749005245200021
:1068E0006164640072657300730D0A00202020004B
:1068F0002A3157004952450020524F004D20430095
:106900004F4D4D00414E4400204D410043524F0039
:10691000733A0D000A203500312E520045414400E3
:1069200020524F004D2028003078330033292000BA
:106930002A666F0072207300696E67006C65200024
:10694000646576006963650020627500730D0A0056
:10695000203835002E4D41005443480020524F004E
:106960004D20280030783500352920002A666F0038
:106970006C6C6F007765640020627900203634000B
:1069800062697400206164006472650073730D00B5
:106990000A20320030342E00534B49005020520060
:1069A0004F4D20002830780043432900202A6600FC
:1069B0006F6C6C006F776500642062007920630063
:1069C0006F6D6D00616E64000D0A20003233360079
:1069D0002E414C0041524D0020534500415243008E
:1069E000482028003078450043290D000A20320055
:1069F00034302E00534541005243480020524F008E
:106A00004D20280030784600302941004C4152008A
:106A10004D20530045415200434820002830780063
:106A20004543290053454100524348002028300087
:106A30007846300029446500766963006520490086
:106A400044732000617265002061760061696C000A
:106A500061626C006520620079204D004143520064
:106A60004F2C20007365650020283000292E52002D
:106A70004541440020524F004D202800307833001B
:106A800033293A00204D41005443480020524F0022
:106A90004D20280030783500352953004B495000EF
:106AA00020524F004D2028003078430043295500E4
:106AB0006E6B6E006F776E00206D610063726F0009
:106AC0002C207400727920003F206F007220280073
:106AD00030292000666F7200206865006C704200EB
:106AE0005553200052455300455420005761720011
:106AF0006E696E00673A20002A5368006F72740056
:106B0000206F7200206E6F00207075006C6C2D007D
:106B1000757020002A4E6F0020646500766963005E
:106B2000652064006574650063746500642044003A
:106B30005331380053323000204869006768200024
:106B40005072650073204400696720005468650036
:106B5000726D4400533138004232300020507200D0
:106B60006F6720005265730020446900672054005D
:106B7000686572006D4453003138320032204500A0
:106B8000636F6E00204469006720540068657200DE
:106B90006D4453003234300034204500636F6E0082
:106BA00072616D00207469006D65200043686900A2
:106BB0007044530032343300312031004B20450003
:106BC000455052004F4D55006E6B6E006F776E0052
:106BD0002064650076696300655057004D206400AD
:106BE00069736100626C650064314B00487A2D0066
:106BF000342C300030304B00487A200050574D0084
:106C000046726500717565006E63790020696E00DB
:106C1000204B48007A2050007265730063616C005D
:106C2000653A500052323A0044757400792063008E
:106C300079636C00652069006E20250020505700A4
:106C40004D206100637469007665450052524F0023
:106C5000523A200050574D0020616300746976005D
:106C6000652C2000672074006F2064006973610048
:106C7000626C6500415558002046720065717500D0
:106C8000656E6300793A20004155580020494E0056
:106C9000505554002F4849002D5A410055582000A6
:106CA000484947004841550058204C004F5756006E
:106CB0004F4C54004D455400455220004D4F440068
:106CC00045564F004C5441004745200050524F005C
:106CD00042453A002056450072726F007228290022
:106CE00020406C00696E65003A20400070676D00BE
:106CF0007370610063653A00206279007465730007
:106D00002E546F006F206C006F6E67002153790066
:106D10006E7461007820650072726F00724E6F00B1
:106D20002045450050524F004D4572006173690087
:106D30006E6764006F6E650053617600696E670070
:106D400020746F0020736C006F742000496E760011
:106D5000616C6900642073006C6F74004C6F61009B
:106D600064696E0067206600726F6D0020736C00AE
:106D70006F742000455252004F523A0020636F005A
:106D80006D6D61006E64200068617300206E6F009D
:106D900020656600666563007420680065726500A2
:106DA00041434B004E4143004B49320043205300C6
:106DB00054415200542042004954490032432000BB
:106DC00053544F00502042004954490032432000A0
:106DD0006D6F6400653A0D000A2031002E205300CB
:106DE0006F66740077617200650D0A0020322E0014
:106DF0002048610072647700617265005365740019
:106E000020737000656564003A0D0A0020312E0081
:106E1000207E35004B487A000D0A2000322E2000DB
:106E20007E3530004B487A000D0A2000332E2000BA
:106E30007E313000304B48007A0D0A0020342E009D
:106E4000207E340030304B00487A570041524E00CB
:106E5000494E47003A2048004152440057415200F1
:106E600045204900324320006973200062726F00A0
:106E70006B656E00206F6E002074680069732000DF
:106E8000504943002120280052455600204133003C
:106E9000295365007420730070656500643A0D0025
:106EA0000A2031002E20310030304B00487A0D008E
:106EB0000A2032002E20340030304B00487A0D007A
:106EC0000A2033002E2031004D487A004932430019
:106ED00020286D006F64200073706400293D280035
:106EE000202030002E4D610063726F00206D650020
:106EF0006E750D000A2031002E3762006974200083
:106F000061646400726573007320730065617200D0
:106F100063680D000A2032002E49320043207300BE
:106F20006E69660066657200536561007263680091
:106F3000696E67002049320043206100646472007A
:106F40006573730020737000616365002E20460036
:106F50006F756E0064206400657669006365730078
:106F6000206174003A536E006966660065722800FD
:106F70004241530049432900526561006479610030
:106F80002F412F00402063006F6E7400726F6C0001
:106F9000732041005558200070696E00612F410038
:106FA0002F402000636F6E0074726F006C732000BE
:106FB0004353200070696E00436F6D006D616E0079
:106FC00064206E006F742000757365006420690092
:106FD0006E20740068697300206D6F006465500056
:106FE000756C6C002D7570002072650073697300FC
:106FF000746F720073204F0046465000756C6C0031
:107000002D7570002072650073697300746F7200D3
:1070100073204F004E5365006C662D00746573003D
:10702000742069006E204800695A20006D6F64006A
:1070300065206F006E6C7900524553004554420044
:107040004F4F54004C4F41004445520041555800A9
:1070500020494E00505554002F4849002D5A2C000D
:107060002052450041443A0020506F00776572007D
:107070002073750070706C0069657300204F4E00BE
:10708000506F77006572200073757000706C690036
:10709000657320004F464600444154004120530090
:1070A00054415400453A200044454C0041592000C9
:1070B0007573570052495400453A2000524541002B
:1070C000443A2000434C4F00434B2C0020314300F6
:1070D0004C4F43004B2C20003044410054412000D1
:1070E0004F555400505554002C2031004441540059
:1070F00041204F005554500055542C0020302000A2
:107100002A7069006E20690073206E006F7720007E
:1071100048695A00434C4F00434B200054494300F8
:107120004B533A002052450041442000424954004C
:107130003A205300796E7400617820006572720005
:107140006F72200061742000636861007220780013
:107150002E206500786974002877690074686F00D4
:1071600075742000636861006E676500296E6F00AA
:10717000206D6F0064652000636861006E676500C4
:107180004E6F6E0065786900737465006E74200040
:1071900070726F00746F63006F6C2100782E200096
:1071A00065786900740D0A00496E7600616C6900AB
:1071B00064206300686F690063652C0020747200AE
:1071C00079206100676169006E44450056494400BA
:1071D0003A68740074703A002F2F6400616E670083
:1071E00065726F0075737000726F74006F74790050
:1071F000706573002E636F006D2A2D002D2D2D00FC
:107200002D2D2D002D2D2D002A4F7000656E200094
:1072100064726100696E20006F757400707574008F
:1072200073202800483D4800692D5A002C204C004E
:107230003D474E0044294E006F726D00616C200086
:107240006F7574007075740073202800483D33001A
:107250002E3376002C204C003D474E0044294D0033
:1072600053422000736574003A204D004F53540080
:1072700020736900672062006974200066697200EB
:1072800073744C0053422000736574003A204C0024
:1072900045415300542073006967200062697400FF
:1072A000206669007273740020426F006F746C0076
:1072B0006F61640065722000762031002E20480046
:1072C00045580D000A2032002E20440045430D0091
:1072D0000A2033002E204200494E0D000A203400BF
:1072E0002E20520041574400697370006C61790090
:1072F00020666F00726D6100742073006574560023
:107300006F6C740061676500206D6F006E697400BA
:107310006F7273003A203500563A2000207C20001E
:10732000332E3300563A2000207C20005650550062
:107330004C4C5500503A2000536574002073650092
:10734000726961006C2070006F72740020737000AD
:10735000656564003A20280062707300290D0A00F8
:1073600020312E0020333000300D0A0020322E0054
:107370002031320030300D000A2033002E20320040
:10738000343030000D0A2000342E20003438300014
:10739000300D0A0020352E002039360030300D0027
:1073A0000A2036002E20310039323000300D0A001C
:1073B00020372E0020333800343030000D0A2000F2
:1073C000382E20003537360030300D000A203900C5
:1073D0002E2031003135320030300D000A313000BE
:1073E0002E20420052472000726177002076610013
:1073F0006C75650041646A007573740020796F00D4
:1074000075722000746572006D696E00616C4100D8
:1074100072652000796F75002073750072653F00FA
:107420002043460047313A002043460047323A00A5
:10743000285C2D002F5F5C002D2928005C5F2F0049
:107440002D295300656C6500637420006F7574000E
:10745000707574002074790070653A000D0A200080
:10746000312E20004F7065006E206400726169004B
:107470006E202800483D4800692D5A002C204C0001
:107480003D474E0044290D000A2032002E204E00B8
:107490006F726D00616C200028483D00332E330070
:1074A000562C20004C3D47004E44290052325700D4
:1074B000202873007064200068697A00293D280044
:1074C000202030002E4D610063726F00206D65003A
:1074D0006E750D000A2031002E4953004F373800D9
:1074E00031362D003320410054520D000A20320065
:1074F0002E4953004F37380031362D0033207000AD
:107500006172730065206F006E6C790049534F0003
:107510002037380031362D003320410054522000EE
:107520002852450053455400206F6E0020435300FD
:10753000290D0A0052455300455420004849470090
:10754000482C2000434C4F00434B2000544943003B
:107550004B2C200052455300455420004C4F5700FF
:1075600049534F002037380031362D003320720048
:1075700065706C00792028007573650073206300C6
:1075800075727200656E7400204C530042207300C7
:1075900065747400696E6700293A200050726F00AC
:1075A000746F63006F6C3A0020736500726961004C
:1075B0006C332000776972006532200077697200B1
:1075C0006552460055756E006B6E6F00776E520007
:1075D000656164002074790070653A0020746F0062
:1075E00020656E006476610072696100626C6500FE
:1075F000206C65006E67740068446100746120004F
:10760000756E690074733A00206E6F0020696E0019
:1076100064696300617469006F6E440061746100A5
:1076200020756E00697420006C656E0067746800D8
:107630002028620069747300293A20004353200017
:10764000454E4100424C450044435300204449000C
:10765000534142004C4544005233570020287300E8
:107660007064200063736C00206869007A293D0013
:10767000282029000D0A4400697363006F6E6E00B4
:107680006563740020616E0079206400657669008E
:10769000636573000D0A43006F6E6E0065637400CE
:1076A0002028560070752000746F20002B3556007E
:1076B000292061006E6420002841440043207400AA
:1076C0006F202B00332E33005629430074726C0058
:1076D000415558004D4F440045204C004544500052
:1076E000554C4C0055502000485055004C4C55000E
:1076F0005020480056524500474144004320610055
:107700006E64200073757000706C790035565600F9
:10771000505533002E3356004144430042757300E8
:1077200020686900676842007573200048692D0071
:107730005A20300042757300204869002D5A2000FD
:10774000314D4F0044452000616E640020565200C8
:10775000454720004C45440073207300686F750056
:107760006C642000626520006F6E2100466F75001A
:107770006E64200020657200726F7200732E4D00DF
:107780004F534900434C4B004D4953004F43530066
:10779000204F4B0020464100494C530065742000A7
:1077A0007370650065643A000D0A2000312E2000D8
:1077B00033304B00487A0D000A2032002E20310071
:1077C00032354B00487A0D000A2033002E2032005B
:1077D00035304B00487A0D000A2034002E2031004D
:1077E0004D487A00436C6F00636B2000706F6C0033
:1077F0006172690074793A000D0A2000312E200070
:1078000049646C0065206C006F7720002A64650075
:10781000666175006C740D000A2032002E2049004C
:10782000646C65002068690067684F0075747000BB
:1078300075742000636C6F00636B200065646700E3
:10784000653A0D000A2031002E204900646C650065
:1078500020746F002061630074697600650D0A0072
:1078600020322E0020416300746976006520740088
:107870006F206900646C6500202A64006566610001
:10788000756C7400496E70007574200073616D0032
:10789000706C650020706800617365003A0D0A0025
:1078A00020312E00204D690064646C0065202A00A0
:1078B0006465660061756C00740D0A0020322E004C
:1078C00020456E0064535000492028007370640006
:1078D00020636B00702073006B652000736D700077
:1078E000206373006C206800697A29003D2820001D
:1078F00020302E004D616300726F20006D656E00B8
:10790000750D0A0020312E00536E69006666200056
:10791000435320006C6F77000D0A2000322E530075
:107920006E696600662061006C6C200074726100F4
:1079300066666900632D7000202D6600202A4200D3
:107940007974650073206400726F70007065640064
:107950002A464100494C4500442C20004E4F20004F
:107960004441540041446100746120006269740024
:10797000732061006E642000706172006974790088
:107980003A0D0A0020312E0020382C00204E4F00E6
:107990004E4520002A646500666175006C74200005
:1079A0000D0A2000322E2000382C200045564500BC
:1079B0004E200D000A2033002E2038002C204F00CE
:1079C000444420000D0A2000342E2000392C2000D1
:1079D0004E4F4E00455374006F7020006269740072
:1079E000733A0D000A2031002E203100202A640055
:1079F00065666100756C74000D0A2000322E20004F
:107A0000325265006365690076652000706F6C0016
:107A10006172690074793A000D0A2000312E20004D
:107A200049646C0065203100202A640065666100AD
:107A3000756C74000D0A2000322E200049646C0021
:107A400065203000554152005420280073706400B6
:107A50002062720067206400627020007362200060
:107A600072787000206869007A293D002820200083
:107A7000302E4D00616372006F206D00656E7500E1
:107A80000D0A2000312E540072616E007370610087
:107A900072656E00742062007269640067650D0093
:107AA0000A2032002E204C0069766500206D6F00A0
:107AB0006E6974006F720D000A2033002E4272004E
:107AC00069646700652077006974680020666C004F
:107AD0006F772000636F6E0074726F006C55410009
:107AE0005254200062726900646765005265730039
:107AF00065742000746F200065786900745261001D
:107B0000772055004152540020696E007075740052
:107B10005541520054204C0049564500204449002C
:107B200053504C0041592C00207D2000544F200020
:107B300053544F00504C49005645200044495300CF
:107B4000504C410059205300544F500050454400C0
:107B5000574152004E494E00473A200070696E006E
:107B600073206E006F7420006F7065006E206400DB
:107B7000726169006E20280048695A00292052006D
:107B800045564900443A0D000A496E0076616C0082
:107B90006964200063686F00696365002C207400CD
:107BA0007279200061676100696E6D007352530045
:107BB000204C4F00572C2000434F4D004D414E00AC
:107BC00044204D004F44450052532000484947008F
:107BD000482C20004441540041204D004F444500B2
:107BE000416464007265730073206F00662050006A
:107BF00043463800353734003F546800697320002D
:107C00006D6F6400652072006571750069726500B2
:107C1000732061006E206100646170007465720001
:107C20004C4344002074790070653A000D0A20002E
:107C3000312E2000484434003437380030202800EA
:107C4000757369006E672000504346003835370071
:107C5000342049004F206500787061006E64650033
:107C600072294C0043442000287479007020610080
:107C70006464720029203D002028200020302E005E
:107C80004D616300726F20006D656E00750D0A0016
:107C900020312E004C43440020526500736574006F
:107CA0000D0A2000322E49006E697400204C4300FA
:107CB000440D0A0020332E00436C650061722000E1
:107CC0004C4344000D0A2000342E430075727300AB
:107CD0006F722000706F7300697469006F6E20000E
:107CE00065783A002834290020300D000A2036003B
:107CF0002E5772006974650020746500737420004B
:107D00006E756D006265720073206500783A280018
:107D10003629200038300D000A2037002E57720017
:107D200069746500207465007374200063686100E5
:107D3000726163007465720073206500783A2800F0
:107D40003729200038304400697370006C61790075
:107D5000206C69006E6573003A0D0A0020312E0018
:107D6000203120000D0A2000322E20004D756C00BD
:107D7000746970006C6549004E495400434C4500DD
:107D800041524300555253004F5220005345540076
:107D90004E6F200041434B002C2063006865630058
:107DA0006B2061006461700074657200434C4B008D
:107DB000094D4F0053490900435309004D495300F1
:107DC0004F5069006E73740061746500733A470028
:107DD0004E440900332E3300560935002E3056002C
:107DE00009414400430956005055090041555800C7
:107DF00009500900500950000949090049092D009E
:107E0000094F570044092D00092D2D000954780011
:107E100044092D0009527800445343004C09530093
:107E2000444109002D092D005047430009504700E7
:107E300044092D00092D31002E2842005229090045
:107E4000322E28005244290009332E00284F5200B8
:107E5000290934002E28590057290900352E2800F9
:107E6000474E290009362E0028424C0029093700C8
:107E70002E28500055290900382E28004752290085
:107E800009392E0028575400290930002E284200B5
:107E90006C6B2900474E440009474E0044094100DD
:107EA00044430900352E3000560933002E33560066
:107EB000095650005509410055580900657865007C
:107EC0006375740065203A0020205400494D450038
:107ED0004F55540020302E00204D610063726F001A
:107EE000206D65006E750D000A2031002E204C00BB
:107EF0006976650020696E0070757400206D6F00F2
:107F00006E6974006F7249006E70750074206D00A8
:107F10006F6E6900746F7200202A730074617200C2
:107F2000746269007420650072726F0072202A000A
:107F3000706172006974790020657200726F72005E
:107F4000202A7300746F70006269740020657200EB
:107F5000726F7200204E4F004E452000554E4B0070
:107F60004E4F57004E20450052524F0052206100A4
:107F700075746F0072616E00676520002B4D4800BC
:107F80007A292B006B487A0029526100772076000D
:107F9000616C7500652066006F72200042524700D8
:107FA00020284D00494449003D313200372957000F
:107FB00041524E00494E47003A2050006F73730003
:107FC00069626C00652062007566660065726F000C
:107FD00076657200666C6F0077416E0079206B00E9
:107FE00065792000746F2000657869007453700013
:107FF0006163650020746F0020636F006E74690018
:108000006E7565004E756D0062657200206F6600CA
:10801000206269007473200072656100642F77002C
:1080200072697400653A200043533A000D0A20003B
:10803000312E200043530D000A2032002E202F0045
:10804000435320002A646500666175006C74470024
:10805000656E650072616C0009090900090950002C
:10806000726F74006F636F006C2069006E7465003E
:108070007261630074696F006E2D2D002D2D2D002F
:108080002D2D2D002D2D2D002D2D2D002D2D2D00D4
:108090002D2D2D002D2D2D002D2D2D002D2D2D00C4
:1080A0002D2D2D002D2D2D002D2D2D002D2D2D00B4
:1080B0002D2D2D002D2D2D002D2D2D002D2D2D00A4
:1080C0002D2D2D002D2D2D002D2D2D002D2D2D0094
:1080D0002D2D2D002D2D2D002D2D2D002D3F090096
:1080E0005468690073206800656C70000909090014
:1080F00028302900094C69007374200063757200F0
:1081000072656E0074206D00616372006F733D00D4
:10811000582F7C00580943006F6E7600657274001A
:10812000732058002F726500766572007365200019
:108130005809090028782900094D610063726F0011
:1081400020787E00095365006C66740065737400C6
:10815000090909005B095300746172007423090066
:108160005265730065740900090909005D0953002F
:10817000746F700024094A00756D700020746F00E0
:1081800020626F006F746C006F616400657209009B
:10819000097B0900537461007274200077697400D0
:1081A0006820720065616400262F2500094465007F
:1081B0006C6179002031200075732F006D73090008
:1081C00009097D00095374006F7061002F412F0071
:1081D0004009410055585000494E2000286C6F005E
:1081E000772F4800492F52004541440029090900D2
:1081F000226162006322090053656E0064207300EF
:10820000747269006E676200095365007420620031
:1082100061756400726174006509090009313200FA
:1082200033632F00430941005558200061737300E8
:1082300069676E006D656E007420280061757800B6
:108240002F4353002909090030783100323364008C
:108250002F4409004D65610073757200652041006F
:1082600044432000286F6E0063652F00434F4E008B
:10827000542E290009306200313130000953650065
:108280006E64200076616C0075656600094D6500BE
:108290006173750072652000667265007175650016
:1082A0006E63790009097200095265006164670014
:1082B000094765006E657200617465002066720092
:1082C00065717500656E6300792F5000574D090088
:1082D000092F0900434C4B002068690068094300DE
:1082E0006F6D6D00616E640068697300746F720079
:1082F00079090900095C0900434C4B00206C6F00B0
:108300006909560065727300696F6E00696E6600D8
:108310006F2F730074617400757369006E666F006F
:1083200009095E0009434C004B20740069636B002F
:108330006C2F4C0009426900746F72006465720012
:1083400020286D0073622F004C5342002909090058
:108350002D0944004154200068696D0009436800FC
:10836000616E670065206D006F6465000909090092
:108370005F094400415420006C6F6F000953650091
:1083800074206F007574700075742000747970002B
:1083900065090900092E0900444154002072650056
:1083A000616470002F50090050756C006C7570008E
:1083B0002072650073697300746F72007320280067
:1083C0006F6666002F4F4E0029092100094269009F
:1083D0007420720065616400730953006372690060
:1083E00070742000656E6700696E650009090900F8
:1083F0003A0952006570650061742000652E6700BF
:108400002E2072003A31300076095300686F7700F1
:1084100020766F006C7473002F73740061746500B4
:10842000730909003B0942006974730020746F00EE
:108430002072650061642F00777269007465200006
:10844000652E67002E203000783535003B327700EE
:108450002F5709005053550020286F0066662F00E3
:108460004F4E290009093C00783E2F003C783D0022
:10847000203E2F003C303E000955730065726D00B0
:10848000616372006F2078002F6173007369670069
:108490006E2078002F6C690073742000616C6C0092
:1084A0000000FA00A0B92000104078000030A000C1
:1084B000A1B9200080487800A0B9200010407800C1
:1084C000704060000004E00002003200CAC2A9004F
:1084D00001003700CAC2A800A0B9200010407800EF
:1084E000704060000004E00003003200F0C2B300FE
:1084F0003470020000000000A100200060AB2000EA
:10850000E09D0200000000000080FA00000006006C
:108510000000FA00A0B92000104078000030A1004F
:10852000A1B9200080487800A0B920001040780050
:10853000704060000004E00002003200CAC2A900DE
:1085400001003700CAC2A800A0B92000104078007E
:10855000704060000004E00003003200F0C2B3008D
:108560003470020000000000A100200060AB200079
:10857000E09D0200000000000080FA0000000600FC
:108580000000FA00A0B920001040780070406000A0
:108590000004E00002003200CAC2A8000100370057
:1085A000CAC2A900A0B92000104078007040600045
:1085B0000004E00003003200F0C2B3003470020097
:1085C00000000000B100200000AC2000E09D02008F
:1085D000000000000080FA00000006000000FA0021
:1085E00000C0EB00270207000080FB000080FA00BB
:1085F000000006000600FA00100798001E00900018
:1086000020020700004F7800A0B920001040780039
:10861000684060000004E000030032001E80FB00A0
:108620002007980002003700001020002007980063
:108630002E0090000080FA00000006000000FA0002
:1086400001022000D0C92000569D02000000000059
:1086500080B7200010407800706E0200000000001B
:1086600000C2B3003470020000000000A0B9200076
:108670001040780061406000706E02000000000051
:1086800000C2B3003470020000000000A0B9200056
:10869000104078000080FB000000D10061406000C5
:1086A000706E02000000000000C2B30034700200CF
:1086B00000000000A0B92000104078000080FB00FE
:1086C0004200DE0061406000706E020000000000A9
:1086D00000C2B3003470020000000000A0B9200006
:1086E000104078000080FB004400DE006140600024
:1086F000706E02000000000000C2B300347002007F
:108700000000000090B72000104078000080FB00BF
:108710004300DE0061406000706E02000000000057
:1087200000C2B300347002000000000031002000DD
:10873000F0AD2000569D0200000000000080FA000D
:10874000000006000C00FA00661A0200000000009B
:10875000901602000000000050079800661A020000
:108760000000000090160200000000004007980082
:10877000661A0200000000009016020000000000CF
:1087800030079800661A02000000000090160200F0
:108790000000000020079800661A02000000000098
:1087A0009016020000000000000F7800661A020018
:1087B0000000000090160200000000001007980062
:1087C0005E0090000000E000090034005E009000B0
:1087D000E40F500006003C005E0090000040E900FD
:1087E0008040780080B72000014878000200370000
:1087F0000000EB00500798004E0090000000E000E1
:108800000F0034004E009000E20F50000C003C00BE
:108810004E0090000040E900E1406000A0B9200057
:108820001040780061C16000E1CFB30001406000FA
:1088300002407000A1B92000804878000200370093
:108840000000EB00500798003E0090000000E000A0
:10885000100034003E009000E20F50000D003C007C
:108860003E0090000040E90061416000A0B9200096
:10887000904078006140610000414000D0CFB300DB
:1088800080C0600082C07000A0B92000014878005C
:10889000020037000000EB00500798002E00900007
:1088A0000000E000100034002E009000E20F5000A5
:1088B0000D003C002E0090000040E9006141600086
:1088C000A0B9200090407800614061004201DD00C5
:1088D000B0CFB30080C0600082C07000A0B920009B
:1088E00001487800020037000000EB0050079800B4
:1088F0001E00E00010003400200020009E0F100039
:108900000D003C001E0078000040E900614160005D
:10891000A0B9200090407800614061004401DD0072
:10892000F0CEB30080C0600082C07000A0B920000B
:1089300001487800020037000000EB005007980063
:108940001E0090000000E000100034001E009000A7
:10895000E20F50000D003C001E0090000040EA00B5
:108960006141600090B72000904078006140610054
:108970004301DD0070CFB30080C0600082C0700092
:1089800090B7200001487800020037000000EB009B
:10899000500798005E0090000000E00079003A0067
:1089A0000000EB007069880071032000D0BB20003C
:1089B000E09D0200000000008001EB00420020006A
:1089C0001100200010002000DC1C0200000000004C
:1089D0000040E9008040780080B72000014878001E
:1089E0005103200040BF2000E09D02000000000075
:1089F0008001EB0022002000110020001000200068
:108A0000DC1C0200000000000040E900E1406000C2
:108A1000A0B920001040780061C16000E1CFB30030
:108A20000140600002407000A1B920008048780039
:108A30003104200090C22000E09D020000000000F0
:108A40008001EB0022002000110020002000200007
:108A5000DC1C0200000000000040E90061416000F1
:108A6000A0B92000904078006140610000414000C2
:108A7000D0CFB30080C0600082C07000A0B92000D9
:108A80000148780011032000C0C62000E09D0200CC
:108A9000000000008001EB002200200011002000F7
:108AA00010002000DC1C0200000000000040E90073
:108AB00061416000A0B920009040780061406100F1
:108AC0004201DD00B0CFB30080C0600082C0700002
:108AD000A0B9200001487800D101200070222100B7
:108AE000E09D0200000000008001EB002200200059
:108AF0001100200020002000DC1C0200000000000B
:108B00000040E90061416000A0B920009040780079
:108B1000614061004401DD00F0CEB30080C0600020
:108B200082C07000A0B9200001487800F104200044
:108B3000B0932000E09D0200000000008001EB00E7
:108B4000220020001100200010002000DC1C020088
:108B5000000000000040EA006141600090B7200082
:108B600090407800614061004301DD0070CFB300A8
:108B700080C0600082C0700090B72000014878007B
:108B800001003700ADFE0700A0B9200010407800BA
:108B90000030A100A1B920008048780080B72000F3
:108BA000104078008080FB00E081200000804000C1
:108BB000104078004B000700A0B92000104078005A
:108BC0000080FB004400DE00614060006140600006
:108BD0004601DD00A12C200091407800F0CBB300CD
:108BE00000C0600002407000CAE2B7000080FA00D6
:108BF000000006000000FA008E0007000080FA0066
:108C0000000006000400FA00000F78001E00780043
:108C1000100798001E009000E10F50000C00320079
:108C20001E009000E10F5000040039001E0090006B
:108C3000E20F5000120032001D00370041032000F7
:108C4000D0CB2000E09D0200000000001C00370097
:108C50007100200050592000E09D0200000000003B
:108C6000F1002000C01E2100E09D02000000000075
:108C700011C0B30010C0B30090000700100037000F
:108C80007100200050592000E09D0200000000000B
:108C9000F1002000C01E2100E09D02000000000045
:108CA00011C0B3000040EB0084000700040037004F
:108CB00041022000C0202000E09D020000000000D2
:108CC0000080FA00000006000000FA000101200008
:108CD000A0042100E09D0200000000000080FA00D6
:108CE000000006000200FA00004F780041E2A900EF
:108CF00090B7200010407800684060000004E00059
:108D000004003200CEE2A800CF02A800CEC2A80024
:108D100003003700CEE2A900CF02A900CEC2A9000D
:108D2000816A20009140780000CEB30000C060004E
:108D30007040B300A8E6B700916C20009140780025
:108D400000CEB30000C060007040B300C9E6B700B9
:108D5000816C20009140780000CEB30000C060001C
:108D60000034A000C8E6B700CAC2A800C8C2A90063
:108D7000C902A900C8E2A800C922A9001E80FB0000
:108D80001012880042A2A800A0B92000104078006C
:108D900061406000614060004601DD002124200048
:108DA00091407800F0CBB30000C06000024070003A
:108DB00042E2B700A0B92000104078000080FB001C
:108DC0000000D1006140600061416000312420005A
:108DD00091407800E0CFB30000C060000240700016
:108DE00043E2B700A0B92000104078000080FB00EB
:108DF0004200DE00614060006140600000414000D0
:108E00003124200091407800D0CFB30000C0600032
:108E10000240700043E2B7000000EB00201288001F
:108E20000000EB000012880041E2A8000080FA0078
:108E3000000006000000FA0041E2A900A8C6BF0039
:108E4000F041B300A8E6B700916C20009140780093
:108E500000CEB30000C06000C9E6B700816C2000FE
:108E60009140780000CEB30000C06000C8E6B700B3
:108E7000CEE2A900CF02A900CEC2A9000080FA006C
:108E8000000006000200FA00004F78001E80FB0080
:108E90004012880085C0BF00644060000004E0000C
:108EA000FCFF320040128000004F78008540A9008E
:108EB0001E80FB000080FA00000006000400FA009B
:108EC000204798003147980010C0B300004F780049
:108ED000DC70020000000000D6FF07007B000700E6
:108EE0002E4090000004E00002003A0042E2A80098
:108EF00062E2A8002E409000E14F500003003E00C7
:108F000041E2A80061E2A800000037001E04E00072
:108F100009003A00CAC2BF000044B2000004E000E9
:108F200005003200D0C5B300EA7002000000000066
:108F300010C0B300004F780040C2BF000042B20032
:108F40000004E0002F003A0060C2BF000042B200FF
:108F50000004E0002B003A00401280001047980007
:108F600010C0B3009E4F100005003A00B0C5B3001A
:108F7000EA700200000000000040EB00004F7800A3
:108F80003E4090000004E000050032001E409000CA
:108F90000080FB00FC6E02000000000006003700AD
:108FA000C0C5B300EA700200000000001E4090003F
:108FB000EA70020000000000401380001047980093
:108FC0003E4090000004E0000B00320080C2B3007D
:108FD000EA700200000000001E4090000080FB00CC
:108FE000FC6E02000000000090C2B300EA700200B4
:108FF00000000000030037001E409000EA700200ED
:109000000000000040C2BF000044B2000004E000C5
:1090100004003A0060C2BF000044B2000004E00057
:109020000A003200CA82A9003E4090000004E0001D
:109030000300320020A22800046C0200000000009F
:1090400040C2A90060C2A900130037001A710200D3
:109050000000000022C2BF00614060000004E00088
:10906000AAFF32003111800020072000808F5000BD
:1090700003003A0041E2A90061E2A900A3FF370022
:109080003E4090000004E0000300320030A32800BE
:10909000046C0200000000008B00070081C6BF00C6
:1090A000F041B30081E6B70080B72000104078009F
:1090B0008080FB00E08120000080400010407800AC
:1090C00008FF07000080FA00000006000000FA0018
:1090D000C8C2A800C902A800C8E2A800C922A80006
:1090E000A16A20009140780000CEB30000C060006B
:1090F0006040B300AAE6B700E16A20009140780022
:1091000000CEB30000C060006040B300AEE6B70020
:10911000816A20009140780000CEB30000C060005A
:109120009040B300A8E6B700916A20009140780013
:1091300000CEB30000C060000034A000A9E6B70074
:10914000C16A20009140780000CEB30000C06000EA
:109150007040B300ACE6B700D16A200091407800BF
:1091600000CEB30000C060000034A000ADE6B70040
:1091700080B72000104078008080FB00E081200054
:1091800000804000104078000080FB001012880032
:10919000A0B920001040780061406000614060008C
:1091A0004601DD002124200091407800F0CBB3007F
:1091B00000C060000240700042E2B700A0B9200089
:1091C000104078000080FB000000D100614060008A
:1091D000614160003124200091407800E0CFB3006D
:1091E00000C060000240700043E2B7000000EB00E6
:1091F000201288000000EB000012880080B72000D9
:10920000104078008080FB00E0812000008040005A
:10921000104078000080FB0010138800A0B92000E7
:109220001040780061406000614060004601DD0050
:109230002126200091407800F0CBB30000C06000F0
:109240000240700062E2B700A0B920001040780030
:109250000080FB000000D1006140600061416000BF
:109260003126200091407800E0CFB30000C06000BC
:109270000240700063E2B7000000EB00201388009A
:109280000000EB00001388000000EB004012880093
:109290000000EB00401388004322A9006322A900CC
:1092A0004362A80042A2A9006362A80062A2A900CA
:1092B00040C2A90060C2A9004402A8006402A8003C
:1092C0000080FA00000006000000FA0041E2A90058
:1092D0004362A90061E2A9006362A900AAC6BF00B7
:1092E000F041B300AAE6B700AEC6BF00F041B3003C
:1092F000AEE6B700A8C6BF00F041B300A8E6B700CD
:10930000A9C6BF00F041B300A9E6B700ACC6BF00D4
:10931000F041B300ACE6B700ADC6BF00F041B3000A
:10932000ADE6B7000080FA00000006000000FA0079
:1093300040A32800D86B0200000000000080FA0063
:10934000000006000400FA0011C0B30080B720003E
:1093500001487800A0B92000104078000000A1006A
:10936000A1B9200080487800A0B920001040780002
:109370000010A000A1B9200080487800A0B920000A
:10938000104078000020A100A1B92000804878009A
:1093900090B72000104078000030A00091B7200066
:1093A0008048780080B72000104078008080FB0063
:1093B00020822000008040001040780049FE070015
:1093C000DAFF07000000370022C2BF0061406000E2
:1093D0000004E000FCFF3200301180008040780083
:1093E00080B920000148780080B920001040780042
:1093F0000080FB004400DE008040780070B920004F
:109400000148780070B92000104078000080FB000F
:10941000100798001E009000E40F500082003200F8
:109420001E009000E40F500007003C001E0090005A
:109430000000E0000B0032001E009000E10F500021
:1094400053003200E40037001E009000E60F500089
:109450007D0032001E009000E80F50008F003200A7
:10946000DD00370080B92000104078000080FB004C
:10947000000F78001E007800E30F50002300320038
:109480001E007800E30F50000A003C001E00780028
:10949000E10F5000130032001E007800E10F500071
:1094A00012003C001E0078000000E0000B003200BB
:1094B000330037001E007800EE0F5000220032000B
:1094C0001E007800EF0F5000260032001E007800CA
:1094D000ED0F5000150032002900370055FE07003F
:1094E000C100370091FF0700B7FF3700601680000A
:1094F000F1FB2F00010060006016880010C0B3006F
:109500003470020000000000AFFF370060168000DA
:1095100001042000010070006016880010C0B30034
:109520003470020000000000A7FF37008040EB000D
:1095300020C0B30061FE070010C0B3003470020009
:1095400000000000A0FF37008040EB000040EB006F
:109550005AFE070010C0B300347002000000000083
:1095600099FF37008040EB0010C0B30053FE0700A6
:1095700010C0B300347002000000000092FF3700FA
:109580000040EB0034700200000000008EFF370046
:1095900080B9200090407800F0C0B30080C0600027
:1095A00080B920000148780080B920001040780080
:1095B0008040E80080B920000148780010C0B30066
:1095C00034700200000000008040EB0060B9200011
:1095D000014878000D00370022C2BF0061406000E2
:1095E0000004E000FCFF32003011800025FE07007F
:1095F000347002000000000060B9200010407800C4
:109600008040E80060B920000148780060B920007F
:109610009040780080B920001040780080CF500042
:10962000EDFF390068FF370080B920001040780056
:1096300038A002000000000010C0B3003470020027
:109640000000000060FF370080B9200090407800E3
:1096500070C0B30080C0600080B92000014878006D
:1096600080B920009040780080B720000148780041
:1096700080B72000104078008080FB00208220000E
:10968000008040001040780096FD070010C0B30035
:1096900034700200000000004BFF3700A0B920002A
:1096A000104078000000A100A1B920008048780097
:1096B000A0B92000104078000010A100A1B920003E
:1096C00080487800A0B92000104078000020A10058
:1096D000A1B920008048780090B7200010407800A1
:1096E0000030A10091B720008048780080B92000A8
:1096F000104078000080FB004200DE006100600046
:109700000004E00005003200A0B9200010407800FD
:109710000000A000A1B920008048780080B9200096
:10972000104078000080FB000000D1006100600064
:109730000004E00005003200A0B9200010407800CD
:109740000010A000A1B920008048780080B9200056
:10975000104078000080FB00610060000004E00021
:1097600005003200A0B92000104078000020A000C1
:10977000A1B920008048780080B92000104078000E
:109780000080FB004300DE000000A20061006000DA
:109790000004E0000500320090B72000104078007F
:1097A0000030A00091B720008048780080B72000EA
:1097B000104078008080FB00208220000080400064
:1097C0001040780047FD070010C0B300347002005D
:1097D00000000000FCFE37000040EB003470020087
:1097E00000000000F8FE37000080FA0000000600CC
:1097F0000400FA00969F0200000000000004E00050
:109800002200320032C2BF00684060000004E00065
:10981000040032003100200010CF2000569D0200CD
:109820000000000032C2BF00644060000004E0009D
:10983000040032003100200040CF2000569D02007D
:1098400000000000849F020000000000004F78002C
:1098500032C2BF00624060000004E0000800320035
:10986000F100200070CF2000569D02000000000093
:1098700090118000D1FF2F0001006000901188003E
:109880001E80FB001007980006003700F100200042
:1098900060D02000569D0200000000000000EB0098
:1098A000100798001E0090000080FA0000000600DB
:1098B0000200FA00000F78001E007800709F02007E
:1098C00000000000001020000080FA0000000600E8
:1098D0000000FA0001022000C0DB2000569D0200BB
:1098E0000000000080B7200010407800706E020079
:1098F0000000000000C2B30034700200000000004D
:1099000080B7200010407800E94F500007003A006F
:10991000C0118000126E02000000000000C2B300FF
:1099200034700200000000000C00370080B72000F7
:10993000104078000080FB0080004000A0B02000B4
:109940000080400010007800126E0200000000004D
:1099500000C2B3003470020000000000C0DD20002F
:109960001040780063406000706E0200000000004C
:1099700000C2B3003470020000000000C0DD20000F
:10998000104078000080FB004200DE006140600073
:10999000706E02000000000000C2B30034700200CC
:1099A00000000000C0DD2000104078000080FB00B7
:1099B0004300DE0061406000706E020000000000A5
:1099C00000C2B300347002000000000090B7200015
:1099D000104078000080FB004300DE006140600022
:1099E000706E02000000000000C2B300347002007C
:1099F0000000000031002000F0AD2000569D020064
:109A0000000000000080FA00000006000C00FA00D0
:109A1000661A02000000000090160200000000001C
:109A2000500798005E009000EA0F500005003A00D1
:109A3000661A0200000000009016020000000000FC
:109A4000000F7800661A0200000000009016020065
:109A50000000000040079800661A020000000000A5
:109A6000901602000000000030079800661A0200FD
:109A7000000000009016020000000000200798007F
:109A8000661A0200000000009016020000000000AC
:109A9000100798005E0090000000E000090034000C
:109AA0005E009000EA0F500006003C005E0090004F
:109AB0000040E9008040780080B72000014878002D
:109AC000020037000000EB00500798004E009000A5
:109AD0000000E0000F0034004E009000E40F500042
:109AE0000C003C004E0090000040E900E3406000A4
:109AF000C0DD20001040780063C16000C1CFB3001A
:109B00000140600002407000C1DD20008048780004
:109B1000020037000000EB00500798003E00900064
:109B20000000E000100034003E009000E20F500002
:109B30000D003C003E0090000040E90061416000E3
:109B4000C0DD200090407800614061004201DD00EE
:109B5000B0CFB30080C0600082C07000C0DD2000C4
:109B600001487800020037000000EB005007980021
:109B70002E0090000000E000100034002E00900045
:109B8000E20F50000D003C002E0090000040E90064
:109B900061416000C0DD20009040780061406100BC
:109BA0004301DD0070CFB30080C0600082C0700050
:109BB000C0DD200001487800020037000000EB0003
:109BC000500798001E0090000000E00010003400D4
:109BD0001E009000E20F50000D003C001E0090009F
:109BE0000040EA006141600090B72000904078009A
:109BF000614061004301DD0070CFB30080C06000B0
:109C000082C0700090B72000014878000200370041
:109C10000000EB00500798005E0090000000E0009C
:109C200073003A000000EB0070698800D108200042
:109C300030872000E09D0200000000008001EB0062
:109C4000A20020001100200010002000DC1C0200F7
:109C5000000000000040E9008040780080B720004C
:109C60000148780080B7200010407800E94F50008C
:109C70000B003A00C1012000001B2100E09D020002
:109C8000000000008001EB00F2FF2700110020001F
:109C900020022000DC1C020000000000000F780001
:109CA0004105200050D12000569D02000000000018
:109CB0008001EB0042002000110020001000200075
:109CC000DC1C0200000000000040E900E3406000EE
:109CD000C0DD20001040780063C16000C1CFB30038
:109CE0000140600002407000C1DD20008048780023
:109CF0001102200090D62000569D020000000000B6
:109D00008001EB0022002000110020001000200044
:109D1000DC1C0200000000000040E900614160001E
:109D2000C0DD200090407800614061004201DD000C
:109D3000B0CFB30080C0600082C07000C0DD2000E2
:109D40000148780021032000A0D82000569D020081
:109D5000000000008001EB00220020001100200024
:109D600010002000DC1C0200000000000040E900A0
:109D700061416000C0DD20009040780061406100DA
:109D80004301DD0070CFB30080C0600082C070006E
:109D9000C0DD200001487800F1042000B0932000CD
:109DA000E09D0200000000008001EB002200200086
:109DB0001100200010002000DC1C02000000000048
:109DC0000040EA006141600090B7200090407800B8
:109DD000614061004301DD0070CFB30080C06000CE
:109DE00082C0700090B72000014878000100370061
:109DF000B7FE070080B7200010407800E94F500000
:109E00001C003A00C0DD2000104078000080FB00FC
:109E10004200DE006140600080417800C0DD20002B
:109E2000104078006340600080427800C0DD200070
:109E3000104078000080FB004300DE0061406000BD
:109E40000041780090B72000104078000080FB00AF
:109E50004300DE0061406000804078001E00780012
:109E60000342780085417800C49E02000000000093
:109E700022003700C0DD2000104078000080FB0089
:109E80004200DE006140600000417800C0DD20003B
:109E9000104078006340600080417800C0DD200001
:109EA000104078000080FB004300DE00614060004D
:109EB0008042780090B72000104078000080FB00BE
:109EC0004300DE00614060000043780080B720005E
:109ED000104078000080FB0080004000A0B020000F
:109EE00000804000100078000242780005417800B0
:109EF00086407800C49E020000000000489F0200D7
:109F000000000000C111800040118000808F5000CF
:109F10000400310001022000C01C2100E09D02006D
:109F2000000000000080FA00000006000000FA00B7
:109F3000549F0200000000000080FA0000000600AC
:109F40000400FA00000F78001E0078001007980047
:109F50001E009000E10F50000C0032001E00900027
:109F6000E10F5000040039001E009000E20F500085
:109F70003D0032005900370031052000C0DD2000CF
:109F8000569D02000000000058003700B10020007C
:109F9000F0E22000E09D020000000000D10020005F
:109FA000A0E32000E09D020000000000869E020069
:109FB000000000000000E0004C0032009011800022
:109FC000D1FF2F00010060009011880000003700D1
:109FD00032C2BF00614060000004E00006003200B1
:109FE00023C2BF00624060000004E00002003A00AB
:109FF000B01180002011880022C2BF0061406000C3
:10A000000004E0000600320033C2BF00624060007E
:10A010000004E00002003A0030118000A011880026
:10A0200032C2BF00624060000004E00004003A0059
:10A0300022C2BF00624060000004E000E4FF320082
:10A0400091118000D0FF2F000080600090118800E7
:10A0500011118000D0FF2F000080600010118800D7
:10A06000CA82A900DAFF3700E100200070E4200076
:10A07000E09D020000000000F1002000C01E210051
:10A08000E09D02000000000090118000D1FF2F0031
:10A09000010060009011880032C2BF006140600082
:10A0A0000004E0000600320023C2BF0062406000EE
:10A0B0000004E00002003A00B01180002011880086
:10A0C00022C2BF00614060000004E000F2FF3200E5
:10A0D00030118000000F780004003700410220009A
:10A0E000C0202000E09D0200000000000080FA0077
:10A0F000000006000000FA0091118000D0FF2F0040
:10A100000080600090118800C0DD200010407800C1
:10A110000040A000C1DD20008048780090B72000FA
:10A12000104078000010A00091B72000804878000F
:10A13000C101200050E52000E09D02000000000069
:10A140000080FA00000006000000FA00C0DD2000D8
:10A15000104078000040A100C1DD20008048780058
:10A1600090B72000104078000010A10091B72000A7
:10A17000804878004101200010E72000E09D0200A7
:10A18000000000000080FA00000006000200FA0053
:10A190000000EB00000F780035003700C0DD200024
:10A1A00010407800704060000004E0002C00320095
:10A1B00020A62800046C02000000000061002000BE
:10A1C00060692000569D02000000000032C2BF00FE
:10A1D000684060000004E00004003200310020000C
:10A1E00010CF2000569D02000000000032C2BF00C8
:10A1F000644060000004E0000400320031002000F0
:10A2000040CF2000569D020000000000849F020005
:10A21000000000000080FB00DC970200000000004E
:10A2200032C2BF00624060000004E000080032005B
:10A23000F100200070CF2000569D020000000000B9
:10A2400090118000D1FF2F00010060009011880064
:10A2500020A62800046C0200000000000200370065
:10A26000849F02000000000010002000000F780012
:10A27000969F0200000000000004E000C7FF3A00C3
:10A280001E0078000080FA00000006000000FA00BE
:10A29000B100200010092100E09D02000000000034
:10A2A0000080FA00000006000000FA0030A6280036
:10A2B000D86B0200000000000080FA0000000600D9
:10A2C0000400FA00C0DD2000104078000000A1006A
:10A2D0000010A100C1DD200080487800C0DD200012
:10A2E000104078000020A100C1DD200080487800E7
:10A2F000C0DD2000104078000030A100C1DD20004A
:10A300008048780090B72000104078000030A0000E
:10A3100091B7200080487800F0588000B06E880027
:10A32000C0DD2000104078000040A100C1DD200009
:10A3300080487800C0DD2000104078000080FB00DD
:10A340004200DE006140600080417800C0DD2000F6
:10A35000104078006340600080427800C0DD20003B
:10A36000104078000080FB004300DE006140600088
:10A370000041780090B72000104078000080FB007A
:10A380004300DE006140600080407800B06E8000D5
:10A390000342780085417800C49E0200000000005E
:10A3A000489F020000000000BFFF070000003700C8
:10A3B000969F0200000000000004E0000C00320044
:10A3C000C0DD200010407800704060000004E00014
:10A3D00005003200849F020000000000347002007B
:10A3E0000000000002003700849F0200000000000F
:10A3F00032C2BF00624060000004E000040032008E
:10A4000090118000D1FF2F000100600090118800A2
:10A4100022C2BF00614060000004E000E4FF32009F
:10A420003011800080407800A0DD200001487800D5
:10A43000A0DD2000104078000080FB004400DE001A
:10A440008040780090DD20000148780090DD2000F9
:10A45000104078000080FB00100798001E0090005C
:10A46000E40F5000D00032009E009000E48F5000B6
:10A4700007003C001E0090000000E0000F003200CA
:10A480009E009000E18F50009F0032008A0137004B
:10A490001E009000E60F5000CB0032009E0090009E
:10A4A000E68F5000840135009E00900068805000C7
:10A4B000E10F500080013E00FB003700A0DD2000CE
:10A4C000104078000080FB00000F78001E0078002C
:10A4D000E20F5000190032009E007800E28F500019
:10A4E00007003C001E0078000000E0000E00320073
:10A4F0009E007800E18F50000E0032007E00370091
:10A500001E007800E70F5000260032009E00780001
:10A51000EF8F50005B0032001E007800E30F500008
:10A520001700320074003700549F02000000000042
:10A53000650137005CFF07009DFF370010C0B300C6
:10A54000347002000000000032C2BF0062406000B0
:10A550000004E0000400320090118000D1FF2F00C1
:10A560000100600090118800C0DD200010407800DC
:10A570000040A000C1DD2000804878008CFF37003B
:10A58000C0DD2000104078000040A100C1DD2000A7
:10A590008048780010C0B300347002000000000052
:10A5A00083FF370010C0B3003470020000000000C9
:10A5B000549F02000000000022C2BF006140600002
:10A5C0000004E000FCFF3200301180004800DD0094
:10A5D000B06E880010C0B3003470020000000000AC
:10A5E00022C2BF00614060000004E000FCFF3200B6
:10A5F000B16E80003011800000807000B06E880065
:10A60000C0DD2000104078000080FB004200DE002A
:10A610006140600080417800C0DD2000104078007B
:10A620006340600080427800C0DD20001040780068
:10A630000080FB004300DE006140600000417800C4
:10A6400090B72000104078000080FB004300DE003F
:10A650006140600080407800B06E80000342780066
:10A6600085417800C49E020000000000489F02005F
:10A670000000000010C0B3003470020000000000B1
:10A680004BFF370010C0B300347002000000000020
:10A6900090118000D1FF2F00010060009011880010
:10A6A0000000370032C2BF00614060000004E000DB
:10A6B0000600320023C2BF00624060000004E000D8
:10A6C00002003A00B01180002011880022C2BF00B1
:10A6D000614060000004E000F2FF320033C2BF00BE
:10A6E000624060000004E000EEFF3A00301180009C
:10A6F000A0118800EBFF37000040EB00347002002F
:10A70000000000002AFF3700A0DD20009040780004
:10A71000F0C0B30080C06000A0DD200001487800D8
:10A72000A0DD2000104078008040E800A0DD20007F
:10A730000148780010C0B30034700200000000002F
:10A740008040EB0080DD2000014878000F003700DA
:10A7500022C2BF00614060000004E000FCFF320044
:10A7600030118000709F02000000000010C0B30094
:10A77000347002000000000080DD200010407800EE
:10A780008040E80080DD20000148780080DD200066
:10A7900090407800A0DD20001040780080CF50006D
:10A7A000EBFF390002FF3700A0DD200010407800E9
:10A7B00038A002000000000010C0B3003470020096
:10A7C00000000000FAFE3700A0DD20009040780075
:10A7D000F0C0B30080C06000A0DD20000148780018
:10A7E000A0DD200010407800EA4F50000300360042
:10A7F000A1C0B300A0DD200001487800A0DD20004A
:10A80000104078000080FB0080004000E0B1200094
:10A810000080400010007800B06E8800549F020055
:10A8200000000000C0DD2000104078000080FB0028
:10A830004200DE006140600080417800C0DD200001
:10A84000104078006340600080427800C0DD200046
:10A85000104078000080FB004300DE006140600093
:10A860000041780090B72000104078000080FB0085
:10A870004300DE006140600080407800B06E8000E0
:10A880000342780085417800C49E02000000000069
:10A89000489F02000000000010C0B30034700200A6
:10A8A00000000000C2FE3700C0DD2000104078002C
:10A8B0000000A1000010A100C1DD20008048780048
:10A8C000C0DD2000104078000020A100C1DD200084
:10A8D00080487800C0DD2000104078000030A100E2
:10A8E000C1DD20008048780090B72000104078003B
:10A8F0000030A10091B7200080487800A0DD200042
:10A90000104078000080FB004300DE006100600022
:10A910000004E0000D003200C0DD2000104078008F
:10A92000634060000014A000E3406000C0DD200030
:10A930001040780063C16000C1CFB30001406000E7
:10A9400002407000C1DD200080487800A0DD2000BA
:10A95000104078000080FB004200DE0061006000D3
:10A960000004E0000D003200C0DD2000104078003F
:10A97000634060000004A000E3406000C0DD2000F0
:10A980001040780063C16000C1CFB3000140600097
:10A9900002407000C1DD200080487800A0DD20006A
:10A9A000104078000080FB000000D10061006000D2
:10A9B0000004E00005003200C0DD200010407800F7
:10A9C0000020A000C1DD200080487800A0DD20002C
:10A9D000104078000080FB00610060000004E0008F
:10A9E00005003200C0DD2000104078000030A000DB
:10A9F000C1DD200080487800A0DD200010407800F4
:10AA00000080FB004400DE000000A2006100600046
:10AA10000004E0000500320090B7200010407800EC
:10AA20000030A00091B7200080487800549F0200B9
:10AA300000000000C0DD2000104078000080FB0016
:10AA40004200DE006140600080417800C0DD2000EF
:10AA5000104078006340600080427800C0DD200034
:10AA6000104078000080FB004300DE006140600081
:10AA70000041780090B72000104078000080FB0073
:10AA80004300DE006140600080407800B06E8000CE
:10AA90000342780085417800C49E02000000000057
:10AAA000489F02000000000010C0B3003470020094
:10AAB000000000003EFE37000040EB003470020052
:10AAC000000000003AFE37000080FA000000060097
:10AAD0000000FA00809C0200000000000080FB00E3
:10AAE0000080FA00000006000200FA00000F780063
:10AAF0001E007800E89B020000000000001020000B
:10AB00000080FA00000006000000FA00E69C020047
:10AB1000000000000080FB000080FA00000006003A
:10AB20000000FA0080BA200010407800469C020025
:10AB3000000000000080FA00000006000000FA009B
:10AB400080BA2000104078000080FB000080FA00EE
:10AB5000000006000000FA008040EB0080BA2000F0
:10AB60000148780041022000B0002000E09D020072
:10AB7000000000000080FA00000006000000FA005B
:10AB800011C0B30080BA20000148780041022000C3
:10AB9000B0002000E09D0200000000000080FA00EC
:10ABA000000006000000FA0090B720001040780076
:10ABB0000030A00091B72000804878008040EB0072
:10ABC000A0BB200001487800C922A800CB22A90020
:10ABD000E1022000F0022000E09D020000000000E1
:10ABE0000080FA00000006000400FA00881F7800C8
:10ABF000000F78001E00E000440032002003200017
:10AC00009E0F100041003E001E0FE900A0BB200077
:10AC1000104078000080FB009E0F500005003E00B1
:10AC200091022000D0052000E09D020000000000FD
:10AC300063013700E100200060082000569D0200FB
:10AC4000000000001E0078000040E800706E020066
:10AC50000000000080A42800D86B02000000000063
:10AC60008040EB0040BB2000014878001F00370007
:10AC70001E01780040BB2000104078008080FB005F
:10AC80004310DD0081004000B0BB20000080400088
:10AC9000104078000080FB00DC97020000000000FC
:10ACA00000C2B30034700200000000001E017800F2
:10ACB00040BB2000104078008080FB004310DD0086
:10ACC00081004000B0BB20000080400010407800B0
:10ACD000E89B02000000000040BB2000104078000C
:10ACE0008040E80040BB20000148780040BB2000C5
:10ACF00010407800E74F5000DDFF3600B0A4280078
:10AD0000046C0200000000002D0137001E007800D6
:10AD100010079800500520009E009000808F500082
:10AD200011013200500520009E009000808F5000DD
:10AD300008003E001E0090000000E00012003200FB
:10AD4000300320009E009000808F5000DD00320014
:10AD500017013700C00E20009E009000808F500029
:10AD600063003200000F20009E009000808F500092
:10AD70005F003200C00C20009E009000808F5000C9
:10AD8000020132000A013700D100200040092000F2
:10AD9000E09D02000000000071012000100A200068
:10ADA000E09D020000000000A0BB200010407800E1
:10ADB0000004E00005003A0091022000D0052000C8
:10ADC000E09D020000000000440037008040EB00DE
:10ADD00050BB2000014878003A00370000C2B300A1
:10ADE000347002000000000050BB200010407800CA
:10ADF0000040E800706E020000000000C0A42800BF
:10AE0000D86B0200000000008040EB0040BB200037
:10AE1000014878001600370050BB20001040780031
:10AE20000081FB0040BB2000104078008080FB00C8
:10AE30004310DD0081004000B0BB200000804000D6
:10AE4000104078000080FB00DC970200000000004A
:10AE500000C2B300347002000000000040BB2000BC
:10AE6000104078008040E80040BB20000148780096
:10AE700040BB200010407800E74F5000E6FF36004E
:10AE800061002000800B2000569D020000000000A1
:10AE900050BB2000104078000080FB00C300DD00A4
:10AEA000B0BB20000080400010407800F700070091
:10AEB00050BB2000104078008040E80050BB2000CC
:10AEC00001487800A0BB20009040780050BB2000D3
:10AED0001040780080CF5000C0FF3E00310D2000B0
:10AEE000E00B2000E09D020000000000B4003700ED
:10AEF0001E00780080407800C08320000148780060
:10AF0000C00E20009E0F100005003A003101200005
:10AF100010192000E09D020000000000040037002E
:10AF2000D1002000401A2000E09D02000000000037
:10AF300071012000100A2000E09D020000000000C6
:10AF40008040EB0040BB2000014878000A01070068
:10AF50008040780050BB2000014878008040EB0022
:10AF6000A0BB2000014878004D00370000C2B300AC
:10AF7000347002000000000040BB20001040780048
:10AF80000040E800706E020000000000C0A428002D
:10AF9000D86B0200000000000000EB00905D88000C
:10AFA0000D003700915D8000B0C02000008040009F
:10AFB000104078000080FB00DC97020000000000D9
:10AFC00000C2B3003470020000000000905D8000F9
:10AFD0000000E800905D8800905D8000E70F500061
:10AFE000F0FF360061002000800B2000569D02001B
:10AFF00000000000B0C0200010407800A30007004F
:10B0000040BB200010407800E94F50001B003E007C
:10B010000000EB00905D880010003700A0BB20000E
:10B02000104078008081FB00945D8000915D80007D
:10B03000B0C0200000804000104178004318DD00BF
:10B0400084004000B0BB200000804000024878002F
:10B05000905D80000000E800905D8800905D8000B9
:10B06000E70F5000EDFF3600A0BB20001040780035
:10B070008040E800A0BB20000148780040BB2000D1
:10B08000104078008040E80040BB20000148780074
:10B09000C70007008040780050BB200001487800BE
:10B0A00050BB2000104078000004E000AFFF3A00E1
:10B0B000B1022000101B2000E09D020000000000F3
:10B0C0003F0037004800070011012000C01D20008C
:10B0D000569D02000000000030C3B300E89B020050
:10B0E000000000000000EB00905D880014003700B5
:10B0F000985D8000809C0200000000008040780085
:10B1000090BA20000000440001487800915D800062
:10B1100090BA200000804000104078000080FB00C2
:10B12000DC9702000000000000C2B300347002008F
:10B1300000000000905D80000000E800905D880045
:10B14000905D8000E70F5000E9FF3600B0A42800B2
:10B15000046C02000000000090BA2000104078004B
:10B160004A000700160037001F00070001012000F9
:10B17000D01E2000E09D02000000000050C5B3007A
:10B18000E89B0200000000000D00370016000700D9
:10B19000F1002000D01F2000E09D02000000000010
:10B1A000C0CCB300E89B02000000000004003700A0
:10B1B00041022000C0202000E09D020000000000AD
:10B1C0004F0478000080FA00000006000000FA003A
:10B1D0009100200080082100E09D02000000000096
:10B1E0000080FA00000006000200FA00629B0200E4
:10B1F00000000000004F7800A10020000023200084
:10B20000569D0200000000001E04E00005003A0008
:10B210003100200050BB2000E09D02000000000033
:10B220001800370091002000A0232000569D020046
:10B23000000000001E80FB00610060000004E000D0
:10B24000040032005101200030242000569D0200ED
:10B25000000000001E80FB000000D10061006000C3
:10B260000004E0000400320041012000802520009D
:10B27000569D020000000000B0A42800046C0200EB
:10B28000000000000080FA00000006000400FA0040
:10B29000004F78001E80FB0010079800200220005D
:10B2A0009E009000808F50001E003200200220007F
:10B2B0009E009000808F500007003C001E00900010
:10B2C000E40F50001C0032009E009000F08F5000F0
:10B2D0000A00320022003700800220009E00900009
:10B2E000808F50000A003200D00220009E009000A3
:10B2F000808F50001500320019003700B101200086
:10B30000C0262000E09D0200000000001800370069
:10B31000A101200070282000E09D02000000000034
:10B320001300370051012000102A2000E09D020088
:10B33000000000000E00370081012000602B20007B
:10B34000E09D02000000000009003700010120001C
:10B35000E02C2000E09D0200000000000400370007
:10B36000E1002000E02D2000569D020000000000BA
:10B370000080FA00000006000000FA008040EB00A8
:10B3800030C12000014878008040EB0050C120000F
:10B39000014878008040EB0040C12000014878005F
:10B3A000080007000080FB000080FA000000060093
:10B3B0000000FA00030007000080FB000080FA0094
:10B3C000000006000A00FA0010C0B30070479800A1
:10B3D0000040EB00604798000040EB0050479800A9
:10B3E00010C0B300104798000040EB0040479800A1
:10B3F0008040EB0060C120000148780050C120006F
:10B40000104078000004E0009C003A00629B0200BB
:10B41000000000000004E0000C0032008040EB005F
:10B4200030C12000014878008040EB0050C120006E
:10B43000014878008040EB0040C1200001487800BE
:10B440000000EB0040079800A1003700C0832000F7
:10B4500010407800E89B020000000000E69C02001B
:10B460000000000030479800E69C02000000000049
:10B47000204798003E409000E14F500003003A0002
:10B480002E409000E14F500068003200BE40900016
:10B490002E40900080CF500003003200BE4090004C
:10B4A000014F78002600370030C12000904078001E
:10B4B0007E409000814F50000E0031005E409000B1
:10B4C0008080FB00B0C020000080400090407800E9
:10B4D0001E40900080C060000040EB00004F7800EC
:10B4E0000104E0000C00320010C0B300004F7800EF
:10B4F0000900370030C12000904078000040EB0088
:10B50000004F78007E409000814F500002003A00CA
:10B5100010C0B300004F78001E04E00008003A009D
:10B520007E409000604798006E409000E84F5000C9
:10B5300003003E0040C12000EE409000014878002A
:10B5400010C0B3009E4F10000D003A005E40900006
:10B550000081FB005E4090008080FB00B0C02000B6
:10B5600000804000904078001E40900080C0700035
:10B57000B0C02000000041000148780011003700F1
:10B580005E4090000082FB005E4090008080FB00E7
:10B59000B0C020000080400010407800804178005A
:10B5A0001E419000024078000080EA008180EA009D
:10B5B00000C0610080407800B0C020000000420060
:10B5C000014878001E407800469C02000000000000
:10B5D0007E4090000040E800704798001E409000B8
:10B5E00000404000104798001E4090000004E0001A
:10B5F0000B003A005E4090008080FB00B0C020004D
:10B600000080400010407800920007005E409000EB
:10B610000040E8005047980010C0B3001047980061
:10B620005E409000E74F50008CFF3600FE409000D7
:10B6300000C4B30080CF50001000360060C120006D
:10B64000104078000004E0000C003A0030C12000F7
:10B65000EE4090000148780030C120001040780092
:10B660000004E00003003A0011C0B30050C1200004
:10B670000148780010C0B300404798004E40900049
:10B680000004E00004003200B0C020001040780048
:10B690000004E0000B003A008040EB0030C12000C5
:10B6A000014878008040EB0050C12000014878003C
:10B6B0008040EB0040C12000014878000040EB00D2
:10B6C000404798004E4090000080FB0040079800E3
:10B6D0004E0090000080FA00000006000E00FA0004
:10B6E0000040EB00404798000C0037004E409000AF
:10B6F0000081FB004E4090008080FB00B0C0200025
:10B70000008040009040780065004700017178009B
:10B710004E4090000040E800404798004E409000A6
:10B72000E74F5000F1FF360030C120009040780014
:10B730002147980050C120009040780011479800A0
:10B7400040C12000104F780001C4B30030C1200078
:10B75000014878008040EB0050C12000014878008B
:10B7600018FF07000004E0001A00320010C0B30008
:10B77000304798000040EB00404798001100370028
:10B780004E4090008080FB006500470061417800DA
:10B790004E4090008080FB00B0C020000080400040
:10B7A00010407800804F5100030032000040EB0051
:10B7B00030479800090037004E4090000040E800F4
:10B7C000404798004E409000E74F5000ECFF360095
:10B7D000020037000040EB00304798000040EB00CB
:10B7E000404798000C0037004E4090000081FB005D
:10B7F0004E4090008080FB0065004700E1407800EB
:10B80000B0C0200000004100014878004E40900088
:10B810000040E800404798004E409000E74F50003D
:10B82000F1FF360030C12000AE40900001487800A2
:10B8300050C120009E4090000148780040C1200087
:10B840001E4878003E4090000080FB000080FA0017
:10B85000000006000200FA00004F780060C12000DE
:10B86000104078001E4068008080FB00D0832000DC
:10B87000008040009040780060C1200001487800BE
:10B8800060C12000104078000080FB000080FA00BA
:10B89000000006000000FA00E0A42800D86B0200B7
:10B8A000000000000080FA00000006000400FA001A
:10B8B000C922A800CB22A900C8C2A90090B72000C5
:10B8C000104078000030A00091B720008048780038
:10B8D00090B72000104078000020A10091B7200010
:10B8E00080487800EBFF07000000370022C2BF004D
:10B8F000614060000004E000FCFF32003011800075
:10B900008040780090BB20000148780090BB200068
:10B91000104078000080FB004400DE00804078008A
:10B9200080BB20000148780080BB200010407800D8
:10B930000080FB00100798001E009000E10F5000EF
:10B94000780032009E009000E48F50009D0032008D
:10B950001E0090000000E00001003200A10037004E
:10B9600090BB2000104078000080FB00000F7800A2
:10B970009E007800E28F5000170032001E00780011
:10B98000E20F500007003C009E0078000100E0003C
:10B99000980032001E007800E10F50000C003200C9
:10B9A0005C0037009E007800E48F500013003200E6
:10B9B0001E007800E40F5000560035009E0078000D
:10B9C00068805000E10F500052003E001000370028
:10B9D000B0FF0700C5FF3700629B020000000000B7
:10B9E0008040780060BB20000148780010C0B300A0
:10B9F0003470020000000000BCFF3700809C020091
:10BA0000000000003470020000000000B7FF3700A3
:10BA100010C0B300347002000000000090BB200092
:10BA200010407800E94F500004003A00C1CEB30046
:10BA3000C0832000014878000300370001CFB30025
:10BA4000C0832000014878004BFE0700804078004A
:10BA500060BB200001487800190037008040EB00EF
:10BA600070BB2000014878000D00370070BB20003B
:10BA7000104078008080FB00B0C0200000804000B3
:10BA800010407800347002000000000070BB2000FD
:10BA9000104078008040E80070BB2000014878002A
:10BAA00070BB200010407800E74F5000EFFF3600D9
:10BAB0003FFE07008040780060BB2000014878000E
:10BAC00060BB2000104078000004E000E3FF3A0073
:10BAD0008040EB0070BB2000014878000800370070
:10BAE00000C0EB00347002000000000070BB2000BA
:10BAF000104078008040E80070BB200001487800CA
:10BB000070BB200010407800E74F5000F4FF360073
:10BB100076FF37000040EB003470020000000000A8
:10BB200072FF370090BB200090407800F0C0B30057
:10BB300080C0600090BB20000148780090BB2000CE
:10BB4000104078008040E80090BB20000148780059
:10BB500010C0B30034700200000000008040EB0011
:10BB600070BB2000014878000F00370022C2BF00E0
:10BB7000614060000004E000FCFF320030118000F2
:10BB8000E89B02000000000010C0B3003470020007
:10BB90000000000070BB2000104078008040E800EA
:10BBA00070BB20000148780070BB200090407800F6
:10BBB00090BB20001040780080CF5000EBFF390090
:10BBC0004AFF370090BB20001040780038A00200E8
:10BBD0000000000010C0B30034700200000000003C
:10BBE00042FF37000040EB0034700200000000000C
:10BBF0003EFF37000080FA00000006000000FA0057
:10BC0000E0A62800D86B0200000000000080FA00C7
:10BC1000000006000000FA000040EB009A7F0200DE
:10BC2000000000000040EB009A7F020000000000CE
:10BC30000040EB009A7F0200000000000040EB0093
:10BC40009A7F0200000000000000EB00D67E020098
:10BC5000000000000000EB00D67E020000000000A3
:10BC60000000EB00D67E0200000000000080FA0019
:10BC7000000006000C00FA0090B720001040780089
:10BC80000030A00091B720008048780090B72000D5
:10BC9000104078000020A10091B720008048780073
:10BCA00011C0B30080B720000148780081C0B30004
:10BCB000A0B720000148780021C0B30030DF200089
:10BCC0000148780080C0EB0020C0B300767D020000
:10BCD00000000000C922A900C902A900C8E2A8000A
:10BCE00010C0B3000680020000000000C3FF070080
:10BCF0000000370022C2BF00614060000004E00085
:10BD0000FCFF3200301180008040780070DF20009E
:10BD10000148780070DF2000104078000080FB00B0
:10BD20004400DE008040780060DF20000148780099
:10BD300060DF2000104078000080FB003007980092
:10BD40003E009000E30F500014013200BE0090004E
:10BD5000E38F50000A003C003E019000E10F5100CB
:10BD6000A4003200BE019000E18F5100F8003C00B9
:10BD70003E0090000000E000120032002003370077
:10BD8000BE009000E68F5000C90232003E019000D4
:10BD9000E60F510004003C00BE019000E48F51000A
:10BDA000BB023200160337003E009000E80F50003F
:10BDB000D6023200BE009000EA8F500031013200FE
:10BDC0000F03370070DF2000104078000080FB0078
:10BDD0006101B9004207980053079800D000200085
:10BDE000010020004E019000DE019000800F510004
:10BDF000818F59007B003E004E009000DE009000D5
:10BE000000600100020337000C0037000D0037000E
:10BE100012003700170037001D00370023003700DD
:10BE200043003700470037004B0037005100370010
:10BE3000570037005D003700630037006FFF0700D1
:10BE4000ACFF3700047E02000000000010C0B30009
:10BE50003470020000000000A6FF3700447E02009C
:10BE60000000000010C0B3003470020000000000A9
:10BE7000A0FF37000040EB00068002000000000039
:10BE800010C0B300347002000000000099FF3700BA
:10BE900010C0B300068002000000000010C0B30014
:10BEA000347002000000000092FF370030DF2000F5
:10BEB00010407800E24F500006003A002A7F02004E
:10BEC000000000008040780050DF2000014878002A
:10BED00006003700F00F2000647E02000000000022
:10BEE0008040780050DF20000148780090B72000A3
:10BEF00010407800644060000004E0000700320059
:10BF000050DF200010407800C498020000000000BC
:10BF10008040780050DF20000148780050DF20008A
:10BF200010407800347002000000000071FF3700FC
:10BF3000787F020000000000347002000000000062
:10BF40006CFF37001880020000000000347002000F
:10BF50000000000067FF370010C0B300BC7F020084
:10BF60000000000010C0B3003470020000000000A8
:10BF700060FF37000040EB00F47F0200000000008B
:10BF800010C0B300347002000000000059FF3700F9
:10BF900010C0B300F47F02000000000010C0B30026
:10BFA000347002000000000052FF37000040EB0038
:10BFB000E27F02000000000010C0B30034700200F5
:10BFC000000000004BFF370010C0B300E27F02000A
:10BFD0000000000010C0B300347002000000000038
:10BFE00044FF37000040EB00347002000000000006
:10BFF00040FF370070DF200090407800F0C0B300B1
:10C0000080C0600070DF20000148780070DF2000F1
:10C01000104078008040E80070DF20000148780080
:10C0200010C0B30034700200000000008040EB003C
:10C0300050DF2000014878003E00370022C2BF00D8
:10C04000614060000004E000FCFF3200301180001D
:10C050008040780040DF20000148780090B7200041
:10C0600010407800644060000004E00007003200E7
:10C0700040DF200010407800C4980200000000005B
:10C080008040780040DF20000148780030DF200049
:10C0900010407800E24F500009003A0040DF2000D5
:10C0A000104078000080FB00D67E020000000000F7
:10C0B00010C0B30034700200000000001800370008
:10C0C00040DF2000104078000080FB00647E02000A
:10C0D000000000008040780040DF20000148780028
:10C0E00090B7200010407800644060000004E00039
:10C0F0000700320040DF200010407800C4980200A2
:10C10000000000008040780040DF200001487800F7
:10C1100040DF200010407800347002000000000072
:10C1200050DF2000104078008040E80050DF200001
:10C130000148780050DF20009040780070DF200038
:10C140001040780080CF5000BCFF3900E9FE370076
:10C1500070DF200090407800F0C0B30080C0600025
:10C1600070DF20000148780070DF20001040780068
:10C170008040E80070DF20000148780070DF200078
:10C1800010407800BC7F02000000000010C0B30027
:10C190003470020000000000D6FE370070DF20007F
:10C1A00090407800F0C0B30080C0600070DF2000D5
:10C1B0000148780070DF2000104078008040E800DF
:10C1C00070DF20000148780010C0B3003470020016
:10C1D0000000000022C2BF00614060000004E000D7
:10C1E000FCFF3200301180008040780060DF2000CA
:10C1F000014878008040EB0050DF200001487800C3
:10C200001600370060DF2000104078000004E000D6
:10C2100004003D0010C0B3009A7F0200000000003F
:10C22000030037000040EB009A7F0200000000008E
:10C2300060DF20001040780000404000804078001F
:10C2400060DF20000148780050DF200010407800B7
:10C250008040E80050DF20000148780050DF2000D7
:10C260009040780070DF20001040780080CF5000B0
:10C27000E4FF390010C0B300347002000000000079
:10C280009CFE370070DF2000104078000080FB002B
:10C2900020079800400A2000AE009000808F5000D8
:10C2A00015003200500A20002E019000800F51002E
:10C2B000C5003200000A2000AE019000808F5100BE
:10C2C000010032006E01370022C2BF0061406000F1
:10C2D0000004E000FCFF3200301180008040780054
:10C2E000E0DE20000148780010C0B3003470020086
:10C2F000000000007FFE3700E0DE200010407800E4
:10C300000080FB00100798001E009000E10F500015
:10C31000040032009E009000E28F50003B0032008B
:10C32000A500370022C2BF00614060000004E000A9
:10C33000FCFF320030118000606F8800606F800069
:10C340006300B900606F88000000EB00506F880048
:10C350000C00370022C2BF00614060000004E00012
:10C36000FCFF320071408000506F800080804000F0
:10C370003011800080487800506F80000000E80095
:10C38000506F8800516F8000606F8000808F500078
:10C39000F0FF39000000EB00506F880013003700F9
:10C3A00071408000506F8000008040000080E800F5
:10C3B0001041780071408000506F80000080400084
:10C3C0000000E8009041780071408000506F8000CC
:10C3D0000080400010407800834078008E01070004
:10C3E000506F800063004000506F8800516F8000E4
:10C3F000606F8000808F5000E9FF390010C0B300EB
:10C4000034700200000000003AFE370022C2BF0074
:10C41000614060000004E000FCFF32003011800049
:10C42000606F8800606F80004200DD00606F8800F0
:10C430000000EB00506F88000C00370022C2BF00E4
:10C44000614060000004E000FCFF320071408000A9
:10C45000506F80008080400030118000804878005C
:10C46000506F80000000E800506F8800516F80001E
:10C47000606F8000808F5000F0FF39000000EB00FB
:10C48000506F8800440037000040EB009A7F0200A4
:10C49000000000000040EB009A7F02000000000056
:10C4A0000040EB009A7F0200000000000040EB001B
:10C4B0009A7F02000000000071408000506F8000F1
:10C4C00000804000104078000080FB00D67E020013
:10C4D0000000000071408000506F8000008040002C
:10C4E0000000E800104078000080FB00D67E0200CB
:10C4F0000000000071408000506F8000008040000C
:10C500000080E800104078000080FB00D67E02002A
:10C510000000000071408000506F800000804000EB
:10C520006301400071408000506F80000080400037
:10C5300063004000104078006F40600000497800C0
:10C540008040EB0050DF20000148780006003700F3
:10C55000B0FD070050DF2000104078008040E80068
:10C5600050DF20000148780071408000506F80004B
:10C5700000804000630040009040780050DF2000C1
:10C580001040780080CF5000F1FF3E00506F8000D7
:10C5900064004000506F8800516F8000606F800021
:10C5A000808F5000B8FF390010C0B3003470020013
:10C5B00000000000CFFD37000040EB0034700200A7
:10C5C00000000000CBFD3700E0DE200010407800C6
:10C5D0000080FB00000F78001E017800E10F510081
:10C5E000040032009E017800E28F510045003200C5
:10C5F000C0FD370022C2BF00614060000004E000BF
:10C60000FCFF320030118000606F880022C2BF0042
:10C61000614060000004E000FCFF32003011800047
:10C620008040780060DF2000014878000000EB00C7
:10C63000506F88002E00370060DF200090407800A7
:10C6400040DF2000014878008040EB0050DF2000F0
:10C65000014878001900370040DF200010407800C2
:10C660000080FB00610060000004E0000400320074
:10C6700010C0B3009A7F02000000000003003700E2
:10C680000040EB009A7F02000000000040DF200025
:10C69000104078000080FB000000D100804078004E
:10C6A00040DF20000148780050DF20001040780073
:10C6B0008040E80050DF20000148780050DF200073
:10C6C00010407800E34F5000E3FF36002A7F02005D
:10C6D000000000002A7F0200000000003470020009
:10C6E00000000000506F80000000E800506F8800DC
:10C6F000516F8000606F8000808F5000CEFF390046
:10C700007CFD370022C2BF00614060000004E000F1
:10C71000FCFF320030118000606F880022C2BF0031
:10C72000614060000004E000FCFF32003011800036
:10C7300080407800F0DE20000148780022C2BF006F
:10C74000614060000004E000FCFF32003011800016
:10C750008040780000DF20000148780022C2BF003E
:10C76000614060000004E000FCFF320030118000F6
:10C770008040780010DF2000014878000000EB00C6
:10C78000506F8800390037000040EB009A7F0200AC
:10C79000000000000040EB009A7F02000000000053
:10C7A0000040EB009A7F0200000000000040EB0018
:10C7B0009A7F020000000000F0DE200010407800A8
:10C7C0000080FB00D67E02000000000000DF200099
:10C7D000104078000080FB00D67E020000000000C0
:10C7E00010DF2000104078000080FB00D67E0200A1
:10C7F0000000000007FD070006FD070010C0B300A1
:10C800009A7F0200000000000040EB009A7F0200C7
:10C81000000000000040EB009A7F020000000000D2
:10C820000040EB009A7F0200000000000000EB00D7
:10C83000D67E0200000000002A7F020000000000F7
:10C8400034700200000000002A7F02000000000097
:10C850003470020000000000EEFC0700EDFC070051
:10C86000506F80000000E800506F8800516F80001A
:10C87000606F8000808F5000C3FF39001DFD3700BE
:10C880000040EB00347002000000000019FD37008A
:10C8900070DF20001040780038A002000000000087
:10C8A00010C0B300347002000000000011FD37001A
:10C8B00070DF20009040780030C0B30080C060007E
:10C8C00070DF20000148780070DF20009040780081
:10C8D00080B720000148780080B7200090407800A1
:10C8E00030DF200010407800767D0200000000005C
:10C8F00010C0B300068002000000000010C0B300AA
:10C900003470020000000000FAFC370090B72000ED
:10C91000104078000030A10091B7200080487800D6
:10C9200070DF2000104078000080FB004300DE0034
:10C930000000A200610060000004E0000500320079
:10C9400090B72000104078000030A00091B7200080
:10C950008048780021C0B30030DF20000148780013
:10C9600070DF2000104078000080FB004200DE00F5
:10C97000610060000004E0000300320031C0B30039
:10C9800030DF20000148780090B720001040780088
:10C990000020A10091B720008048780070DF2000BF
:10C9A000104078000080FB000000D10061006000B2
:10C9B0000004E0000500320090B72000104078002D
:10C9C0000020A00091B720008048780080B72000A8
:10C9D0009040780030DF200010407800767D020023
:10C9E0000000000010C0B30006800200000000003C
:10C9F00010C0B3003470020000000000BDFC37001E
:10CA00000040EB003470020000000000B9FC370069
:10CA10000080FA00000006000600FA002047980097
:10CA200031479800424798002E4090000080FB005C
:10CA30004600DE00004F78000040EB0010479800F1
:10CA4000220037001E409000E34F50000C003A00D7
:10CA50001E04E0000A00320010C0B300F47F0200A0
:10CA6000000000001E80FB00629802000000000031
:10CA70000040EB00F47F02000000000010003700CF
:10CA80002E4090000080FB00610060000004E00088
:10CA90000400320010C0B3009A7F020000000000C2
:10CAA000030037000040EB009A7F02000000000006
:10CAB0002E4090000080FB000000D100204798002D
:10CAC0001E4090000040E800104798001E40900073
:10CAD000E34F5000DBFF36003E4090000080FB003B
:10CAE000D67E0200000000004E4090000080FB0057
:10CAF000D67E0200000000000080FA000000060060
:10CB00000200FA00105D80000000E0001200320018
:10CB100000C2B300347002000000000031002000A9
:10CB200010442000569D02000000000000C2B30027
:10CB30003470020000000000005D80000000E00092
:10CB400003003A000040EB009A7F02000000000062
:10CB50000000EB00105D8800005D80000000E00038
:10CB600003003A002A7F020000000000004F780016
:10CB700010002000105D88001E80FB000080FA007D
:10CB8000000006000400FA00000F7800105D80002D
:10CB90000000E0001200320000C2B3003470020056
:10CBA000000000003100200010442000569D0200CB
:10CBB0000000000000C2B30034700200000000005A
:10CBC000005D80000000E00003003A000040EB0040
:10CBD0009A7F0200000000000000EB00105D88005A
:10CBE000005D80000000E00007003A001E007800B1
:10CBF000D67E020000000000787F020000000000E6
:10CC00000080FB00000F780000C2B3003470020007
:10CC1000000000001E00E00007003A003100200084
:10CC200010442000569D020000000000003020004B
:10CC30001007980006003700410020004044200003
:10CC4000569D020000000000001020001007980010
:10CC50001E0090000080FA00000006000000FA00AC
:10CC6000105D80000000E0000F0032004100200055
:10CC700040442000569D020000000000A0A32800B0
:10CC8000046C020000000000005D80000000E00075
:10CC900003003A0010C0B3009A7F020000000000B9
:10CCA0000000EB00105D8800005D80000000E000E7
:10CCB0000F003A00047E0200000000000000E000C7
:10CCC0000B00320091002000A0232000569D02009E
:10CCD000000000005101200030242000569D020079
:10CCE00000000000A0A32800046C02000000000067
:10CCF000D100200080442000E09D020000000000E0
:10CD00000080FA00000006000000FA00105D8000BC
:10CD10000000E0000F0032004100200040442000ED
:10CD2000569D020000000000A0A32800046C020031
:10CD300000000000005D80000000E00003003A00F9
:10CD400010C0B3009A7F0200000000000000EB005A
:10CD5000105D8800005D80000000E00002003A00E5
:10CD6000447E020000000000C10020005045200069
:10CD7000E09D0200000000000080FA0000000600B4
:10CD80000000FA000101200020522000569D020000
:10CD9000000000000040EB00706E02000000000088
:10CDA00000C2B300347002000000000080B7200011
:10CDB00010407800706E02000000000000C2B30056
:10CDC0003470020000000000B0A32800046C0200D0
:10CDD000000000000080FA00000006000400FA00D5
:10CDE0000000EB00100798000000EB00005D8800D9
:10CDF000661A020000000000901602000000000009
:10CE0000000F78001E00E000090034004000200000
:10CE10009E0F100006003C001E0078000040E90054
:10CE20008040780080B72000014878000200370079
:10CE30000000EB00000F78001E00E0002D003A001B
:10CE40000000EB00706988000000EB00005D8800C6
:10CE5000005D80000000E0000F003A00B1032000F8
:10CE600060482000E09D0200000000008001EB000F
:10CE7000420020001100200010002000DC1C0200F5
:10CE8000000000000040E9008040780080B72000EA
:10CE90000148780022003700C140800030002300A4
:10CEA000808F500004003E0051032000104C2000F1
:10CEB000569D020000000000C1022000604F2000CB
:10CEC000569D0200000000008001EB0032002000AF
:10CED0001100200010002000DC1C020000000000F7
:10CEE0000040E9008040780080B7200001487800C9
:10CEF0000B003700C140800030002300808F5000BD
:10CF000004003E0051032000104C2000569D0200FA
:10CF1000000000009AFF07000000EB00105D880091
:10CF200090B72000104078000030A00091B720009A
:10CF300080487800005D80000000E00009003A00B1
:10CF4000C922A800C902A800CB02A900CB22A900CF
:10CF500080B720009040780020C0B300767D0200AA
:10CF6000000000000080FA00000006000000FA0047
:10CF70000000EB00105D8800005D8000E10F5000B4
:10CF800001003A0007E2A9000080FA000000060054
:10CF90000600FA00100798001E0090002007980075
:10CFA0002E009000E10F50000C0032002E00900087
:10CFB000E10F5000040039002E009000E20F5000F5
:10CFC0006500320073003700510320002053200019
:10CFD000569D020000000000720037008040EB0008
:10CFE000003020002480020000000000E102200048
:10CFF00070562000E09D020000000000CBC2BF0080
:10D00000614060000004E00004003200CBC2BF00B9
:10D01000624060000004E0000C003A009100200033
:10D02000A0232000569D02000000000051012000B6
:10D0300030242000569D020000000000A0A328001C
:10D04000046C020000000000560037000000EB00F6
:10D05000000F780039003700005D80000000E0001C
:10D0600009003A00047E0200000000001E00780063
:10D07000D67E020000000000787F02000000000061
:10D080000080FB00100798001E0090000000E000E8
:10D0900024003A001E007800DC9702000000000027
:10D0A00080C2B30034700200000000001E0078004F
:10D0B0000080D100DC970200000000001E00780014
:10D0C0000000A200610060000004E00004003200E3
:10D0D000D0A32800D86B0200000000000B0037002E
:10D0E000005D80000000E00005003A002A7F020099
:10D0F0000000000010C0B3009A7F02000000000092
:10D1000000A42800D86B020000000000B0A3280093
:10D11000D86B02000000000000C2B30034700200AF
:10D1200000000000005D80000000E00002003A0006
:10D13000447E0200000000001E0FE800F00F2000F7
:10D140009E0F1000C4FF3400A0A32800046C02004E
:10D150000000000013003700005D8000E10F500068
:10D1600001003A0007E2A900710020005059200098
:10D17000E09D020000000000F1002000C01E210020
:10D18000E09D02000000000010C0B3000E00070088
:10D190000400370041022000C0202000E09D020072
:10D1A000000000000080FA00000006000000FA0005
:10D1B000B1002000C0092100E09D02000000000035
:10D1C0000080FA00000006000A00FA00004F9800F4
:10D1D0000040EB00204798000040EB00104798000B
:10D1E0000040EB00004F7800DC70020000000000FF
:10D1F000C922A800C902A800CB02A900CB22A9001D
:10D2000062A0A80062C0A8008660A900CBC2BF00CF
:10D210000080FB000000D100614060006047980082
:10D220006E40900050479800CBC2BF006140600044
:10D23000604798006E40900030479800000037002B
:10D2400086C0BF00684060000004E00012003A00A1
:10D2500023C2BF00624060000004E0000E003A00FC
:10D260001A7102000000000022C2BF00614060008D
:10D270000004E000F2FF320030118000004F78001F
:10D2800062A0A90062C0A9000E4890000004E0005E
:10D2900061003A00630037008660A900CBC2BF007E
:10D2A0000080FB000000D1006140600060479800F2
:10D2B000CBC2BF0061406000404798002E40900004
:10D2C0000004E0002E0032003E4090000004E00028
:10D2D0002B003A004E4090000004E000280032008D
:10D2E0001E409000E74F50000B003E001E407800AB
:10D2F00000404000004F78006E4090000004E000C5
:10D30000010032001E04A0001E4090000040E80012
:10D31000104798003B0037000E4890000004E000E2
:10D32000040032001E80FB00FC6E020000000000C2
:10D3300006003700C0C5B300EA700200000000001C
:10D340001E407800EA700200000000006E4090006D
:10D350000004E00004003200D0C2B300EA70020012
:10D360000000000003003700B0C2B300EA70020002
:10D37000000000000040EB0010479800210037003B
:10D380003E4090000004E0001E0032004E4090003D
:10D390000004E0001B0032005E4090000004E0004A
:10D3A0000B0032006E4090000004E00008003A00DC
:10D3B00010C0B300204798000040EB0010479800D1
:10D3C000B0C5B300EA700200000000000D00370095
:10D3D0005E4090000004E0000A003A006E409000B9
:10D3E0000004E000070032000040EB0020479800F6
:10D3F0000040EB0010479800D0C5B300EA7002006F
:10D40000000000006E409000504798004E40900091
:10D41000304798008AFF3700A0A32800046C020060
:10D42000000000000080FA00000006000000FA0082
:10D4300030A42800D86B0200000000000080FA0031
:10D44000000006000400FA00C922A800C902A800D2
:10D45000CB02A900CB22A900C8C2A90090B7200026
:10D46000104078000030A00091B72000804878007C
:10D4700090B72000104078000020A10091B7200054
:10D480008048780080C0EB0020C0B300767D0200A9
:10D4900000000000E5FF07000000370022C2BF00C7
:10D4A000614060000004E000FCFF320030118000A9
:10D4B00080407800E0B9200001487800E0B9200001
:10D4C000104078000080FB004400DE0080407800BF
:10D4D000D0B9200001487800D0B920001040780071
:10D4E0000080FB00100798001E009000E10F500024
:10D4F0005E0032001E009000E10F500004003C006E
:10D500001E0090000000E000080032009700370085
:10D510001E009000E40F50008C0032001E009000AE
:10D52000E60F50007A00320090003700E0B920008A
:10D53000104078000080FB00000F78001E0078008B
:10D54000E30F5000260032001E007800E30F500069
:10D550000A003C001E007800E10F50001800320065
:10D560001E007800E10F500017003C001E007800FC
:10D570000000E00081003200380037001E00780013
:10D58000E60F5000210032001E007800E60F500028
:10D5900004003C001E007800E40F5000160032002A
:10D5A0002E0037001E007800E70F50001E003200EA
:10D5B0001E007800EF0F50002200320027003700D5
:10D5C0009AFF0700B5FF3700047E0200000000004C
:10D5D00010C0B3003470020000000000AFFF37003D
:10D5E000447E02000000000010C0B300347002004E
:10D5F00000000000A9FF37002A7F020000000000A1
:10D600003470020000000000A4FF37000040EB006F
:10D610009A7F02000000000010C0B30034700200C6
:10D62000000000009DFF370010C0B3009A7F020089
:10D630000000000010C0B3003470020000000000C1
:10D6400096FF37000040EB00DFFE070010C0B3007C
:10D65000347002000000000090FF37000040EB0033
:10D6600034700200000000008CFF3700E0B9200099
:10D6700090407800F0C0B30080C06000E0B92000A6
:10D6800001487800E0B92000104078008040E800B0
:10D69000E0B920000148780010C0B30034700200E7
:10D6A000000000008040EB00C0B920000148780075
:10D6B0001000370022C2BF00614060000004E0009B
:10D6C000FCFF320030118000D67E02000000000016
:10D6D000787F0200000000003470020000000000AB
:10D6E000C0B92000104078008040E800C0B9200098
:10D6F00001487800C0B9200090407800E0B92000CF
:10D700001040780080CF5000EAFF390063FF3700F7
:10D71000E0B920009040780030C0B30080C06000C5
:10D72000E0B9200001487800E0B92000904078007E
:10D7300020C0B300767D02000000000010C0B300DE
:10D74000347002000000000054FF3700E0B92000F0
:10D750001040780038A002000000000010C0B300A4
:10D7600034700200000000004CFF37000040EB0066
:10D77000347002000000000048FF37000080FA000B
:10D78000000006000200FA00000F78001E00E00012
:10D790000300320010C3B300330207000200370059
:10D7A00000C3B300300207000080FA00000006004A
:10D7B0000600FA0010079800020037001E407800AB
:10D7C000290207001E009000104F78001E407800CC
:10D7D000404798004E4090000004E00002003200F4
:10D7E00010C0B300404798004E4090009E0090004B
:10D7F0008100E800110798000004E000EFFF3A0004
:10D800000080FA00000006000600FA0010079800E9
:10D81000020037001E407800130207001E0090002F
:10D82000104F78001E407800404798004E4090000E
:10D830000004E0000200320010C0B300404798002E
:10D840004E4090009E0090008100E8001107980073
:10D850000004E000EFFF3A00D0C0B300020207006E
:10D86000A0C0B300000207000080FA00000006001C
:10D870000400FA002047980000C8B300004F780069
:10D8800040A02800CAFF07000040EB0010479800A6
:10D890000F0037002E4090001E4060000004E000A2
:10D8A0000300320010C3B300EF010700020037008D
:10D8B00000C3B300EC0107001E80FB000000D10094
:10D8C000004F78001E4090000040E800104798008C
:10D8D0001E409000E74F5000EEFF36000080FA0037
:10D8E000000006000E00FA0050079800610798003B
:10D8F0000040EB00004F780000102E00515F200028
:10D9000030079800410798000040EB00104798004E
:10D91000320037003E019000CE0190005E00900082
:10D92000EE0090003406020000000000100798008E
:10D93000210798001E04E00005003A001E00900038
:10D94000AE009000E00F5000E08F58001800320049
:10D950001E0090000043B000C30107009E0090002D
:10D960003E009000000AB8009E0090004E0090001B
:10D970000088B9000501780000014100BE00900058
:10D980002E0090000088B90000014100820278005A
:10D990005E009000EE00900004005000858058006A
:10D9A000500798006107980010C0B300004F78003E
:10D9B0003E009000CE009000A20020000300200056
:10D9C000340602000000000030079800410798006C
:10D9D0001E4090000040E800104798001E40900054
:10D9E000E74F5000CBFF36005E0090000043B000D0
:10D9F0009D0107000080FA00000006000C00FA00FC
:10DA000040079800510798000000EB0010079800AD
:10DA10000000EB00000F78006000B80020079800BD
:10DA2000310798004E019000DE019000F0232400A1
:10DA3000F1002000800F5100818F59002100360035
:10DA40004E009000DE00900002242400F30020002D
:10DA500034060200000000002007980031079800FB
:10DA60002E0090006F000700C0C2B3007E010700C7
:10DA70004E009000DE00900002242400F3002000FD
:10DA8000540602000000000040079800510798006B
:10DA90004E019000DE019000703E20000100200049
:10DAA000800F5100818F590002003E0070A02800B5
:10DAB0003FFF070010002000100798001000200012
:10DAC000000F78004E019000DE019000703E2000B3
:10DAD00001002000800F5100818F59003200360074
:10DAE0004E009000DE009000823E200003002000E7
:10DAF000340602000000000020079800310798005B
:10DB00002E019000BE019000400620000100200080
:10DB1000800F5100818F5900030036002E009000C5
:10DB200040000700140037001E0090000000E000D5
:10DB30000F0032002E019000BE019000A0002000D6
:10DB400001002000800F5100818F59000300360032
:10DB500000C3B3004401070002003700C0A0280042
:10DB600013FF07002E0090002E0007000200370070
:10DB70002E0090002B000700C0C2B3003A0107003E
:10DB80004E009000DE009000823E20000300200046
:10DB9000540602000000000040079800510798005A
:10DBA00010002000000F78004E019000DE01900070
:10DBB0004006200001002000800F5100818F590095
:10DBC000030036004E0090001600070013003700D7
:10DBD0001E00E0000F0032004E019000DE019000B8
:10DBE000A000200001002000800F5100818F59000B
:10DBF0000300360000C3B3001B010700020037001A
:10DC0000C0A02800EAFE07004E00900005000700B3
:10DC1000020037004E009000020007000080FA006A
:10DC2000000006000800FA00300798000040EB00F2
:10DC3000004F780000712200200798000040EB00A0
:10DC4000104798001E0037003E0090002E01900003
:10DC5000110009000280D800100798001E04E0009F
:10DC600003003A001E0090000000E0000C003200AB
:10DC70001E0090000043B000FB0007009E009000D3
:10DC80002E0090000088B900800078003E009000CF
:10DC9000010050003007980010C0B300004F78001A
:10DCA0002E009000A2002000110009000280D80080
:10DCB000200798001E4090000040E80010479800A0
:10DCC0001E409000E34F5000DFFF36003E00900002
:10DCD0000043B000E40007000080FA0000000600E6
:10DCE0000600FA00404798000040EB00004F780023
:10DCF00040C6B300304798000040EB002047980032
:10DD0000200037004E4090008080FB003E40900095
:10DD10000081FB00110009008280D80010479800A4
:10DD20001E04E00003003A001E4090000004E000E2
:10DD30000B0032001E4090000043B000CA000700F4
:10DD40004E4190009E4090003E4090000088B900F7
:10DD5000004051004047980010C0B300004F7800C9
:10DD60003E4090000080FB00A2002000110009004E
:10DD70000280D800304798002E4090000040E80014
:10DD8000204798002E409000E14F5000DDFF360004
:10DD90004E4090000043B000B30007000080FA003E
:10DDA000000006000400FA0010079800F0A1280007
:10DDB0007FFE07001E0090004400DE006F0F600031
:10DDC0009E007800F0A028000080400010407800FD
:10DDD000A50007001E0090006F0F60009E007800F5
:10DDE000F0A0280000804000104078009E0007004E
:10DDF0000080FA00000006000400FA0010079800F6
:10DE000000C3B300F300070080C7B300F1000700B0
:10DE10001E0090004400DE006F0F60009E0078003E
:10DE2000F0A028000080400010407800E9000700C2
:10DE30001E0090006F0F60009E007800F0A0280088
:10DE40000080400010407800E20007000080FA00E7
:10DE5000000006000400FA0010079800F0A1280056
:10DE600053FE07001E0090004C00DE006F0F6000A4
:10DE70009E007800F0A0280000804000104078004C
:10DE8000790007001E0090004800DE006F0F600060
:10DE90009E007800F0A0280000804000104078002C
:10DEA000710007001E0090004400DE006F0F60004C
:10DEB0009E007800F0A0280000804000104078000C
:10DEC000690007001E0090006F0F60009E00780040
:10DED000F0A0280000804000104078006200070099
:10DEE0000080FA00000006000800FA0030079800E1
:10DEF0003E009000CF80DE00F8030200000000002A
:10DF0000926C2200B331240056040200000000008D
:10DF100010079800210798001E009000AE009000A6
:10DF20005A06020000000000004F78001E407800F2
:10DF30006BFF0700E0C2B3004B0007001E0090001B
:10DF4000AE0090005A06020000000000CF80DE0004
:10DF5000F8030200000000000001BE001E00900057
:10DF6000AE009000DA0402000000000010079800E4
:10DF70002107980002002000031224001E009000D8
:10DF8000AE00900096050200000000001007980007
:10DF9000210798001E009000AE0090005A06020073
:10DFA00000000000004F78001E4078004CFF070082
:10DFB0001E009000AE0090005A0602000000000013
:10DFC000CF80DE00F8030200000000000001BE0068
:10DFD0001E009000AE009000DA0402000000000075
:10DFE0001007980021079800020020000312240067
:10DFF0001E009000AE009000960502000000000098
:10E0000010079800210798001E009000AE009000B5
:10E010005A06020000000000004F78001E40780001
:10E020002FFF07000080FA00000006000000FA0041
:10E0300022C2BF00614060000080FB000080FA0047
:10E04000000006000000FA0022C2BF00614060002C
:10E050000004E000FCFF3200301180000080FB0073
:10E060000080FA00000006000200FA00004F78006D
:10E07000D040800001102000010060000000E0009E
:10E0800006003A0023C2BF00624060000004E000C6
:10E09000FCFF3A001E00FB00201188000080FA00FF
:10E0A000000006000200FA00004F78001E80FB000E
:10E0B000401188000080FA00000006000000FA000D
:10E0C00095C0BF00704060000004E00010003A00FE
:10E0D0005140800040408000808F50000C00320092
:10E0E00023C2BF00624060000004E000FCFF3A0071
:10E0F0008580A9009580A8003140800040408000C4
:10E1000000804000104078000080FB002011880053
:10E110000080FA0000000600809FBE000000FA00A8
:10E12000014080002040800080804000301180004D
:10E1300080487800204080000000E80020408800EF
:10E140002140800010408000808F500001003A0084
:10E150009560A9008560A9000080FA004F00BE000C
:10E1600000400600809FBE000000FA004040800092
:10E170000000E8004040880041408000504080009E
:10E18000808F500002003A009580A90006003700F9
:10E190003140800040408000008040001040780006
:10E1A0000080FB00201188008580A9000080FA0013
:10E1B0004F00BE00004006000000FA000000EB0027
:10E1C000A06E880010002000906E88000080FA0089
:10E1D000000006000200FA00004F7800916E8000F7
:10E1E000A06E8000808F500002003A00CA82A90011
:10E1F0000E00370071408000906E800080804000EB
:10E200001E40780080487800906E80000000E80092
:10E21000906E8800916E800000002100808F500079
:10E2200002003A000000EB00906E88000080FA00C7
:10E23000000006000200FA00A06E8000000FE80057
:10E24000000021009E0F100002003A000000EB00C9
:10E25000000F7800906E80009E0F10000C003200BE
:10E2600023C2BF00624060000004E00008003A00E2
:10E270001E007800A06E880071408000A06E8000B3
:10E2800000804000104078000080FB0020118800D2
:10E290000080FA00000006000400FA00000F780079
:10E2A000110798001E007800900188001E00900061
:10E2B0001080BA00C800DD001E0090001000BA00F7
:10E2C000008070000080FA00000006000000FA00E4
:10E2D00080A62800D86B0200000000000080FA0031
:10E2E000000006000200FA00CA82A800E000070051
:10E2F000F6FF070000003700D400070080407800D8
:10E3000080DE20000148780080DE20001040780088
:10E310000004E000C700350080DE200010407800D7
:10E320000004E00002003A00E8FF0700F2FF3700B7
:10E3300080DE200010407800E14F500006003A00D7
:10E34000CB000700A249020000000000C80007003F
:10E35000DEFF0700E8FF370080DE20001040780075
:10E36000E24F500006003A00C1000700226A020096
:10E3700000000000BE000700D4FF0700DEFF3700EA
:10E3800080DE200010407800E34F500006003A0085
:10E39000B70007006051020000000000B400070051
:10E3A000CAFF0700D4FF370080DE2000104078004D
:10E3B000E44F500006003A00AD000700565C020032
:10E3C00000000000AA000700C0FF0700CAFF3700D6
:10E3D00080DE200010407800E54F500006003A0033
:10E3E000A30007003A5E020000000000A000070042
:10E3F000B6FF0700C0FF370080DE20001040780025
:10E40000E64F500006003A0099000700EC90020029
:10E410000000000096000700ACFF0700B6FF3700C1
:10E4200080DE200010407800E74F500004003A00E2
:10E430008F0007008E000700A4FF0700AEFF370023
:10E4400080DE200010407800EF4F50000A003A00B4
:10E4500010C0B3003470020000000000CA82A9009E
:10E4600023C2BF00614060000004E000FCFF3200F6
:10E470000000FE00A0FF370080DE20001040780082
:10E48000F24F500035003A000000EB008008880091
:10E490000000EB00F00888000000EB00E00C8800B2
:10E4A000A16C20009140780000CEB30000C0600055
:10E4B0006041B300CAE6B700640007000080FB00BB
:10E4C000000F78001E0078000000D100610060009D
:10E4D0000004E0000100320010A1A8009E007800B6
:10E4E000618060000004E000010032001081A8009B
:10E4F000560007000080FB004800DD00000F780098
:10E50000520007000080FB001E0F70001E00780004
:10E51000D00C88009E007800C10C880060002000AC
:10E52000E00C8800490007000080FB004800DD0087
:10E53000000F7800450007000080FB001E0F7000F0
:10E540001E0078006008880011E1A80010C0B30028
:10E55000347002000000000067FF370080DE2000FA
:10E5600010407800F34F50000D003A000000EB001F
:10E57000800888000000EB00E00C8800A16C2000FF
:10E580009140780000CEB30000C06000CAE6B7003A
:10E5900010C0B300347002000000000056FF3700C6
:10E5A00080DE200010407800F44F50000E003A004A
:10E5B00021E3A800C0C0B3002497020000000000BF
:10E5C000000F780021E3A9001E0078004800DE005B
:10E5D00034700200000000001E0078003470020059
:10E5E0000000000044FF370080DE2000104078006B
:10E5F0000080FB004500DE000080FB000000D10031
:10E60000610060000004E0000600320080DE2000AF
:10E61000104078001F000700347002000000000066
:10E6200035FF37000040EB003470020000000000AE
:10E6300031FF370080DE200010407800A500070081
:10E6400034700200000000002BFF37000000FA00C9
:10E6500022C2BF00614060000004E000FCFF320005
:10E66000301180000080FB000080FA0000000600EE
:10E670000000FA0000C0EB00060007000040EB00BD
:10E6800094000700C962A900CB62A9000080FA00CB
:10E69000000006000400FA00204798000040EB004C
:10E6A000004F78002E4090000080FB004400DE0008
:10E6B000610060000004E0000200320010C0B300FE
:10E6C000004F78009E40780061C0600061406000AB
:10E6D0004201DD00912C200091407800B0CFB300C2
:10E6E00000C0600002407000C9E2B7000040EB00CB
:10E6F000004F78002E4090000080FB004300DE00B9
:10E70000610060000004E0000200320010C0B300AD
:10E71000004F78009E40780061C06000614060005A
:10E7200000414000912C200091407800D0CFB300F0
:10E7300000C0600002407000C9E2B7000040EB007A
:10E74000004F78002E4090000080FB004200DE0069
:10E75000610060000004E0000200320010C0B3005D
:10E76000004F78009E40780061C060006141600009
:10E77000912C200091407800E0CFB30000C06000F1
:10E7800002407000C9E2B7000040EB00004F780083
:10E790002E4090000080FB000000D100610060006E
:10E7A0000004E0000200320010C0B300004F780007
:10E7B0009E40780061C06000C700DD00C8C2BF0095
:10E7C0000074A10001407000C8E2B7000040EB00F7
:10E7D000004F78002E4090000080FB006100600038
:10E7E0000004E0000200320010C0B300004F7800C7
:10E7F0009E40780061C06000614060004601DD001D
:10E80000812C200091407800F0CBB30000C0600064
:10E8100002407000C8E2B700500020008E9802004D
:10E8200000000000AE40900000CEB30000C06000C9
:10E8300020479800CBC2BF00644060000004E000A5
:10E84000030032002E4090000044A00020479800B2
:10E85000CBC2BF00624060000004E0000300320051
:10E860002E4090000034A00020479800CBC2BF008B
:10E87000614060000004E000030032002E40900080
:10E880000024A00020479800CAC2BF0001C8B300FE
:10E89000014060000004E000030032002E409000C0
:10E8A0000014A00020479800CAC2BF000044B20074
:10E8B0000004E000030032002E4090000004A0009D
:10E8C000204798002E4090000080FB000080FA0056
:10E8D000000006000400FA00204798002E40900037
:10E8E0000080FB004600DE00610060000004E000E4
:10E8F00005003200C082A900C282A800C8A2A900F7
:10E90000CAA2A80004003700C082A900C282A900E0
:10E91000C8A2A900CAA2A9000040EB00004F7800DD
:10E920002E4090000080FB004400DE00610060008B
:10E930000004E0000200320010C0B300004F780075
:10E940009E40780061C06000614060004201DD00CF
:10E95000B12C200091407800B0CFB30000C060001F
:10E9600002407000CBE2B7000040EB00004F78009F
:10E970002E4090000080FB004300DE00610060003C
:10E980000004E0000200320010C0B300004F780025
:10E990009E40780061C0600061406000004140001E
:10E9A000B12C200091407800D0CFB30000C06000AF
:10E9B00002407000CBE2B7000040EB00004F78004F
:10E9C0002E4090000080FB004200DE0061006000ED
:10E9D0000004E0000200320010C0B300004F7800D5
:10E9E0009E40780061C0600061416000B12C200051
:10E9F00091407800E0CFB30000C06000024070009A
:10EA0000CBE2B7000040EB00004F78002E409000B2
:10EA10000080FB000000D100610060000004E00005
:10EA20000200320010C0B300004F78009E40780012
:10EA300061C06000C700DD00CAC2BF000074A10051
:10EA400001407000CAE2B7000040EB00004F7800C0
:10EA50002E4090000080FB00610060000004E00098
:10EA60000200320010C0B300004F78009E407800D2
:10EA700061C06000614060004601DD00A12C200003
:10EA800091407800F0CBB30000C0600002407000FD
:10EA9000CAE2B700500020008E980200000000007B
:10EAA000AE40900000CEB30000C060002047980048
:10EAB000CBC2BF00644060000004E00003003200ED
:10EAC0002E4090000044A00020479800CBC2BF0019
:10EAD000624060000004E000030032002E4090001D
:10EAE0000034A00020479800CBC2BF006140600006
:10EAF0000004E000030032002E4090000024A0003B
:10EB000020479800CAC2BF0001C8B300014060009E
:10EB10000004E000030032002E4090000014A0002A
:10EB200020479800CAC2BF000044B2000004E000C1
:10EB3000030032002E4090000004A00020479800FF
:10EB40002E4090000080FB000080FA0000000600CC
:10EB50000000FA0090B72000104078000030A000BC
:10EB600091B7200080487800960007000080FA00E6
:10EB7000000006000000FA003C01070053000700F7
:10EB800090272100104078000080FB000080FA00F0
:10EB9000000006000400FA00100798001E00900014
:10EBA00071010700004F78001E04E00005003A00E4
:10EBB0003100200010442000569D0200000000009B
:10EBC0000C00370010C0B3009E4F100005003A0043
:10EBD0004100200040442000569D0200000000003B
:10EBE000040037008100200000122100569D020021
:10EBF00000000000001020000080FA000000060065
:10EC00000400FA00000F78001E007800100798003A
:10EC10001E0090000000E000040032001E00900082
:10EC2000E10F500006003200220037006102200090
:10EC300080122100E09D020000000000210037004A
:10EC4000D1002000E0142100E09D0200000000003F
:10EC5000F1002000C01E2100E09D02000000000025
:10EC6000020107000004E00008003A00902721009C
:10EC7000104078000080FB00DC97020000000000DC
:10EC800000C2B300347002000000000022C2BF00C6
:10EC9000614060000004E000F1FF320030118000AC
:10ECA000000F7800A0A82800046C020000000000FB
:10ECB0000400370041022000C0202000E09D020037
:10ECC000000000000080FA00000006000400FA00C6
:10ECD000004F78001E80FB00100798009E009000F7
:10ECE000E28F50001A0032001E009000E20F500028
:10ECF00007003C009E0090000100E0002F00320061
:10ED00001E009000E10F50000C0032002700370079
:10ED10009E009000E48F5000170032001E0090000B
:10ED2000E40F50000F003500F00F20009E0090000F
:10ED3000808F5000180032001C00370001012000B5
:10ED4000B0152100E09D0200000000001B0037000C
:10ED5000E1002000B0162100E09D0200000000004C
:10ED600016003700F100200090172100E09D0200FE
:10ED7000000000001100370000C2B3003470020030
:10ED8000000000008100200000122100569D0200BA
:10ED90000000000009003700510020008018210009
:10EDA000E09D02000000000004003700E1002000A8
:10EDB000D0182100E09D0200000000000080FA0051
:10EDC000000006000000FA00C922A800C902A9003C
:10EDD000CB02A900CB22A9000080FA0000000600A7
:10EDE0000400FA000040EB00410107000004E000CD
:10EDF0000300320020002000100798000E003700AA
:10EE0000CBC2BF000080FB000000D1006140600069
:10EE1000004F780010C0B300350107000004E00087
:10EE20000300320020002000100798000200370085
:10EE30001E80FB00100798001E0090000080FA0062
:10EE4000000006000600FA000040EB002047980092
:10EE50000040EB0010479800CBC2BF000080FB00D1
:10EE60000000D100E14060008027210010407800C0
:10EE700061C16000E1CFB30001406000024070005A
:10EE800081272100804878008027210010407800E9
:10EE9000614060000004E000030032001000200028
:10EEA000200798006E00370010C0B3001001070063
:10EEB0000004E00003003200410020002107980018
:10EEC000670037000040EB0030479800190037001A
:10EED0001E4090000080FB000000D1001047980009
:10EEE000BFFF0700004F780020C0B3009E4F100006
:10EEF00003003A0041002000210798005800370025
:10EF000010C0B3009E4F100007003A009E409000D2
:10EF100000C8B30000C04000104798002E40900089
:10EF20000004A200204798003E4090000040E80006
:10EF3000304798003E409000E74F5000E4FF360015
:10EF4000902721009E40900001487800A4FF070010
:10EF5000004F780020C0B3009E4F100003003A001D
:10EF600041002000210798003D0037001E40780036
:10EF7000E1406000A02721001040780061C16000DE
:10EF8000E1CFB3000140600002407000A1272100E2
:10EF900080487800A0272100104078006140600080
:10EFA0008080FB002E4090000080FB00808F50008E
:10EFB00008003A00A0272100104078000020A0009F
:10EFC000A127210080487800210020002107980017
:10EFD00023003700A0272100104078000020A10066
:10EFE000A1272100804878007DFF0700004F7800AE
:10EFF00020C0B3009E4F100003003A0041002000E3
:10F0000021079800160037001E407800614160001B
:10F01000A02721009040780061406100004140003D
:10F02000D0CFB30080C0600082C07000A027210054
:10F0300001487800C902A900A027210010407800EB
:10F04000624060000004E00003003A00310020004C
:10F0500021079800020037000000EB00200798000D
:10F060002E0090000080FA00000006000200FA0066
:10F0700000C0EB00004F7800C922A800C902A80018
:10F080000040EB001047980011003700CBC2BF00D2
:10F09000614060000004E00007003A0069FF0700DB
:10F0A000004F78001E04E0000C00320040C0B300A6
:10F0B0009E4F100009003200500020008E98020080
:10F0C000000000001E4090000040E800104798003B
:10F0D0001E409000E14F4000ECFF3A00C902A90039
:10F0E0001E80FB000080FA00000006000400FA0009
:10F0F000004F780010C0B3007D0007000004E0005E
:10F100000300320020002000100798001300370091
:10F110009E40780061C06000614060000041400096
:10F12000912C200091407800D0CFB30000C0600047
:10F1300002407000C9E2B7000040EB006C0007001D
:10F140000004E000030032002000200010079800B7
:10F15000020037008000EB00110798001E009000AD
:10F160000080FA00000006000800FA0040479800FE
:10F170000040EB0020479800C902A900CB02A9007B
:10F18000C00320008E98020000000000CB22A900DE
:10F19000C922A900C902A800100020008E98020010
:10F1A000000000000040EB00510007000004E000F8
:10F1B000030032004000200030079800490037006B
:10F1C0000000EB00000F78001C0037004E4090005C
:10F1D0000080FB00610060000004E0000B003200D2
:10F1E00010C0B300C1FF07000004E00003003200BC
:10F1F00040002000300798003A0037002E40900071
:10F200000004A20020479800070037000040EB00F0
:10F21000B6FF07000004E0000300320040002000B9
:10F22000300798002F0037004E4090000080FB0010
:10F230000000D100404798001E0FE8007000200039
:10F240009E0F1000E1FF36002E4090000004A20047
:10F25000204798002E409000A4FF07000004E00023
:10F260000300320040002000300798001D003700E6
:10F27000C922A800CB22A90010C0B3001C000700BF
:10F280000004E00003003200400020003007980036
:10F2900014003700D2FE0700E24F500003003A008E
:10F2A00040002000300798000E003700CCFE070019
:10F2B0000080FB00000F7800200020009E0F10004F
:10F2C00003003A0040002000300798000500370096
:10F2D000C902A900CB02A9001E0078000080FB0033
:10F2E000300798003E0090000080FA000000060001
:10F2F0000600FA00204798000080EB00000F78001D
:10F30000CBC2BF00614060008080FB002E409000B7
:10F310000080FB00808F500003003A000000EB00EB
:10F3200020079800050037001E0FE9001E00E000CE
:10F33000F3FF3A0010002000200798002E009000F4
:10F340000080FA00000006000600FA000000EB0052
:10F35000800888000000EB00F00888000000EB0047
:10F36000E00C8800306180000000E00008003A00F6
:10F37000A16C20009140780000CEB30000C0600076
:10F38000CAE6B7000000EB00C06088003D0037000F
:10F3900030618000E30F500005003C00E0032000D6
:10F3A000000F780010A1A8001081A80015003700F8
:10F3B00030618000FE0F500005003C00A00F2000CF
:10F3C000000F780010A1A8001081A9000D003700DF
:10F3D00031618000400F2000808F500005003C000C
:10F3E000007D2000000F780010A1A9001081A80066
:10F3F0000400370000E82300000F780010A1A900E6
:10F400001081A90030618000000178001E007800A2
:10F41000110009000280D8000000E90020079800D0
:10F420002E00900060088800406180008000780015
:10F430002E0090000088B90042062000110009004B
:10F440000280D80010079800A16C2000914078003D
:10F4500000CEB30000C060006041B300CAE6B70050
:10F460001E009000D00C88001E009000C00C880088
:10F4700060002000E00C880011E1A80020002000BE
:10F48000C06088000080FA00000006001200FA0048
:10F490000000EB00800888000000EB00F008880006
:10F4A0000000EB00E00C8800C0608000E20F50001C
:10F4B00014003A00A16C20009140780000CEB30007
:10F4C00000C06000CAE6B700C1002000C02E2000C6
:10F4D000E09D0200000000000000EB00C06088001A
:10F4E000606980008000E800F00F200080806000EC
:10F4F000A0C2200000804000104078000004E0001E
:10F50000AE0032000000EB00200798006069800028
:10F510000000E8006069880061698000F00F200049
:10F520000080600060698800661A02000000000028
:10F53000901602000000000040079800661A0200C2
:10F54000000000009016020000000000CF80DE00E6
:10F55000F803020000000000008FBE004E00900083
:10F560000000E00007003200CE009000F0F920001B
:10F57000808F500003003E002E0090000000E80045
:10F58000200798006011B8001E00BE004E04020063
:10F59000000000000000E00001003C000B0037000C
:10F5A00002002000832C24001E00BE005204020032
:10F5B000000000000000E0000100350003003700FB
:10F5C0002E0090000000E800200798002E00900018
:10F5D000E20F5000110032000000EB00706988005B
:10F5E00011012000802F2000E09D0200000000009B
:10F5F0001101200090302000569D02000000000004
:10F600008001EB0002FA20001100200020032000FE
:10F61000DC1C020000000000400798004E00900033
:10F62000E30F500005003E00E00320003007980083
:10F6300010A1A8001081A800150037004E0090000E
:10F64000FE0F500005003E00A00F2000300798007C
:10F6500010A1A8001081A9000D003700CE00900075
:10F66000400F2000808F500005003E00007D2000EC
:10F670003007980010A1A9001081A80004003700ED
:10F6800000E823003007980010A1A9001081A9000C
:10F690003E0090004E019000110009000280D80049
:10F6A0000000E900600798002E009000E20F500073
:10F6B0000E0032000101200070322000569D020031
:10F6C000000000008001EB00320620008000EB000B
:10F6D00020032000DC1C020000000000CF80DE00C0
:10F6E000F803020000000000008FBE0002002000AE
:10F6F000832C24001E00BE005604020000000000FF
:10F70000008FBE006E009000CF80DE00F803020084
:10F710000000000070079800010F98006E00900034
:10F720000000E00008003D000200200003782400F3
:10F730007E0090008E089000DC04020000000000B3
:10F7400070079800010F98001E01BE007E00900017
:10F750008E0890009605020000000000FE050200E1
:10F760000000000050079800A16C20009140780034
:10F7700000CEB30000C060006041B300CAE6B7002D
:10F780005E009000D00C88005E009000C00C8800E5
:10F7900060002000E00C88006E0090006008880087
:10F7A00011E1A800A100200070332000E09D0200BC
:10F7B0000000000020002000C06088000080FA00E7
:10F7C000000006000000FA00C0608000E20F500058
:10F7D00005003A00F101200010342000E09D0200F5
:10F7E000000000003E003700F1002000003620003D
:10F7F000569D0200000000000000EB00F0088800A9
:10F800000000EB0080088800C942A8006168200061
:10F810009140780000CEB30000C06000A040B3006B
:10F8200086E6B700A0032000800888002E000700AD
:10F83000D0608800E1608800D2608000E3608000D2
:10F84000F00F200001002000800F5100818F59002F
:10F8500009003600D0608000E1608000C808DD004B
:10F860000080FD00804078000040EB00D060880000
:10F87000E160880009003700B1002000B0192100C4
:10F88000569D020000000000A000200080088800B3
:10F8900015000700D0608800E1608800D06080001B
:10F8A000E1608000FE6C020000000000C0A528009E
:10F8B000D86B02000000000000A62800046C0200C3
:10F8C0000000000086C6BF00F041B30086E6B70026
:10F8D0000000EB00F00888000000EB0080088800C2
:10F8E0000080FA00000006000000FA000080EB0033
:10F8F000700888000080EB00600888000000EB00C2
:10F90000400888000000EB00300888000000EB0091
:10F91000B00888000000EB00A008880080002000EC
:10F92000F0088800400F2000E00888000040220016
:10F93000D00888008780A9001FE1A80011E1A80075
:10F9400087C0BF00704060000004E000FCFF320090
:10F9500011E1A9001FE1A9003008800020618800A2
:10F9600040088000106188001061800001002000C4
:10F97000F060880001618800F06080000161800013
:10F98000C000DD0000002000F060880001618800F8
:10F99000206180006101B800F0608000016180009A
:10F9A0000200400083804800F06088000161880008
:10F9B000F0608000016180000080FA000000060015
:10F9C0000000FA0090B7200010407800614060000D
:10F9D0000004E00002003A00C942A800010037001C
:10F9E000C8C2A800E1002000F0362000569D0200A9
:10F9F000000000000080FA00000006000000FA008D
:10FA000090B7200010407800614060000004E000E2
:10FA100003003A00C942A900CB42A8000200370007
:10FA2000C8C2A900CAC2A80081002000D0372000A7
:10FA3000E09D0200000000000080FA0000000600C7
:10FA40000000FA0090B7200010407800614060008C
:10FA50000004E00003003A00C942A900CB42A9001B
:10FA600002003700C8C2A900CAC2A9007100200064
:10FA700050382000E09D0200000000000080FA00E5
:10FA8000000006000200FA0090B720001040780045
:10FA9000614060000004E00009003A00C942A8008B
:10FAA0000000000000000000CBC2BF000080FB008F
:10FAB0004200DE0061406000004F7800080037001F
:10FAC000C8C2A8000000000000000000CAC2BF00B9
:10FAD0000080FB004600DE0061406000004F7800BF
:10FAE0001E80FB000080FA00000006000400FA00FF
:10FAF000004F780011479800E0DD20001E48780094
:10FB000030C0B3009E4F100005003A0000202000D6
:10FB1000006F880000082000106F88000400370084
:10FB200000202000006F880000202000106F880057
:10FB30001E4090000080FB00100798001E009000FF
:10FB4000E10F5000110032001E009000E20F500043
:10FB5000180032001E0090000000E000010032009A
:10FB60001E00370041C1B30040DE2000014878008C
:10FB700041C6B30050DE20000148780021C3B30025
:10FB800060DE2000014878001D00370021C0B3006E
:10FB900040DE200001487800A1C0B30050DE200004
:10FBA0000148780051C0B30060DE200001487800B1
:10FBB0001300370011C0B30040DE20000148780078
:10FBC00051C0B30050DE20000148780021C0B300CE
:10FBD00060DE200001487800090037008040EB001B
:10FBE00040DE2000014878008040EB0050DE20001D
:10FBF000014878008040EB0060DE2000014878007A
:10FC00000080FA00000006000200FA000000EB008D
:10FC1000000F780050DE2000904078000030200077
:10FC200009010700CBC2BF00614060000004E00092
:10FC300004003200CBC2BF00624060000004E0005C
:10FC400002003A0010002000000F780050DE200073
:10FC500090407800002020001701070050DE2000AF
:10FC600090407800001020001301070050DE2000B3
:10FC70009040780000202000F30007001E0078006C
:10FC80000080FA00000006000000FA0050DE2000AC
:10FC900090407800003020000701070050DE20006F
:10FCA0009040780000102000E700070050DE2000A0
:10FCB0009040780000202000E30007000000EB00E7
:10FCC0000080FA00000006000C00FA0050079800BF
:10FCD0000000EB00000F7800A0B720001040780073
:10FCE0000080FB008000E900100020000100DD0022
:10FCF000300798005E009000200798000000EB009D
:10FD0000400798002000370040DE200010417800B6
:10FD1000AE0090003E0090000080600001202000B6
:10FD2000FC00070050DE200090407800001020000A
:10FD3000C500070000082000260107000080FB0026
:10FD40001007980050DE200090407800001020003E
:10FD5000D90007002E009000000040002007980006
:10FD60001E00780000004000000F78001E00900088
:10FD70000000E000010032001E0FE8004E0090007D
:10FD80000000E80040079800A0B72000104078006D
:10FD90008080FB004E009000808F5000DAFF3E0014
:10FDA0001E0078000080FA00000006000800FA003B
:10FDB00030079800A0B72000104078000080FB00BA
:10FDC0008000E900100020000100DD00100798000D
:10FDD0003E009000000F78000000EB002007980024
:10FDE0001400370040DE2000104178001E00900013
:10FDF0001E00600001202000C600070050DE200029
:10FE000090407800001020008F00070050DE200096
:10FE10009040780000102000A70007001E00780026
:10FE200000004000000F78002E0090000000E80065
:10FE300020079800A0B72000104078008080FB00C9
:10FE40002E009000808F5000E6FF3E000080FA00F8
:10FE5000000006000600FA000000EB00000F78002A
:10FE600000202000DB0007000000EB0020079800C6
:10FE70001600370050DE200090407800001020006F
:10FE80007100070000202000D20007000080FB0066
:10FE90001007980050DE20009040780000102000ED
:10FEA000850007001E00780000004000000F780069
:10FEB0001E0090000000E000010032001E0FE8006C
:10FEC0002E0090000000E80020079800A0B7200056
:10FED000104078008080FB002E009000808F500042
:10FEE000E4FF3E001E0078000080FA0000000600DB
:10FEF0000200FA00106F8000B600070050DE2000FC
:10FF000090407800001020004F000700106F800024
:10FF1000B0000700004F780050DE200090407800CD
:10FF200000102000640007001E80FB000080FA0023
:10FF3000000006000200FA00004F780040DE2000BA
:10FF400010417800016F80001E80FB0071000700E7
:10FF500050DE200090407800001020003A0007009A
:10FF600050DE200090407800001020005200070072
:10FF70000080FA00000006000400FA002047980004
:10FF80000040EB00004F78000900370050DE2000F1
:10FF900090407800001020002B00070050DE200069
:10FFA0009040780000102000430007001E4FE8003A
:10FFB0002E4090009E4F1000F4FF39000080FA00A0
:10FFC000000006000200FA00004F780040DE20002A
:10FFD00010417800016F80001E80FB004D0007007B
:10FFE0000080FA00000006000200FA00004F7800CE
:10FFF00040DE2000104178001E80FB000110200030
:020000040001F9
:10000000440007000080FA00000006000200FA0029
:10001000004F780040DE2000104178001E80FB0079
:10002000010420003B0007000080FA0000000600E9
:100030000000FA00106F8000660007000080FB00DF
:100040000080FA00000006000400FA00000F7800AB
:100050002147980090B72000104078006840600069
:100060000004E0000B003A00601680001E007000E3
:10007000601688001E0078000080EA008180EA0097
:1000800080007800401680000080600040168800E4
:1000900003003700401680001E00700040168800E4
:1000A0002E4090000080FB008E98020000000000AF
:1000B0000080FA00000006000400FA00000F78003B
:1000C000214798001E0078000080EA008180EA0045
:1000D0008000780060168000008060006016880054
:1000E0001E0078000080EA008180EA00800078002D
:1000F0004016800000806000401688002E4090006E
:100100000080FB008E980200000000000080FA00D2
:10011000000006000600FA00000F780011079800A2
:10012000424798001E00E0000F003A001E009000B9
:100130000080EA008180EA0080007800601680007C
:1001400000806000601688001E0090000080EA00B9
:100150008180EA0080007800401680000080600006
:10016000401688001500370090B720001040780036
:10017000684060000004E0000C003A006116800056
:100180001E00900000807000601688001E00900025
:100190000080EA008180EA0080007800401680003C
:1001A0000080600040168800040037004016800080
:1001B0009E00900001007000401688004E409000A4
:1001C0000080FB008E980200000000000080FA0012
:1001D000000006000400FA00000F780040168000BE
:1001E0001E007000401688000000000000000000A3
:1001F00000000000501680001E0060000000E000BB
:1002000003003200100020001007980002003700A1
:100210000000EB00100798001E0090000080FA001C
:10022000000006000000FA002A7F02000000000023
:100230000080FA00000006000200FA00000F7800BB
:100240001E007800D67E0200000000000010200092
:100250000080FA00000006000000FA00047E0200A0
:100260000000000081002000D0922000569D020076
:1002700000000000D100200080442000E09D02002A
:10028000000000000080FA00000006000000FA00F4
:10029000447E020000000000610020005093200016
:1002A000569D020000000000C100200050452000C3
:1002B000E09D0200000000000080FA00000006003F
:1002C0000000FA00787F0200000000000080FB00C0
:1002D0000080FA00000006000000FA00188002000A
:1002E000000000000080FB000080FA000000060013
:1002F0000000FA000040EB00F47F02000000000064
:100300000080FA00000006000000FA0010C0B300F0
:10031000F47F0200000000000080FA0000000600E8
:100320000000FA0010C0B300BC7F02000000000013
:100330000080FA00000006000000FA000040EB0018
:10034000E27F0200000000000080FA0000000600CA
:100350000000FA0010C0B300E27F020000000000BD
:100360000080FA00000006000000FA0001012000F1
:10037000A0982000569D02000000000080B72000D9
:1003800010407800706E02000000000000C2B30050
:10039000347002000000000090B720001040780088
:1003A0000080FB004300DE0061406000706E0200D0
:1003B0000000000000C2B300347002000000000022
:1003C00031002000F0AD2000569D0200000000002A
:1003D0000080FA00000006000400FA00661A02001D
:1003E00000000000901602000000000010079800B6
:1003F000661A0200000000009016020000000000D3
:10040000000F78001E0090000000E000090034009A
:100410001E009000E40F500006003C001E009000FB
:100420000040E9008040780080B720000148780053
:10043000020037000000EB00100798001E00E000EB
:1004400010003400200020009E0F10000D003C0022
:100450001E0078000040EA006141600090B7200073
:1004600090407800614061004301DD0070CFB3002F
:1004700080C0600082C0700090B720000148780002
:10048000020037000000EB00100798001E009000EB
:100490000000E00026003A000000EB0070698800D0
:1004A000B103200060482000E09D02000000000031
:1004B0008001EB004200200011002000100020000D
:1004C000DC1C0200000000000040E90080407800D1
:1004D00080B7200001487800F1042000B09320008C
:1004E000E09D0200000000008001EB0022002000DF
:1004F0001100200010002000DC1C020000000000A1
:100500000040EA006141600090B720009040780010
:10051000614061004301DD0070CFB30080C0600026
:1005200082C0700090B720000148780001003700B9
:100530008DFF0700CB02A900CB22A900C922A80089
:10054000C902A90080B720009040780020C0B30005
:10055000767D0200000000000080FA000000060026
:100560000400FA00000F78001E00780010079800C1
:100570001E009000E10F50000C0032001E009000A1
:10058000E10F5000040039001E009000E20F5000FF
:10059000070032000800370081032000A0992000E6
:1005A000569D020000000000070037001000070001
:1005B000250007000400370041022000C020200071
:1005C000E09D0200000000000080FA00000006002C
:1005D0000200FA00000F7800B1002000C0092100DD
:1005E000E09D0200000000000080FA00000006000C
:1005F0000000FA00F1032000209D2000E09D020091
:10060000000000000040EB00068002000000000037
:10061000F00F20008E9802000000000010C0B30010
:10062000068002000000000010C0B300BC7F020082
:10063000000000000040EB00068002000000000007
:100640000080FA00000006000A00FA00881F780007
:10065000D102200010A12000569D020000000000E1
:100660000000EB00000F7800100037001E04780037
:100670002A7F0200000000008040780063004700ED
:10068000017478009E0078006300470061407800A4
:100690000080FB00D26E02000000000000C2B30028
:1006A00034700200000000001E0FE800300020003F
:1006B0009E0F1000EDFF360020A82800046C0200F9
:1006C00000000000A1002000E0A32000569D0200D1
:1006D0000000000063004700104078000080FB002D
:1006E0004400DE000080FB00400798004E009000B0
:1006F000E90F5000130032004E009000E90F500047
:1007000004003C004E009000E80F5000080032004A
:100710001B0037004E009000EA0F50000E00320020
:100720004E009000EF0F5000100032001400370010
:100730006100200080A42000569D020000000000FF
:100740001300370061002000E0A42000569D020045
:10075000000000000E0037006100200040A52000CE
:10076000569D020000000000090037003100200003
:10077000A0A52000569D02000000000004003700E4
:1007800071002000D0A52000569D0200000000004E
:1007900020A82800046C020000000000B100200026
:1007A00040A62000569D02000000000063004700A4
:1007B000104090000080FB004700DE000004E000D5
:1007C00005003A0061002000F0A62000569D0200BE
:1007D0000000000004003700F100200050A72000B6
:1007E000569D02000000000020A82800046C0200B2
:1007F00000000000C100200040A82000569D02001B
:100800000000000063004700104090008080FB0063
:1008100080F72F00008060004380DE0020479800B2
:100820002E4090000004E00005003A00D1002000B6
:1008300000A92000569D0200000000001E003700A5
:100840002E409000EF4F500005003A00310020008C
:10085000A0A52000569D02000000000016003700F1
:1008600000042000000F7800E30047000040EB0088
:1008700080487800080037001E0078000000400023
:10088000000F780063004700104078008040E800C7
:1008900063004700014878006300470090407800FB
:1008A0002E40900080CF5000F3FF39001E007800EA
:1008B000126E02000000000020A82800046C020054
:1008C0000000000091012000D0A92000569D0200E8
:1008D00000000000630047009040900070C0B3002B
:1008E00000C060002047980010002000000F780032
:1008F000E30047000040EB00804878000800370024
:100900001E00780000004000000F780063004700E0
:10091000104078008040E8006300470001487800FC
:1009200063004700904078002E40900080CF500038
:10093000F3FF39001E007800706E02000000000016
:1009400020A82800046C0200000000004F0478007A
:100950000080FA00000006000600FA001007980068
:10096000210798001E009000000F78003800370023
:100970001E00780032002000110009000200D8009B
:100980008000FD000000E0000B003A001E0078002F
:1009900032002000110009000200D80000004000D1
:1009A0008000780000912900008040001000BA000B
:1009B00034700200000000001E00780032002000A9
:1009C000110009000200D8008000FD00E10F500076
:1009D0000C003A001E0078003200200011000900CF
:1009E0000200D8000000400080007800009129003B
:1009F000008040001000BA004800DE0034700200A1
:100A0000000000001E0078003200200011000900E4
:100A10000200D8008000FD00E20F50000B003A00F9
:100A20001E00780032002000110009000200D800EA
:100A30000000400080007800009129000080400004
:100A40001080BA0034700200000000001E0FE800A1
:100A50001E009000AE009000010040009E0F50006C
:100A6000C3FF3C000080FA00000006000400FA000A
:100A7000000F7800110798009E0090001E0078007B
:100A8000B5FF070020A02800046C02000000000051
:100A90000080FA00000006000600FA00661A020054
:100AA0000000000061698000A0C2200000804000BA
:100AB000104078000000FB0020079800E0062000AE
:100AC000AE009000808F500012003200E00620003F
:100AD000AE009000808F500005003C0050062000C2
:100AE000AE009000808F50001000320015003700DB
:100AF00030072000AE009000808F50000E003200C2
:100B000070072000AE009000808F5000040032007B
:100B10000C0037000000EB00000F780013003700D6
:100B200010002000000F7800100037002000200087
:100B3000000F78000D00370030002000000F780013
:100B40000A00370050002000000F78001101370024
:100B5000606980000000E8006069880061698000C9
:100B6000F00F2000008060006069880061698000EB
:100B7000A0C22000008040009040780000C2B30076
:100B800080CF50000600320061698000A0C22000C2
:100B900000804000104078000004E000ECFF3A00C4
:100BA000B05B80009E0078004200DD0081004000C4
:100BB000E09D280000804000104078000004E00024
:100BC00003003200500020009E0F100004003A0085
:100BD00021012000E00B2000A4FF0700ED003700FA
:100BE000B05B80009E0078004200DD008100400084
:100BF000E09D280000804000104078000080FB004D
:100C0000B05B880081002000600B200052FF0700CD
:100C1000B15B8000110798001E009000E40F5000A7
:100C20004E0032009E009000E48F50000A003C000D
:100C30001E009000E20F5000180032009E0090004D
:100C4000E28F500019003C001E009000E10F5000A0
:100C50000E0032009E0037009E009000E68F50008C
:100C6000520032001E009000E60F50003F00350099
:100C70009E009000E78F5000500032001E00900050
:100C8000E80F500058003200910037009101200019
:100C9000D00E200075FF07008D003700B101200045
:100CA0006010200071FF0700890037003103200029
:100CB000101220006DFF070051002000209220003C
:100CC000569D020000000000C1BF2A000000EB009A
:100CD0004C710200000000002A6F020000000000BA
:100CE0006100200070922000569D0200000000006C
:100CF000E1BF2A000000EB004C7102000000000080
:100D00002A6F02000000000000C2B300347002002D
:100D1000000000006100200000762000569D0200C7
:100D200000000000B04080002A6F020000000000B8
:100D30007100200070EA2000569D020000000000B3
:100D4000C04080002A6F02000000000020A02800A0
:100D5000046C0200000000005D003700110220005A
:100D60004015200041FF07005900370041002000D6
:100D7000501720003DFF070021E3A800A0C0B300EA
:100D80002497020000000000800078000015200079
:100D9000808F500003003600B10220000000EB00FD
:100DA00032FF070021E3A90049003700310220008B
:100DB000901720002DFF070045003700010120009B
:100DC000C019200029FF0700CAC2BF000042B200BC
:100DD0000004E0003E00320021022000B0022000AA
:100DE00022FF07003A00370041022000C01A20000D
:100DF0001EFF070021E3A800A0408000E30F500081
:100E000027003A00CAC2BF000042B2000004E0005E
:100E100023003200A0C0B3002497020000000000AD
:100E20008000780000152000808F50001C003600E4
:100E300051032000D00420000CFF070051032000C4
:100E4000001D200009FF0700710320005020200032
:100E500006FF070071032000C023200003FF0700E6
:100E6000610320003027200000FF0700510320000D
:100E7000902A2000FDFE070041032000E02D200005
:100E8000FAFE07005103200020312000F7FE070082
:100E90004103200070342000F4FE07000B003700EF
:100EA0004103200020082000F0FE07001000200071
:100EB000B05B880081002000600B2000A6FE0700C8
:100EC00091012000D00E2000E8FE070021E3A900D8
:100ED00071002000000D20009FFE0700B05B800025
:100EE000C200DD00E09D2800008040001040780036
:100EF0000004E0000300320061002000700D2000BB
:100F000095FE0700B05B80004200DD008000E80035
:100F1000E09D280000804000104078000004E000C0
:100F20000300320051002000D00D20008AFE07008F
:100F3000B05B80004200DD008080E800E09D28007A
:100F400000804000104078000004E0000300320000
:100F500051002000200E20007FFE0700B05B8000C3
:100F60004200DD00E3004000E09D280000804000DA
:100F7000104078000004E00003003200610020000F
:100F8000700E200074FE070020A02800046C0200F0
:100F9000000000000080FA00000006000000FA00D7
:100FA00040168000017C200001007000401688007F
:100FB0001100070020C0B3002D00070016700200CA
:100FC000000000000004E000050032002270020072
:100FD00000000000260007000004E00004003A00C2
:100FE000360107000004E00001003A00F3FF37007B
:100FF0000080FA00000006000000FA00CA82A90082
:101000000000EB00400388000000EB005003880064
:101010000000EB00000388000000EB0010038800D4
:101020000000EB00F0088800D10A20009140780011
:10103000F0C8B30000C06000ADE0B7000000EB00F6
:10104000E008880000642000D0088800000021002B
:10105000607088008040EB00A0E02000014878002C
:101060000000EB00C06F88000080FA00000006005E
:101070000A00FA00004F78001070800040079800C6
:10108000CE009000E18F5000440032004E019000ED
:10109000E10F5100040039004E009000E20F5000B3
:1010A0004F003200000137009E80FB00310798009E
:1010B0003E019000E20F5100150032003E0090000A
:1010C000E20F500007003C00BE0090000100E0006D
:1010D0000B0032003E019000E10F51001000320081
:1010E000230037003E009000F10F5000EE00320068
:1010F000BE009000F38F5000EB0032001C00370060
:10110000BDFF07001200200022079800E80037000A
:1011100040A72800D86B020000000000E200370062
:10112000CA82A8000000EB00F00888000000EB0075
:10113000B00888000000EB00A008880080002000B4
:10114000F00888008660A9009660A900D10A2000F6
:1011500091407800F0C8B30000C060000044A000D7
:10116000ADE0B70010002000C06F8800CE0037004F
:10117000A0DF20001E48780041C0B300F0DF20004F
:10118000014878008040EB0000E020000148780032
:101190001000200010708800C300370000E020001D
:1011A000104078008040E80000E02000014878000E
:1011B00000E02000104078008080FB00A0DF2000CD
:1011C000008040001E48780000E020009040780039
:1011D000F0DF20001040780080CF5000B2003900CE
:1011E000A0DF2000104078000080FB00100798006E
:1011F000100820009E009000808F50003E003200BA
:10120000000C20001E019000800F510005003200EC
:10121000000820009E009000808F50004E00320099
:101220009F003700B0DF2000104078000080FB00F6
:101230004400DE00610060000004E00003003200B2
:10124000100380000000A00010038800B0DF200021
:10125000104078000080FB004300DE006100600069
:101260000004E000040032001003800001022000AE
:101270000100700010038800B0DF200010407800EB
:101280000080FB004200DE00610060000004E0001E
:1012900004003200100380000104200001007000EF
:1012A00010038800B0DF2000104078000080FB00B1
:1012B0000000D100610060000004E0000400320082
:1012C0001003800001082000010070001003880056
:1012D000B0DF2000104078000080FB00610060005B
:1012E0000004E00004003200100380000110200020
:1012F0000100700010038800C0DF2000104078005B
:101300000080FB0060708800607080004800DD0095
:1013100060708800B0DF2000104078008080FB0003
:1013200060708000008070006070880060708000D5
:101330004200DD0064004000607088006170800041
:1013400000002100808F5000550036000000210071
:101350006070880052003700D0DF20001040780015
:101360000080FB00010020002070880031708800A0
:101370002070800031708000C808DD000080FD0012
:10138000804078000040EB002070880031708800B9
:10139000C0DF2000104078000081FB000300200027
:1013A0002070800031708000000071008180710029
:1013B00020708800317088002070800031708000BB
:1013C000C808DD000080FD00804078000040EB0090
:1013D0002070880031708800B0DF20001040780055
:1013E0000081FB000300200020708000317080002D
:1013F00000007100818071002070880031708800C9
:1014000020708000317080004209DD00CE00DE00D7
:10141000810071004200DD0064004000E08048006F
:1014200092012000030020003406020000000000AA
:101430002070880031708800227080003370800036
:101440000001200001002000800F5100818F590011
:10145000070036002070800031708000700050005E
:10146000E080580020708800317088000400370048
:1014700010002000010020002070880031708800DA
:1014800020708000317080004008DE0001002000E4
:10149000E00888002070800031708000D00888004B
:1014A0000000EB00107088000000EB00200798009F
:1014B0002E0090000080FA00000006000200FA00F2
:1014C000C06F8000E10F500001003200360037008D
:1014D00086C0BF00684060000004E00003003A00DE
:1014E000100380000000E0002F003A001FE1A80078
:1014F0008780A9000000EB00407088000E003700D4
:101500007140800040708000808040005016800054
:101510004600DE008048780087C0BF007040600051
:101520000004E000FCFF32008780A90040708000CA
:101530000000E8004070880041708000607080000A
:10154000808F5000EEFF39000000EB001003880090
:101550000000EB00F0088800607080004070880098
:101560000A00370071408000407080000080400019
:101570000000E90010407800347002000000000014
:10158000407080000000E9004070880040708000DA
:101590000000E000F3FF3A0097FE07001000200073
:1015A000000F7800020037000000EB00000F780009
:1015B0001E0078000080FA00000006000200FA0019
:1015C000000F78001E00780080407800602721001E
:1015D000104078000080FB000000D10061406000F6
:1015E00046010700001020000080FA0000000600FD
:1015F0000000FA0060272100104078000010A100D0
:10160000612721008048780041012000B0EC2000D3
:10161000E09D0200000000000080FA0000000600CB
:101620000000FA0060272100104078000010A000A0
:10163000612721008048780021012000F0ED200082
:10164000E09D0200000000000080FA00000006009B
:101650000000FA0090B72000104078000030A00091
:1016600091B7200080487800602721001040780062
:101670000010A0006127210080487800816A2000C6
:101680009140780000CEB30000C060007040B3000D
:10169000A8E6B700916C20009140780000CEB3001E
:1016A00000C060007040B300C9E6B700816C200044
:1016B0009140780000CEB30000C060000034A0006C
:1016C000C8E6B700CAC2A900C8C2A900C902A900D9
:1016D000C8E2A800C922A900D01320001012880077
:1016E0000000EB00201288000000EB0000128800D0
:1016F00041E2A800D101200040F02000E09D02005E
:10170000000000000080FA00000006000800FA0057
:1017100020079800606980000000E8006069880088
:1017200061698000F00F200000806000606988001F
:10173000661A02000000000090160200000000007F
:10174000100798000000EB00706988002E009000E0
:10175000300798003E009000E30F50003C0032003C
:101760003E009000E30F500004003E003E00900059
:101770000000E0000B0032000F0037003E00900038
:10178000E60F5000480032003E009000E70F500086
:101790006A0032003E009000E40F50003700320033
:1017A0008B0037008109200060F62000E09D0200D8
:1017B000000000008A003700510020003063200044
:1017C000E09D020000000000AC0007002E00900029
:1017D000E10F5000820032001E0090000000E00087
:1017E000030034001E009000E20F5000130034008C
:1017F00041022000E0FF2000E09D02000000000008
:101800008001EB00220020001100200020002000B9
:10181000DC1C020000000000100798001E00900071
:10182000E10F500003003A000040EB007500070094
:101830000200370080C0B3007200070041002000A2
:1018400020022100E09D020000000000640037003B
:1018500011C0B3000040EB00A8000700F00020001A
:101860006298020000000000510020006002210088
:10187000E09D020000000000590037001E009000AB
:101880008040780000C8B30080C070000040EB00CA
:101890009A000700A1002000B0022100E09D020094
:1018A000000000004E00370011C0B3000040EB0004
:1018B00092000700F0002000629802000000000083
:1018C00000032000200798001E0090000000E000A8
:1018D00002003A0000052000100798000000EB000D
:1018E000000F780011003700AE0090009003200038
:1018F000808F50000200360000032000200798006F
:101900002E0090008040780010C0B3007B000700DC
:101910002E00900034700200000000002E009000A5
:101920000000E800200798001E0FE8001E0090004D
:101930009E0F1000ECFF35002900370011C0B300E6
:101940000040EB006D000700F000200062980200EC
:101950000000000010022000200798001E009000E8
:101960000000E00002003A00000520001007980087
:101970000000EB00000F780011003700AE0090006F
:10198000F0072000808F5000020036001002200077
:10199000200798002E0090008040780010C0B3000F
:1019A000560007002E009000347002000000000076
:1019B0002E0090000000E800200798001E0FE800AD
:1019C0001E0090009E0F1000ECFF35000400370051
:1019D00041022000C0202000E09D02000000000025
:1019E0000080FA00000006000000FA00B1002000AC
:1019F000C0092100E09D0200000000000080FA0004
:101A0000000006000200FA00004F78001E40780037
:101A10000042B000804078000040EB003700070033
:101A2000F0002000629802000000000081C0B300B6
:101A30000040EB0031000700F00020006298020037
:101A40000000000011C0B3000040EB002B000700B5
:101A5000F00020006298020000000000E1C0B30026
:101A60000040EB0025000700F00020006298020013
:101A7000000000000080FA00000006000000FA00EC
:101A80000040EB004A000700F000200062980200CE
:101A90000000000031C0B3000040EB00260007004A
:101AA00050002000629802000000000031C0B30026
:101AB0000040EB0020000700000A20008E98020082
:101AC0000000000031C0B3000040EB001A00070026
:101AD000000A20008E9802000000000021C0B30020
:101AE0000040EB0014000700000A20008E9802005E
:101AF000000000000080FA00000006000200FA006A
:101B0000004F7800114798001E4090000080FB00B5
:101B10004400DE00804078001E4078000600070088
:101B20001E409000EF4060001E4078000200070059
:101B30000080FA00000006000200FA00004F780062
:101B4000114798001E4090004400DD0010479800A7
:101B50001E4090000004A0001047980010C0B30081
:101B60009E4F100003003A001E4090000014A00099
:101B7000104798001E4090000D0007001E40900086
:101B80000034A000104798001E4090000800070095
:101B90009E40900070CFB30000C0600010479800D6
:101BA0001E409000020007000080FA0000000600BE
:101BB0000200FA00004F78001E4078004247020001
:101BC00000000000CAC2A800CAC2A9000080FA0032
:101BD000000006000C0800001200000002000000D7
:101BE00000007E0012000000000000000000000065
:101BF0000000000000000000780B00001C00000046
:101C0000000000007E120000001000000000000034
:101C1000940B000002000000000000001E080000FD
:101C20000C0000000200000000181C001D0018003D
:101C30001C1D030008101800960B00000600000091
:101C4000000000002A08000012000000020000004E
:101C5000143404000D8206004003A00001CF0000F0
:101C600067004400002200009C0B000008000000F8
:101C700000000000A40B00000400000000000000B1
:101C80003C0800000201000002000000F0005E00BD
:101C9000BCE261003FDD8300C29C7E0020A3FD000A
:101CA0001F419D00C3217F00FCA240001E5F010078
:101CB000E3BD3E006082DC00237D9F00C1421C002A
:101CC000FEA0E100BF5D030080DE3C0062BEE000DC
:101CD000025CDF0081633D007C22C0009E1D43004A
:101CE000A1FF460018FAA40027799B00C584DA00FA
:101CF0003866E500BB590700DB85670039BAE400A8
:101D00000658190047A5FB007826C4009A653B00D9
:101D1000D98704005AB8E600A7F91B0045C6980009
:101D20007A24F800A6441A0099C725007B3A64007B
:101D300086D85B0005E7B9008CD230006EEDB300A9
:101D4000510F4E0010F2AC002F719300CD114F00D7
:101D5000ADF370002ECC9200D38D6F0031B2EC0049
:101D60000E50AF00F1134D00CE9072002C6D330079
:101D7000D18F0C0052B0EE00326C8E00D0530D00AB
:101D8000EFB1F000AE4C120091CF2D0073CA940059
:101D90007628AB00F51749000856B400EA69370009
:101DA000D58B570009EBB50036688A00D495CB0077
:101DB0002977F400AA481600E9B755000B88D60029
:101DC000346A2B007597C9004A14F600A8742A00DB
:101DD000C89615004BA9F700B6E80A0054D7890049
:101DE0006B350000A80B0000700000000000000030
:101DF000180C000012000000000000003E09000066
:101E0000CC01000002000000A29FA2009FA29F0040
:101E1000A29FB4009FCA9F00A29FA2009FA29F0002
:101E2000A29FCA009FA29F00CA9FCA009FDE9F0078
:101E3000F29F0800A01EA0002CA04800695A0000D4
:101E40000000000000F45800F458A2009FA29F0078
:101E50007455680055A29F00A29FBE0055AA550068
:101E60009E55900055845500CA9FF40055D25500E8
:101E700008A0E600582CA000312D5700495245001B
:101E800000007A00507A5000A450A40050584C0032
